:020000040800F2
:1000000000000220B90406085D9C0008CD6F0208BC
:10001000690506086905060869050608000000006C
:1000200000000000000000000000000021B10008F6
:1000300023B100080000000025B10008F5150108F3
:1000400069050608690506086905060869050608C0
:10005000690506086905060807FE00080BFE00088A
:10006000690506080FFE000813FE000805A3000836
:1000700019A300082DA3000841A3000855A30008F8
:1000800069A300087DA300086905060800000000B8
:1000900000000000000000000000000017FE000843
:1000A0003DA2000865A200088DA2000827A2000852
:1000B000B5A20008C9A20008DDA20008690506086B
:1000C0006905060869050608690506086905060840
:1000D00069050608799D0008859D0008000000005C
:1000E0001BFE00086905060827B100080000000093
:1000F00000000000000000000000000091A30008C4
:100100000000000069050608F1A20008690506085C
:1001100000000000000000000000000000000000DF
:10012000A5A30008B9A30008CDA30008E1A3000817
:10013000F5A300080000000000000000000000001F
:1001400000000000000000000000000071B1000885
:1001500009A400081DA4000831A4000869050608C8
:100160006905060869050608000000000000000097
:10017000000000000000000000000000000000007F
:1001800000000000690506080000000000000000F3
:0801900069050608690506086F
:0801980058F50500010000000C
:1001A000CC6701200201000002001400EC6701206E
:1001B00002020000020014000C680120020A000084
:1001C000020014002C680120020600000200140046
:1001D0004C68012002070000020014006C68012036
:1001E00002030000040014008C68012002080000D3
:1001F00004001400AC680120010B0000000077002F
:10020000CC680120010C000000007600EC680120A1
:1002100001100000000076000C690120010D0100B2
:10022000000077002C690120011200000000760018
:100230004C6901200114000000001E006C690120BF
:10024000011A000000000D008C690120011C000053
:1002500000000E00AC690120011D000000001E001E
:10026000CC6901200117000000000C00EC6901209E
:100270000118000000000E000C6A01200129010095
:10028000000018002C6A0120012100000000480035
:100290004C6A012001220000000049006C6A012024
:1002A0000123000000004A008C6A012001240000A4
:1002B00000004B00AC6A01200125000000004C004A
:1002C000CC6A01200126000000004D00EC6A0120EC
:1002D0000127000000004E000C6B012001280000E7
:1002E00000004F002C6B0120012C000000002900B1
:1002F0004C6B0120012D0100000029006C6B0120D6
:10030000012E0100000070008C6B01200130000004
:1003100000003100AC6B0120012F010000005200F1
:10032000CC6B01200131010000002800EC6B0120A2
:1003300001320100000028000C6C0120023604008C
:1003400000012C002C6C01200135000000003C0055
:0C0350004C6C012001380000000020006F
:10800000D0E907239A423CBFC1685218D01A704782
:10801000D0E9092300699A4238BF1218D31A0138EF
:10802000C01A7047D0E90902131A584258417047E4
:10803000036A41690246C85CD16801338B4228BF9C
:10804000002313627047436A8269D154436A02690C
:108050000133934228BF0023426B4362D36843F04D
:108060008003D3607047436B188810F010001EBF68
:108070001A889B8801207047436B99891A88890662
:1080800010B592B2044607D5900605D5E26A2AB328
:108090009888216B80B29047636B99891A8809068A
:1080A00092B210D510060ED5D4E909128A4223D017
:1080B000A169895CC9B2998021690132B2FBF1F0F2
:1080C00001FB1022A262998A1A88C90592B204D5CE
:1080D000D20744BF4FF6F7721A8010BD9B88E26941
:1080E0006169DBB28B54E369E2680133B3FBF2F1FF
:1080F00002FB1133E361CFE7DA6822F08002DA6035
:10810000E1E7036941681F2B30B54FF0200285BFBE
:10811000A3F120054C680C68AA4098BF9A402242FF
:108120001DD0826900201074D0688468206820F017
:1081300001002060546820686579094C828934F810
:10814000154092B21F2B22EA0402828188BF203B95
:108150004FF020028BBF9A409A40CA608A6030BDBF
:10816000407506080E4BDA68D20310D4DA68D106DF
:108170000FD4DA68D2050ED4DA6812F0E00F0CD111
:10818000DB6813F0020F0CBF0920082070470120A4
:10819000704706207047022070470720704700BFD5
:1081A000003C024007B509238DF80730FFF7DAFFDE
:1081B0008DF807009DF80730012BF7D09DF80700D8
:1081C00003B05DF804FB838A028B9BB243EA02434F
:1081D00099430CBF01200020704782B00023019317
:1081E0000093012300900193019B63B1009A21F059
:1081F0007F4314320092009A12681A4214BF012081
:10820000002002B07047009A1832F3E770477047B9
:10821000704701207047034BD3E90003C01AC0F335
:108220000A007047901A0020054AD2E900138B42D9
:10823000FDD0D1180133C3F30A03087A53607047A5
:10824000901A0020044BD3F8080820B1D3F808088E
:10825000431F584258417047901A0020012380F86C
:1082600049307047044BD3E90003C01AC0F30A0039
:10827000C0F50060704700BF901A002010B5D0F81C
:10828000E83504461B699847032384F8123100201F
:1082900010BD08B590F8123180F81331042380F82E
:1082A0001231D0F8E835DB689847002008BD08B5E2
:1082B000D0F8E435DB6903B19847002008BD08B564
:1082C000D0F8E4351B6A9847002008BD08B5D0F8FF
:1082D000E4355B6A9847002008BD70B504460D463A
:1082E000164657F065FAC3B201335B0033802B703A
:1082F00003236B70601E0223002410F8011F01B9D4
:1083000070BD5A1CD2B2E9540233AC54DBB2F4E76C
:1083100010B5074C2068FF2808D00649D1F80C2872
:1083200001F5016100F07CF8FF232360002010BDFF
:1083300000000020901A0020432301480B80704762
:1083400004000020122301480B80704747000020E2
:10835000042301480B8070475900002010B5044CDD
:1083600004480A462146FFF7B8FF204610BD00BF6B
:10837000A82200202020070810B5044C04480A4613
:108380002146FFF7AAFF204610BD00BFA82200200B
:108390003320070810B5044C04480A462146FFF76D
:1083A0009CFF204610BD00BFA822002038200708EF
:1083B00010B5044C04480A462146FFF78EFF2046BC
:1083C00010BD00BFA82200204220070810B5044CB1
:1083D00004480A462146FFF780FF204610BD00BF33
:1083E000A82200204D20070870477047704770474B
:1083F000704770477047054B00200522C3F80828D6
:10840000C3F81809C3F81C09704700BF901A002070
:10841000024B0020C3F80808704700BF901A0020E4
:10842000212838B50C461BD022282BD0202815D166
:10843000A1B1072A12D11A4DD5F81C3913B1096818
:10844000002098472368C5F82039237985F8243916
:10845000637985F82539A37985F82639002038BD58
:108460000029FBD0072AF9D10D4BD3F820290A6047
:1084700093F824290A7193F825294A7193F826392B
:108480008B71EBE70029E9D0022AE7D1044BD3F83E
:108490001839002BE2D0098800209847DEE700BF9A
:1084A000901A002030B50E4CD4E900329A1AC2F36B
:1084B0000A020A44B2F5006F10D80144002281423A
:1084C00003D102B12360002030BDE21810F8015B37
:1084D00015720133C3F30A030122F0E70220F3E728
:1084E000901A0020034BD3F8280908B103691847F4
:1084F000704700BF901A0020034B93F850090038D2
:1085000018BF0120704700BF901A0020034B93F85A
:108510005009032894BF002001207047901A0020C2
:1085200000487047E4230020837B042B0DD0074BC9
:10853000D3F898200132C3F8982042600422827355
:10854000D3F89C200132C3F89C207047C05E002005
:10855000202301480B8070475D0000201223014852
:108560000B8070477D000020042301480B8070477A
:108570008F0000200A4608B5044920B90448FFF7D7
:10858000ACFE024808BD0348F9E700BF14240020F0
:108590005B2007087320070810B5044C04480A46FE
:1085A0002146FFF79AFE204610BD00BF142400208C
:1085B0008B20070810B5044C04480A462146FFF7F3
:1085C0008CFE204610BD00BF142400209E2007080A
:1085D00010B5044C04480A462146FFF77EFE2046AB
:1085E00010BD00BF14240020A9200708002370B587
:1085F0004D1C1E46040FB0F1204F34BF30343734C9
:1086000001F8134005F813600133DCB2A2424FEACF
:108610000010EFD870BD1A2310B50B80094BD3F8AA
:10862000E807D3F8EC2780180AD0D3F8EA470649C0
:108630000822FFF7DBFF042210312046FFF7D6FFA8
:10864000024810BD00F0FF1F95000020930000209D
:1086500008B5FFF747FF013840B208BD002070475A
:108660000020704770477047D0ED007AD0ED036A64
:1086700030EE677AE6EE877AB0EE670AC0ED007AF0
:10868000704790ED017AB5EE407AF1EE10FAF0EE17
:10869000407A09D19FED0E7A60EE870AF7EE006A04
:1086A00086EEA07A80ED017A90ED017A90ED000AD5
:1086B00080ED021A31EE077A77EEC07AC1EE076AD2
:1086C000A6EEA70AC0ED036A80ED000A704700BF5E
:1086D000DB0FC940D0ED056AD0ED017A90ED026A5A
:1086E000D0ED045AB0EE407A26EEA70AD0ED007A1B
:1086F00080ED057AA7EE870AD0ED067AC0ED066A0E
:10870000A6EE270AD0ED077A90ED036AA6EE670A77
:1087100090ED086AC0ED087AA5EEC60A80ED070A5A
:108720007047B0EE407AD0ED007A90ED050AD0EDBA
:10873000016AA7EE870AD0ED037A67EEC07AE6EE0B
:10874000877AD0ED066A76EEA77AD0ED026AC0EDA0
:10875000057AD0ED047A67EEC07AE6EE877AC0ED4E
:10876000067A704703685A1C0260197070472DE939
:10877000F04F87B083680193D0E90032511C91FB20
:10878000F3F403FB1411416000EB820181ED200A38
:10879000B1EE400A00F18005009281ED400A00F53B
:1087A0008070A3F1020E4FF0010C019A6245009A0D
:1087B00017DA01991A44521A92FBF3F103FB1122C2
:1087C00005EB820500EB8200D5ED007A90ED007A92
:1087D00077EEC77AB6EE000A27EE800A07B0BDE84A
:1087E000F08F0EEB020494FBF3F103FB1144611CC8
:1087F00091FBF3F603FB161105EB840600EB8404F2
:1088000094ED007A03940CEB0104D6ED007A029605
:1088100094FBF3F603FB1644F246F14626460F4658
:10882000A3EB0C0BD9450CDB029AD2ED007A039A2C
:1088300092ED007ADA454EDB0CF1010CAEF1020E3E
:10884000B3E7BB42D8BF002705EB8702D2ED006A31
:108850000492B342D8BF002600EB8702F4EEE76A29
:1088600092ED006A0592F1EE10FA00EB8602D2ED6D
:10887000005A4FEA860811DDA84498ED005AF4EE3C
:10888000C56AF1EE10FA09DDB4EEE75A049AF1EE8A
:1088900010FA58BFF0EE457AC2ED007AB4EEC76A1E
:1088A000F1EE10FA0EDDB4EEE56AF1EE10FA09DD34
:1088B000F4EEC75A059AF1EE10FA58BFB0EE657A99
:1088C00082ED007A0137013609F10109B0EE467AEE
:1088D000F0EE667AA6E78B42D8BF002105EB81084F
:1088E000D8ED006AA342D8BF0024F4EEE76A00EB9B
:1088F000810700EB8409F1EE10FA97ED006AD9EDDB
:10890000005A4FEA840610D52E4496ED005AF4EE34
:10891000C56AF1EE10FA08D5B4EEE75AF1EE10FA96
:10892000D8BFF0EE457AC8ED007AB4EEC76AF1EE32
:1089300010FA0DD5B4EEE56AF1EE10FA08D5F4EEB2
:10894000C75AF1EE10FAD8BFB0EE657A87ED007A1B
:10895000013101340AF1010AB0EE467AF0EE667A8E
:1089600068E703690133012B036108D1DFED107A59
:1089700080ED010A80ED000AC0ED027A704790EDAB
:10898000006A07EE903A70EE466AF8EEE77A86EEF5
:10899000A77AD0ED027A37EE067A30EE470A80EDFC
:1089A000017AE6EE807AB0EE470AC0ED037AE1E79D
:1089B0000000000003685A1C0260197070470079BB
:1089C00070470079C0F34010704700794009704744
:1089D0002DE9F843D0F8148007468946B8F1000F16
:1089E00057D10568C5F30D0606B3D9F80060FFF747
:1089F000D9FB092840F08680444C236923F4407356
:108A00002361236943F400732361236943F0010365
:108A100023612E60FFF7C6FB2369092823F00103B9
:108A200023616FD13B6804333B6032E0384B9D4299
:108A300029D303F580439D4224D303F580439D420F
:108A40002AD3344B9D4229D903F580339D4227D93F
:108A500003F500339D4225D903F500339D4223D908
:108A600003F500339D4221D903F500339D421FD900
:108A700003F580239D421DD9B5F1016F1CD305205C
:108A80000BF0A2F80826FFF78DFB092816D04FF04F
:108A9000FF384046BDE8F8831026F4E71826F2E7D1
:108AA0002026F0E72826EEE73026ECE73826EAE72E
:108AB0004026E8E74826E6E75826E4E7134C236912
:108AC00023F440732361236943F400732361236912
:108AD00023F0F80323612369334343F00203236146
:108AE000236943F480332361FFF75CFB236923F0A0
:108AF000020323612369092823F0F80323613FF46B
:108B000074AFC4E76FF00108C3E700BF003C024048
:108B100000400008FFFF000803682DE9F0410D4602
:108B2000416813448B42044619D8AE1800F10C0773
:108B30004FF00008B54202D16069BDE8F0812369B9
:108B40005A1C2261234415F8011B1973042AF1D120
:108B500039462046FFF73CFFC4E90480EAE74FF0BE
:108B6000FF30EAE72DE9F0479846444B914603EB86
:108B7000800205469468002C51D02833636004F1CC
:108B80003E03A36104F59F73E3614FF48073C4E96E
:108B90000433236894F83D00E160A36307F06AFAA8
:108BA000064694F8440294F83CA0271D08B152F000
:108BB00013FE94F8450208B152F00EFED4F840328C
:108BC0001BB12F4A116B0B43136318F0080F2FD002
:108BD0000135EDB21EB140F20673F380357218F024
:108BE000100F94F846221DD00221304607F002FAF9
:108BF000D4F8482294F9471294F847321201002918
:108C0000D2B236DB1F49C81880F800235809012268
:108C100003F01F0302FA03F341F820303C462046DC
:108C2000BDE8F08718F0200F0CBF32211221DCE7DD
:108C300019F0020F0CD06B1CDBB21EB140F20652D1
:108C4000F280337294F846220221304607F0D2F9BE
:108C500019F0010FCCD0504607F00CFA0135EDB2F7
:108C600018B140F20663C380057294F846220221CF
:108C7000BCE7054903F00F03CA54CFE74075060867
:108C80000038024000E100E014ED00E02DE9F3417E
:108C9000038A8689B6B205460C461E404FF000484E
:108CA00016B902B0BDE8F081B6FA86F328FA03F2ED
:108CB000D24391B2298216401B3B002C3ED0042B9C
:108CC000EED8DFE803F037312B250300E368EF6AC5
:108CD00023B19B6813B1B9B2201D9847636A2BB1C9
:108CE0009B681BB1B9B204F11C009847E36B2BB130
:108CF0009B681BB1B9B204F134009847636D002B37
:108D0000CED09B68002BCBD0B9B204F14C0003E06D
:108D1000E368696B5B68201D9847C1E7636AA96BCC
:108D20005B6804F11C00F7E7E36BE96B5B6804F137
:108D30003400F1E7636D296C5B68E6E7042B06D825
:108D4000DFE803F00D0B09070300EB6A0193019BB9
:108D5000A6E76B6BFAE7AB6BF8E7EB6BF6E72B6C10
:108D6000F4E790F84820531C0244DBB280F8483006
:108D700082F8341090F849200AB1132B01D956F02B
:108D800067BA7047002280F8492056F061BA70B582
:108D9000124D044695F8833A002BFBD16618B44275
:108DA00004D1002070BD01200AF0B4FBD5F8843A4C
:108DB000D5F8882A0133C3F30A039342F3D0D5F8D8
:108DC000843A14F8012B2B4483F88C2AD5F8843A82
:108DD0000133C3F30A03C5F8843AE0E7901A002090
:108DE00038B50C461146FFF72DFA48B1054D002A5B
:108DF000D5F8943104DD2046FFF7C9FFD5F894314A
:108E000038BD00BF882B0020F0B585B0D0F8CC1558
:108E100090F8CC650291D0F8D0150391012180F82B
:108E2000111106F01F01B0F8D22590F8CD75B0F8F9
:108E3000CE35B0F8D055C0F840210129044600F0E5
:108E40000981022900F01A81002940F09381092F3D
:108E50005ED8DFE817F0B600F4005D00C8005D00E2
:108E600057000A005D00A90076001D0A022DADF82A
:108E700006200BD0032D25D0012D49D1D0F8EC359B
:108E80001B68A0780DF10601984709E0D0F8E43599
:108E900080789B6A0DF1060198474570C4F8F0058B
:108EA000BDF80620002A47D0BDF80E30002B43D075
:108EB0009A4228BF1A46ADF806200146204655F0D2
:108EC0000BFD39E0DBB2052B22D8DFE803F0030706
:108ED0000B0F1317D0F8EC355B68D2E7D0F8EC3500
:108EE0009B68CEE7D0F8EC35DB68CAE7D0F8EC3504
:108EF0001B69C6E7D0F8EC355B69C2E7D0F8EC3502
:108F00009B69BEE72A4303D190F81211032903D1CC
:108F1000204655F00BFC0FE003F07F05016980F857
:108F2000145163F30A120B681A430A6055F0E8FC07
:108F30002DB1022384F81231002005B0F0BD0123C9
:108F4000F8E7D9B28D4D012985F89811E0D890F84D
:108F50001231022B0FD0032BDAD1C1B9022380F8D2
:108F60001231D0F8E43580F810115B68984720463C
:108F700055F0C6FCE0E70029F9D00121032380F871
:108F8000101180F81231204655F092FBEFE790F86F
:108F900010110129EBD0D0F8E4355B68984795F8BB
:108FA000981184F81011EEE7012AB1D190F812312E
:108FB000022B04D0032BABD100F588717EE77049FA
:108FC0007CE790F81231023B012BA1D86B4B0022B9
:108FD000C3F8A021D0F8182112B10222C3F8A021B1
:108FE000684902226AE7012B08D1C4F81831D4F885
:108FF000E43502A99B6820469847B8E7022B9BD12D
:10900000EBB2002B98D103692D0A023D5A68032D5B
:1090100013D8DFE805F0020C0E10022363F30612EA
:10902000564BC3F8A421012384F816319FE703238C
:10903000F4E70423F2E70523F0E70123EEE790F8D5
:109040001221023A012A3FF663AF012B7FF474AF7D
:109050000023CAE790F81231032B7FF459AFEDB229
:10906000012D3FF655AFD0F8E43502A99B6898472B
:10907000BDF80E30002B7FF45FAF78E706F0600696
:10908000202EE9B205D1D0F8E43502A99B689847B3
:1090900052E7012F35D0032F23D0002F7FF44CAFA0
:1090A00090F81231022B5FD0032B7FF431AF15F013
:1090B000800F4FF028031BBF01F07F0103FB01016C
:1090C00003FB010191F81E3108BF91F876332B495B
:1090D000003B18BF0123C1F8A831022201F5D47169
:1090E000ECE690F81221022A3ED0032A7FF410AF5A
:1090F000002B7FF47CAF4A063FF479AF55F0E4FAD9
:1091000075E790F81221022A2ED0032A7FF400AFCF
:10911000002B7FF411AF11F07F023FF428AF6DB246
:109120002823002DB5BF03FB020303FB010303F556
:109130008E7303F55D73002199701A70E90F00EBCF
:1091400082025970002DB4BF9269526DD9781368AC
:10915000023923F4001301298CBFC3F300710121EC
:1091600061F31C73136042E74B063FF4E5AE55F024
:10917000ABFAE1E606F08001F9E700BF882B00209A
:10918000242D0020282D002010B5044671BB90F836
:109190001131032B1BD1D0F89023D0F87C339A42A5
:1091A00017D9C178012908BFD0F88013A2EB0302B8
:1091B00004BFC918C0F88013934228BF1346C0F8F3
:1091C00090239BB2D0F88023002155F049FC002069
:1091D00010BDD0F8E4351B6923B190F81221032AA1
:1091E00000D19847204655F08BFBF0E7D0F8E435E6
:1091F0009B69002BEBD090F81221032AE7D1984706
:10920000E5E770B50A7812F0600305460C4628D0F1
:10921000202B2DD1CB884E78EBB112060AD51D49F3
:109220001A463046FFF7FCF8E2881A49284655F0FE
:1092300053FB0EE0184A1660184A0321C2F80C3896
:1092400080F81111C0E9E43302F50162002155F004
:1092500007FC002070BD022211443046FFF7E0F801
:10926000F7E74B780A2B08D00B2B09D0062BF0D14F
:10927000284655F05BFA0220ECE709490122D6E7BF
:109280008B781BB9074AC2F8AC31E2E755F04EFAC9
:10929000DFE700BFA022002000000020901A00207D
:1092A000342D0020882B002038B5282303FB010132
:1092B000074DB1F88C1304462846FFF7F3F8204613
:1092C00040232A46012155F0CBFB002038BD00BFCA
:1092D000382D002070B50E4BD3F8FC2193F8F051D7
:1092E000044632B193F800322B4302D1012155F0EC
:1092F000EBF98121204655F0E7F9022D07D12046F0
:10930000044ABDE870401F23012155F0A9BB70BD80
:10931000882B00207C2D0020002310B51946044620
:10932000402255F03BFA402280212046002355F090
:1093300035FA012384F81231D4F8E835A0785B6857
:109340009847002010BD38B54022044602238121F1
:1093500055F024FA204602234022012155F01EFA3E
:10936000204603230822822155F018FA084B0222D6
:10937000002583F84B2083F84C500121FFF73BF880
:109380002046044A402355F06BFB284638BD00BFF9
:1093900000000020382D002010B58121044655F032
:1093A000D3F92046012155F0CFF92046822155F00E
:1093B000CBF9FFF72DF8002010BD10B58121044630
:1093C00055F0C2F92046012155F0BEF9024B0020AC
:1093D00083F8140210BD00BF882B0020F8B5224C82
:1093E00094F8832A012A03462ED1204FD7F8185229
:1093F00015B984F8835A23E0402D23D8AEB2402E0D
:1094000002D1022284F8832AD4F8881A184A0A441E
:10941000C3E9542240F201110022A3F84411C3E928
:10942000566203F5A271184655F081FAD4F8883ACD
:109430003344C3F30A03AD1BC4F8883AC7F8185283
:109440000020F8BD4026DFE7022AF9D1002540F2CE
:109450000112C0E95455C0E95655A0F8442100F561
:10946000A27155F064FAC4E7901A0020882B0020FE
:109470001C250020F8B5284FD7F81C320F2B03F11C
:10948000010203D0C7F81C220020F8BD234C0023A2
:10949000C7F81C3294F8833A002BF5D1D4F8882A07
:1094A000D4F8843A9A42EFD0D4F8882AD4F8843A8F
:1094B0009A4295BFD4F8845AD4F8885AD4F8883A96
:1094C000C5F5006598BFED1A402D22D8AEB2402EEA
:1094D0000CBF02230123D4F8882A84F8833A104B66
:1094E0001344C0E9543340F201120023C0E956632B
:1094F000A0F8442100F5A27155F019FAD4F8883A81
:109500003344C3F30A03AD1BC4F8883AC7F81852B2
:10951000BAE701234026DEE7882B0020901A0020BE
:109520001C250020064BD3F880391A79022A05D170
:109530009A68920702D5586953F008BF704700BF78
:10954000901A002010B50A4CD4F8800906F030FBC0
:1095500058B9D4F880090379022B08D183689B0796
:1095600005D5BDE8104008F075B800BFECE710BDA8
:10957000901A002073B50A4E441C0025D6F88009C5
:10958000012300220DF1070155F0A4FE9DF807000C
:10959000FF2802D10135A542F0D102B070BD00BF55
:1095A000901A002070B5044608200D46FFF7E2FF30
:1095B000FF2812D0FE2812D10A4E2B46D6F8800979
:1095C0000022214655F086FE0022D6F880090223AB
:1095D000114655F07FFE002070BD0120FCE70220FF
:1095E000FAE700BF901A002037B5124D4FF6FF532F
:1095F0000024D5F88009ADF8043001AA02232146E1
:10960000C5F84C4955F066FE0120FFF7B3FFFF286F
:1096100005D1042385F85039022003B030BD092359
:1096200085F85039044BD3F89431C5F840392046B9
:10963000F3E700BF901A0020882B002013B540F0FC
:1096400040038DF800300B0E8DF801300B0C8DF8B7
:1096500002300B0A8DF80330952304468DF8041070
:109660008DF8053055F05CFE00B964B90748062353
:10967000D0F880096A46002155F02CFE0820FFF73B
:1096800079FF02B010BDFF20FBE700BF901A002059
:109690002DE9F041194C1E4694F85039042B05462B
:1096A000884617461CD1FFF73DFF94F84739FBB9B0
:1096B00069021120FFF7C2FFE0B9052384F8503991
:1096C0000F4BC4F82C89D3F89431C4F83059C4F83E
:1096D0003879C4F83C69C4F840390120BDE8F0810C
:1096E000082B03D1FFF780FF0228DCD00020F5E72C
:1096F0002946DEE7FFF726FFF8E700BF901A0020B3
:10970000882B002038B500220D233621022006F0D8
:109710006FFE224CC4F8800910B984F8500938BD96
:10972000002106F0D3F8012009F0F4FED4F88059A6
:10973000686906F02CFC95F910301948194D14226F
:1097400002FB03000022D0F8B0000A23114655F0B6
:1097500097FDD4F8800906F02BFA50B9124B84F823
:109760004409D3F89431C4F84039012384F85039BE
:10977000D5E7013DEDD1D4F88009022106F0A6F825
:10978000D4F8800906F075F894F84439C4F8805983
:10979000013384F8505984F84439C0E7901A002006
:1097A00000000020A1860100882B002038B5134C52
:1097B0000023A07BE0B125688D4219D1104C03F540
:1097C00081751AB904EB0514A27138BD04F11801B2
:1097D00001EB43239A4209D1831E5842584104EBBE
:1097E000051454F067FE0123A371EEE70020F6E7AD
:1097F0000133082B04F11004DBD1E6E7D85E00202A
:10980000C04E0020174838B5002380F8A03000F182
:10981000180425688D421ED1A57B032D1BD1124C47
:1098200003F581754AB904EB05140423A371D0F83C
:109830009C300133C0F89C3038BD04F1180000EBB7
:109840004320131A5842584104EB051454F032FED9
:109850000123A371F0E70133082B04F11004D8D1E0
:10986000EAE700BFC05E0020C04E0020F8B5044605
:10987000144EFFF7A2FD204602234022812154F01E
:109880008DFF402201212046022354F087FFD6F8A5
:10989000203200251B6886F81452284686F8F051BD
:1098A0009847E768384655F01FFB3846012155F0C8
:1098B00031FB20461F2306F5FA72012155F0D0F83E
:1098C0002846F8BD882B00202DE9F74F0F460121CF
:1098D00008460192984606F01BFFDFF87CA00024A2
:1098E000A04532DD019B07EB442941F2893603EBA9
:1098F000040B0FE0FEF7F6FD013E08D10120002128
:1099000006F006FF4FF0FF3003B0BDE8F08F0120F6
:1099100009F000FEDAF82839002BEBD05B681D4611
:1099200000231A4649465846A8470028E2D041F28B
:10993000893604E0013EE1D0012009F0EBFDFEF79D
:10994000D1FD0028F6D00134CAE70120002106F03D
:10995000DFFE0020D8E700BF901A00202DE9F74F66
:109960000F46012108460192984606F0D1FEDFF825
:1099700078A00024A04530DD019B07EB442941F28B
:10998000893603EB040B02E0012009F0C3FDDAF88D
:10999000283933B941F28936FEF7A4FDB8B1013454
:1099A000E8E7DB681D4600231A4649465846A847A3
:1099B0000028EFD0FEF796FD013EE5D10120002101
:1099C00006F0A6FE4FF0FF3003B0BDE8F08F013E79
:1099D000F4D0012009F09EFDDEE70120002106F011
:1099E00097FE0020F0E700BF901A0020024BD3F84A
:1099F000240207F05DBD00BF882B00200068F02224
:109A0000FF2107F057BECB4341EA0311CAB20068F9
:109A1000D22107F04FBE0068B422FF2107F04ABEF2
:109A20000A460068A52107F045BE5521F8E7006801
:109A30009622FF2107F03EBE0A460068872107F004
:109A400039BECA01006802F08002782107F032BEF8
:109A500038B50446154600680A46E12107F02AFE9B
:109A600030B120682A46FF21BDE8384008F080BDAB
:109A700038BD0A46E121EBE70A46C321E8E738B5DD
:109A8000021D0D46F0210446FFF7E2FF08B12379DD
:109A90002B7038BDF8B504460E461546071D2068E4
:109AA0003A46FF2108F064FD30B116B12379DB0797
:109AB000F5D40DB123792B70F8BD00220121E9E71F
:109AC00010B50446FFF7A7FF18B12046BDE81040C7
:109AD000F3E710BD10B50446FFF7A2FF18B120460A
:109AE000BDE81040E9E710BD70B506460C468D187C
:109AF000AC4201D1012006E014F8011B3046FFF70B
:109B0000E9FF0028F4D170BDCC21E3E738B5044665
:109B10000D46FFF78CFF40B12046FFF7CEFF20B186
:109B200029462046BDE83840A3E7002038BD70B57F
:109B300006460C468D18AC4201D1012006E02146B4
:109B40003046FFF7E3FF01340028F4D170BD38B58B
:109B500005461446FFF770FF2846FFF7AEFF20B119
:109B60001CB12B79C3F34013237038BD10B50446E4
:109B7000FFF7A6FF38B12046FFF7C6FF18B1204611
:109B8000BDE8104099E7002010BD73B50546CDE94A
:109B90000023FFF795FFA8B12846FFF746FF88B1DD
:109BA0002846FFF78AFF68B16E46082416F8011BA5
:109BB0002846FFF78FFF28B1013C14F0FF04F5D1D0
:109BC00002B070BD0020FBE7C90138B501F080018B
:109BD00004461546FFF735FF08B9002038BD0022BE
:109BE00001212046FFF756FF0028F6D023795B09B4
:109BF0002B70F3E710B5021D0446FF21006808F042
:109C0000B7FC18B12079C04300F0010010BD0F4926
:109C1000D1F8883043F47003C1F888300C4B1A68CF
:109C2000002042F001021A6098601A6822F08472E3
:109C300022F480321A60074A5A601A6822F480229D
:109C40001A60D860044B8B60704700BF00ED00E0E5
:109C5000003802401030002400000008704782B035
:109C60000023019300933C4B1A6842F480321A603F
:109C70001A6802F400320092019A01320192009AAD
:109C80001AB9019AB2F5A04FF2D11B6813F4003350
:109C900018BF01230093009B012B57D12E4B2F4956
:109CA0001A6C42F080521A640A6842F440420A6018
:109CB0009A689A609A689A609A6842F480529A60A8
:109CC000274A5A601A6842F080721A601A68900136
:109CD000FCD5244A40F2027111609A6822F0030216
:109CE0009A609A6842F002029A601B4B9A6802F0EE
:109CF0000C02082AFAD19A6802F00C02042A27D032
:109D0000082A27D159685A685B684902C3F3881347
:109D10004CBF1549154902F03F02B1FBF2F2534323
:109D20000D4A5268C2F3014201325200B3FBF2F312
:109D3000094A91680E4AC1F303110A4492F85C2063
:109D4000D3400C4AC2F8003102B0704700BFFDE7B3
:109D5000054BEDE7054BEBE7003802400070004093
:109D600019304004003C024040787D010024F4009A
:109D700040750608000000200148FEF77DB900BFCD
:109D8000080100200148FEF777B900BF5403002006
:109D9000064A002352F83310814201D1D8B27047ED
:109DA00001330E2BF6D1FF20704700BFAC750608BB
:109DB000704770B5002828D04C684CB942681568C7
:109DC0005679AB8902229BB2B24023EA0203AB81EF
:109DD0008A683AB943681D68AB8923F001031B0404
:109DE0001B0CAB81816044B1436819685D798C8933
:109DF0000223AB4023439BB28B8132B143681A6884
:109E000093899BB243F00103938170BD0B4B30B536
:109E10001A4600241D79854208D1DD68294203D005
:109E2000142303FB042030BD0029F9D001340A2C8F
:109E300003F11403EED10020F5E700BF9C050020DC
:109E40000028ACBF00F16040064B4FEA0111ACBFE7
:109E500000F5614000F00F00C9B2B4BF195480F89A
:109E60000013704714ED00E038B503681B681C68E8
:109E7000244B07EE902A93ED407AF8EE677AB8EE1D
:109E8000477A013987EE270A8DB2DFED1F7A30EE6F
:109E9000270A57F087F91D4A23880138944280B277
:109EA0009BB212D002F5806294420ED0B4F1804F82
:109EB0000BD0A2F58032944207D002F58062944222
:109EC00003D002F58062944206D123F070039BB266
:109ED00023F440739BB206E00D4A944203D002F58E
:109EE00080629442F4D12380084BE5629C42208535
:109EF00003D003F580639C4201D100232386012314
:109F0000A38238BD000000200AD7233C0000014096
:109F100000100040F0B543689A795D7912F00400B2
:109F200002F0020C11BF0022E6464FF48072844614
:109F30000FBF0124964604201446032D38D8DFE8CD
:109F400005F0023872AC1B681D8C25F001052D044C
:109F50002D0C1D841D8C9F881E8B25F002052D0461
:109F600044EA0E042D0C26F073062543634C360498
:109F7000360CA342BFB246F0600603D004F58064FD
:109F8000A34209D14FF6F3742C4044EA0C0427F4A1
:109F9000407744EA000517439F801E8359631D8460
:109FA0001A8B22F008021204120C42F008021A83E3
:109FB000F0BD1D682B8C23F010031B041B0C2B849D
:109FC0002B8CAF882E8B23F020031B0444EA0E0455
:109FD0001B0C26F4E64643EA0413484C3604360CC0
:109FE000A542BFB246F4C04603D004F58064A54242
:109FF0000CD123F0800343EA0C1323F040039BB2FF
:10A0000027F4406743EA001347EA8207AF802E83B4
:10A01000A9632B842B8B23F400631B041B0C43F4D8
:10A0200000632B83C4E71D682B8C23F480731B040F
:10A030001B0C2B842B8CAF88AE8B23F400731B047A
:10A0400044EA0E041B0C26F0730643EA04232B4C4F
:10A050003604360CA542BFB246F0600603D004F5C4
:10A060008064A5420CD123F4006343EA0C2323F45B
:10A0700080639BB227F4405743EA002347EA021764
:10A08000AF80AE83E9632B84AB8B23F008031B0402
:10A090001B0C43F00803AB838AE71B68188C20F481
:10A0A00080500004000C1884188C9E889D8B20F42E
:10A0B0000050000444EA0E04000C25F4E64540EA92
:10A0C00004300E4C2D042D0CA342B6B245F4C0450D
:10A0D00003D004F58064A34203D126F4804646EA07
:10A0E00082169E809D83196418849A8B22F40062E4
:10A0F0001204120C42F400629A8359E700000140F6
:10A1000043685A79032A0FD8DFE802F00205080BEA
:10A1100018683430704718683830704718683C3019
:10A1200070471868403070470020704710B543688A
:10A130001A685879084B0344012093F8DC40138CCB
:10A14000A0409BB223EA00031384138CA14019435F
:10A1500089B2118410BD00BF40750608F0B5EFF359
:10A160001184102383F31288C5684668AA681368AF
:10A1700023F00103136032687779104E938936F823
:10A1800017609BB223EA060393812A696D681F2A30
:10A190004FF0200385BF203A93409340EB6098BF77
:10A1A000AB60E3B283F31188C3689B6859601A6897
:10A1B00042F001021A6001230374F0BD40750608E5
:10A1C0000268137D012B04BF0223137592F82C1033
:10A1D0000CBF4FF400730023012904BF022182F851
:10A1E0002C1092F8441008BF43F48063012904BF87
:10A1F000022182F8441092F85C1008BF43F4006317
:10A2000001290DD1022182F85C1043F48053426889
:10A21000126800215162918989B20B43938101E058
:10A22000002BF4D17047034B0348D3F82812FEF7F4
:10A230002DBD00BF882B00200000014010B5064C4A
:10A240000648D4F82812FEF721FDD4F84812044835
:10A25000BDE81040FEF71ABD882B00200000014029
:10A260000040014010B5064C0648D4F82812FEF70D
:10A270000DFDD4F84C120448BDE81040FEF706BDB1
:10A28000882B0020000001400044014010B5064C1E
:10A290000648D4F82812FEF7F9FCD4F85012044806
:10A2A000BDE81040FEF7F2BC882B00200000014002
:10A2B00000480140034B4FF08040D3F82C12FEF7CA
:10A2C000E5BC00BF882B0020024B0348D3F83012B6
:10A2D000FEF7DCBC882B002000040040024B034842
:10A2E000D3F83412FEF7D2BC882B002000080040BF
:10A2F000024B0348D3F83812FEF7C8BC882B002065
:10A30000000C00400348D0F8703613B100F26460CE
:10A3100018477047000000200348D0F8903613B16A
:10A3200000F2846018477047000000200348D0F80E
:10A33000B03613B100F2A460184770470000002047
:10A340000348D0F8D03613B100F2C4601847704704
:10A35000000000200348D0F8F03613B100F2E460AA
:10A3600018477047000000200348D0F8103713B199
:10A3700000F2047018477047000000200348D0F82E
:10A38000303713B100F224701847704700000020E6
:10A390000348D0F8503713B100F2447018477047A3
:10A3A000000000200348D0F8703713B100F2647049
:10A3B00018477047000000200348D0F8903713B1C9
:10A3C00000F2847018477047000000200348D0F85E
:10A3D000B03713B100F2A470184770470000002096
:10A3E0000348D0F8D03713B100F2C4701847704753
:10A3F000000000200348D0F8F03713B100F2E470F9
:10A4000018477047000000200348D0F8103813B1F7
:10A4100000F6040018477047000000200348D0F8F9
:10A42000303813B100F624001847704700000020B0
:10A430000348D0F8503813B100F64400184770476D
:10A4400000000020036823F0010303600023036081
:10A4500043608360C3600361212343612A4B9842B8
:10A4600003D13D2243F8082C7047284B984204D171
:10A470004FF4746243F8202C7047254B984204D166
:10A480004FF4741243F8382C7047224B984204D191
:10A490004FF0746243F8502C70471F4B984203D121
:10A4A0001E4A43F8642C70471D4B984203D11D4A45
:10A4B00043F87C2C70471C4B984203D11B4A43F84D
:10A4C000942C70471A4B984204D14FF03D5243F8F8
:10A4D000AC2C17E0174B9842C3D0174B9842C7D00B
:10A4E000164B9842CCD0164B9842D1D0154B98427F
:10A4F000D6D0154B9842DAD0144B9842DED0144B8C
:10A500009842E2D0704700BF1060024028600240CD
:10A510004060024058600240706002403D000020F0
:10A5200088600240400F0020A060024000003D20F3
:10A53000B860024010640240286402404064024057
:10A54000586402407064024088640240A064024083
:10A55000B86402402DE9F0410022012603250B6872
:10A5600006FA02F737EA030334D10368540005FA08
:10A5700004FE23EA0E0303600B79D0F800806FEA33
:10A580000E0C03FA04FE013B4EEA080E012BC0F844
:10A5900000E014D883680CEA030383604B79D0F899
:10A5A00008C0A34043EA0C038360436823EA07031F
:10A5B00043608B79476893409BB23B434360C368D9
:10A5C00005FA04F723EA0703C360CB79C768A34001
:10A5D0003B43C3600132102AC1D1BDE8F081204B5A
:10A5E0009A6802F00C02042A10B534D0082A34D13B
:10A5F00059685A685B684902C3F388134CBF19490C
:10A60000194902F03F02B1FBF2F25343144A526877
:10A61000C2F3014201325200B3FBF2F3104C03606B
:10A62000A168124AC1F30311114491F8E010CB4024
:10A630004360A168C1F38221114491F8E01023FA2C
:10A6400001F18160A168C1F342310A4492F8E0202F
:10A65000D340C36010BD034BE0E7034BDEE700BF10
:10A660000038024040787D010024F400407506085F
:10A67000F0B5446B8668A38923F400531B041B0CBC
:10A68000A3818579290201F4806C417901F00103ED
:10A690008907218A4FEA053289B221F4405102F438
:10A6A000005242EA01022282A289C5F3800722F405
:10A6B000B0524FEA83034FEA073722F00C0248BF3B
:10A6C00043F008034CEA07011204120C0B43134336
:10A6D000A381A38A23F440731B041B0C85B0A382BF
:10A6E0006846FFF77CFF204B9C4203D003F5806354
:10A6F0009C4237D1039BA2891921170401FB03F364
:10A700004FF064014CBF7600B600B3FBF6F3B3FB29
:10A71000F1F001FB10330201A08900044BBFDB0004
:10A720001B01323332334BBFB3FBF1F3B3FBF1F315
:10A7300003F0070303F00F0313439BB22381A38AA3
:10A740002A0755BF23F008039BB21B0443F00803FC
:10A7500058BF1B0CA382A3899BB243F40053A3816F
:10A7600005B0F0BD029BC6E7001001402DE9F8439B
:10A770001E46204B9DF820509DF824709842894633
:10A7800090462CD13B462A4631460020FEF7EAF996
:10A7900004460020C4E90700C4E90900C4E90B9895
:10A7A0006571A660A7712046FFF762FFEA0707D52B
:10A7B000636B4FF6DF721A80DA6842F02002DA60CB
:10A7C000626BAB0742BFD36843F08003D3609389C9
:10A7D0009BB243F4005393812046BDE8F883064BB7
:10A7E000984204D13B462A4631460120CEE7002458
:10A7F000F2E700BF0010014000440040816037E7ED
:10A80000417135E7817133E72DE9F043654F07EB7F
:10A81000C00985B005464FEAC00899F8680805F0F8
:10A8200029FC064699F8690805F024FC044699F8C5
:10A830006A0850F0D1FF6B1CDBB21EB140F60C125F
:10A84000F28033721CB140F60C22E28023720422A3
:10A850003A21304605F0CEFB204604223A2105F08D
:10A86000C9FB07EB0803D3F864484F4B9C4263D104
:10A8700003F5F2331A6A42F400121A621A6A22F4D9
:10A8800000121A62474497F86B38022B6ED0032BE4
:10A890006ED0464E464A012B18BF1646A78827F0B1
:10A8A0003F0768463F04FFF79AFE3F0C029A414B70
:10A8B000B2FBF3F398B20743A780218821F001018E
:10A8C0000904090C21803C498E4253D13B4BB2FB19
:10A8D000F3F2013091B2042980B238BF0421208400
:10A8E000A18323889BB243F001032380238823F4B0
:10A8F000816323F002031B041B0C43F48063238059
:10A900004FF480432381238823F080031B041B0C16
:10A91000238023889BB243F001032380284B03EB61
:10A920004513012283F86122002283F8605283F8E4
:10A93000622205B0BDE8F083224B9C4209D103F5A9
:10A94000F0331A6A42F480021A621A6A22F4800210
:10A9500097E71D4B9C4295D103F5EE331A6A42F4FA
:10A9600000021A621A6A22F400028AE7124E95E780
:10A97000124E93E706EB4606B2FBF6F291B2C2F333
:10A980000B020AB941F001014FF4967253434FF4A0
:10A990007A72B3FBF2F301339BB241F4004123849A
:10A9A0009EE700BF000000200054004000350C006E
:10A9B000801A060040420F00A0860100400D0300EF
:10A9C000882B002000580040005C00402DE9F04733
:10A9D000BE4D460105EB401908F0AAFC99F960222A
:10A9E000BB4B8846D10003EBC2020746D2F864484D
:10A9F00099F86222013A142A00F28380DFE812F00B
:10AA0000790089009F00B800C300CD00D600EB009C
:10AA1000F600FF000A014C0174019A01FD010E02CB
:10AA20002002290249026D0215005F184FF0090A41
:10AA300097F8680805F01EFB044697F8690805F0CA
:10AA400019FBB5F8C03201339BB207462046A5F882
:10AA5000C03205F09CFA384605F099FA11212046DB
:10AA600005F09FFA1121384605F09BFA4FF0650872
:10AA700003E00520002108F0ADFC204605F07EFA39
:10AA800010B9B8F10108F4D1204605F085FA00218B
:10AA9000052008F09FFC204605F079FA05200021EA
:10AAA00008F098FCBAF1010AE0D1204605F074FAEA
:10AAB0000021052008F08EFC384605F06DFA0021D3
:10AAC000052008F087FC204605F061FA05200021EA
:10AAD00008F080FC384605F05AFAAB1993F9600289
:10AAE000431C01D0FFF790FEAB19002283F86222CD
:10AAF00007E0238813F4007340F0BA81AA1982F8A2
:10AB00006232AB1993F86232002B7FF465AFBDE877
:10AB1000F087238823F400631B041B0C2380238805
:10AB20009BB243F48063238023889BB243F48073F9
:10AB30002380AB19C3E99A78032283F8622265491E
:10AB40002046FDF740FB002800F09281AB1993F8F6
:10AB500072225AB993F87322FF2A04D193F8702213
:10AB60000AB10A22C2E7AB190422BFE70F22BDE7F0
:10AB7000AB1993F8712202F0FE022282C3E99A789F
:10AB8000052283F8622254492046FDF71CFB002869
:10AB900000F06681AB190622A8E7AB1993F873227F
:10ABA0002282C3E99A78072283F862224B49204621
:10ABB000FDF709FB002800F05381AB19D3F874228C
:10ABC0003AB9228892B242F400722280C3E99A789C
:10ABD00004E108228AE723889BB243F48073238030
:10ABE000AB19C3E99A78092283F8622239492046D1
:10ABF000FDF7E9FA002800F03B81AB19B1E7AB198A
:10AC000093F8712242F001022282C3E99A780B2262
:10AC100083F8622232492046FDF7D5FA002800F079
:10AC20001F81AB19D3F87432012B1AD1238823F476
:10AC300080631B041B0C2380EFF31182102383F32A
:10AC40001288238B23889BB243F400732380D3B2F2
:10AC500083F311880C22AB19C3E99A7883F8622236
:10AC60004FE7022B15D123889BB243F40063238066
:10AC7000EFF31182102383F31288238B238823F4AC
:10AC800080631B041B0C2380D3B283F311880D2235
:10AC9000E1E7238B0E22DEE712492046FDF79DFAFD
:10ACA000002800F0E580AB19D3F87822511CC3F8D6
:10ACB0007812218A1170D3F87422013AC3F87422F1
:10ACC0000122C3E99A7883F87C220FE7882B0020C1
:10ACD000000000200100030082000700840007003C
:10ACE000020003004000001081492046FDF775FA7C
:10ACF000002800F0BD80EFF31182102383F3128847
:10AD000023889BB243F400732380AB19D2B2D3F8EB
:10AD10007812481CC3F87802208A087082F31188E0
:10AD2000D3F87822511CC3F87812218A11706FF081
:10AD30000102C3E76E492046FDF74FFA002800F0F4
:10AD40009780AB1903F51A71D3F87422032A30D116
:10AD5000228822F480621204120C2280EFF3118008
:10AD6000102282F31288D3F8782202F1010CC3F882
:10AD700078C2B4F810C082F800C0228892B242F4BF
:10AD800000722280C2B282F31188D3F87822501C5C
:10AD9000C3F87802208A1070D3F87422023AC3F8FC
:10ADA00074220C2283F86222C3F86872C1F804800E
:10ADB000A7E6022A14D8228822F480621204120C18
:10ADC0002280228892B242F400722280228AC3F842
:10ADD0006872002283F87C22C1F80480012285E693
:10ADE000D3F87822501CC3F87802208A1070D3F868
:10ADF0007422013AC3F87422D6E7238823F48063CF
:10AE00001B041B0C2380AB1993F8712202F0FE0285
:10AE10002282C3E99A78102283F8622235492046BB
:10AE2000FDF7D1F9E0B1AB1993F87322FF2A04D1F1
:10AE300093F870220AB1132258E6AB19112255E695
:10AE4000AB1993F873222282C3E99A78122283F80D
:10AE5000622229492046FDF7B6F908B1AB19EAE7A5
:10AE600026492046FDF7B9F910B1AB1914223DE689
:10AE7000A919D1E99A2342F21070BA1A68EB0303B8
:10AE8000824273F10003FFF43CAE152381F8623275
:10AE900037E6AB1903F51A70D3F8742282B1D3F8F0
:10AEA0007812013A11F801CBA4F810C0C3F874224B
:10AEB000C3F86872C3F87812C0F80480122215E64D
:10AEC000228892B242F4007222800122C3F8687292
:10AED00083F87C22C0F8048008E623889BB243F400
:10AEE000007323804FF6FF33A382AB196EE600BFD9
:10AEF0000400001082000700840007000004001016
:10AF000038B5114C04EB401494F86152D5B1C4F833
:10AF10007432049BC4F87832002384F87C32022314
:10AF2000490084F8732284F8623201229DF81430BB
:10AF300084F8711284F8722284F87032FFF746FDAB
:10AF400094F87C52284638BD882B002038B5114C27
:10AF500004EB401494F86152CDB1C4F87432049BF0
:10AF6000C4F878320223490084F8732284F86232EC
:10AF700000229DF8143084F8711284F8722284F84B
:10AF80007C2284F87032FFF721FD94F87C52284629
:10AF900038BD00BF882B002082B000230193054BF1
:10AFA0000193019B03EB80030193019B196002B0A5
:10AFB000704700BF5028004082B000230193054B2A
:10AFC0000193019B03EB80030193019B186802B07E
:10AFD000704700BF5028004010B51C2005F04AF80B
:10AFE0001121044604F0DDFF204604F0D5FFC820FF
:10AFF00008F090FA2046BDE8104004F0C8BF436D49
:10B00000064A1A61C278012A06D100F2CC50586172
:10B010001A684FF080221A60704700BF180008605D
:10B0200038B5044600296DD190F81131022B28D192
:10B03000D0F83821D0F824118A4230D9C378012BB6
:10B0400002BFD0F828315B18C0F82831521AD0F866
:10B050002831C0F838214FF48071002592B2A0F851
:10B060001C11C0E94A33C0F83451C0F8302100F552
:10B070008E7153F0DDFB2B462A462946204653F0BD
:10B08000EFFC94F81631012B07D1244A2369D2F83A
:10B09000A4215A60002384F81631002038BDD0F86E
:10B0A0003C31B3FBF1F501FB1535A5B9994212D836
:10B0B000D0F8402193420ED24FF48073C0E94A5534
:10B0C000C0E94C55A0F81C3100F58E7153F0B0FB6F
:10B0D000C4F84051CFE7D4F8E435DB682BB194F8DD
:10B0E0001221032A01D120469847052384F8113103
:10B0F000002320461A46194653F0B2FC2046FFF7BB
:10B100007EFFBEE7D0F8E4355B69002BC5D090F830
:10B110001221032AC1D19847BFE700BF882B002026
:10B1200070477047704710B50F4C94F8CE32B3B1EA
:10B130004FF0E022D2F8103D23F00603C2F8103D94
:10B14000FEF765FDD4F8D4329B68DB0707D5D4F849
:10B15000D023136823F0030161F307031360034B4B
:10B160004FF480225A6110BD882B0020003C014022
:10B170002DE9F04FB14CD4F8D0325A69D0078BB0DA
:10B1800000F196815A699B6912EA030A00F09081E6
:10B19000CAF307431AF4002F01930FD0D4F8D43226
:10B1A000DFF8A0829E69DB691E40360C04F5467B01
:10B1B00004F531790027002E40F07D81019B59076D
:10B1C0000DD5D4F8D4329E4D9F69DB691F40BFB2C4
:10B1D00005F118064FF00008002F40F0AD811AF07D
:10B1E000020F1FBF954BD3F8D03202225A61BAF139
:10B1F000000F5FFA8AF51BDA904B93F8CE223AB132
:10B20000D3F8D023136823F0030161F3070313601D
:10B21000D4F8D4228A48536823F001035360894B41
:10B22000D3F894389847D4F8D0324FF000425A619E
:10B230001AF4006FCAF307262FD000238DF81730B9
:10B2400094F8D6338DF817307E4B7D48D3F890387C
:10B250009847D4F8D022D4F8D4324FF400619B68D8
:10B26000516194F8CE22C2B1DB0716D594F8D933D8
:10B27000012B12D19DF81730032B0ED1D4F8D03307
:10B280001A6842F001021A601A6842F003021A605A
:10B290006D4A136943F0060313612F0708D5694B04
:10B2A0006748D3F888389847D4F8D03208225A61D2
:10B2B000ED0614D5D4F8D002836923F0100383611E
:10B2C000036AC3F34341022903F00F0200F0E9814E
:10B2D000062900F00D82836943F010038361F006B4
:10B2E00033D5D4F8D452D4F8D0826B68002723F039
:10B2F00001036B603946404653F00CFE94F8C5C21A
:10B300005249B9463B46FF206345C0F0FF814FF0EC
:10B31000FF33AB614FF00113EB610B2363F30707BE
:10B3200063F307096F61C5F810902B68444823F454
:10B33000FE632B60FFF763FE4FF48053C8F81430B0
:10B34000404B3F48D3F88C389847B1066DD5D4F8B8
:10B35000D462D4F8DC22B3681168C3F34103022B32
:10B3600014BF0023032363F30A011160736843F4DD
:10B370008073736006A8FFF732F9D4F8D0520799AA
:10B38000E86820F47050E860B36813F0060FC3F368
:10B39000410200F0C2812E4B2E4A0B44934240F2F0
:10B3A000C0812D4AA1F57403A3F51053934240F2D6
:10B3B000BC812A4B2A4A0B449342C0F0BA81294AE5
:10B3C000A1F18C73A3F54343934240F2B681264B1F
:10B3D000264A0B449342C0F0B481254B254A0B44C6
:10B3E0009342C0F0B281244AA1F1B773A3F5585338
:10B3F0009342C0F0AD81214B214A0B449342C0F0EF
:10B40000AB81204B204E0B4401224021B34234BF7C
:10B4100006230523094E63F38D204FF40053E860A3
:10B4200086F8C622A6F8C8126B61019BDA0632D5EF
:10B43000044B0348D3F89838984727E0882B00201E
:10B440004C2E00200000002000ED00E0602E0020C7
:10B45000401E1BFF3F420F00DFC810002013FBFE01
:10B4600020D61300FF69180000D3CEFE40771B00E2
:10B47000C05BB3FEC091210040AC2700C01D6AFE36
:10B4800040E13300803C36FEE09C4100D4F8D032ED
:10B490004FF480125A61019B9B0609D5B04BB1480D
:10B4A000D3F89C389847D4F8D0324FF400125A6140
:10B4B0000BB0BDE8F08FF10737D5DBF80010D4F8FA
:10B4C000D4328D685B691D40EA071ED594F8C732F7
:10B4D0000125AB428D6007D10969D9F87C33C1F3EE
:10B4E00012015B1AC9F88C33D8F87C389D48F9B240
:10B4F000984794F8C732012B07D137B994F8D53360
:10B50000052B02D19748FFF77AFDAB0742BFDBF866
:10B51000003002259D60280707D5D8F88438914867
:10B520009847DBF8003008229A60013776080BF163
:10B53000040B09F128093EE6FA0772D5D4F8D43293
:10B5400032681869D3F83490916829FA08F94FEAFB
:10B55000C9195FFA89F949EA000909EA010919F0EC
:10B56000010F1FD0596B012000FA08F021EA0001F9
:10B5700059637B4B7B48D3F880384FF00109C2F800
:10B5800008905FFA88F1984794F8C7324B4509D183
:10B59000B8F1000F06D194F8D533042B02D17148CD
:10B5A000FFF72DFD19F0080F1EBF33684FF0080993
:10B5B000C3F8089019F0100F1EBF33684FF0100940
:10B5C000C3F8089019F0400F1EBF33684FF04009D0
:10B5D000C3F8089019F0020F1EBF33684FF002093C
:10B5E000C3F8089019F0800F1BD0D5E94C329B1A94
:10B5F000D5F82421D6F800B0934228BF13465A4A02
:10B60000DBF8180092F8C7C2D2F8D49203339B0833
:10B610000293029B80B2984203D9D5E94C03984229
:10B6200005D808F101087F0828350436D4E5C01A8A
:10B63000D5F82431984228BF1846C31C9B080293B2
:10B64000BCF1000F1BD0D5F82811D5F834210144E6
:10B65000C5F82811D5F8301102448A42DBF81800E9
:10B66000C5F83421D5D195F81C11D9F8342001231F
:10B6700003FA01F122EA0102C9F83420C9E782B2D3
:10B68000D6F8B810D5F828E10332931003930A4690
:10B690006146039B8B42D6D05EF8213013600131A6
:10B6A000F7E747F6F07119423FF415AE282101FB88
:10B6B0000241C3F30A13DD1CD4F894C3D1F84476D5
:10B6C000AD1000218D420DD1282101FB0242D2F89C
:10B6D00044161944C2F84416D2F850161944C2F858
:10B6E0005016F8E5DCF800E047F821E00131E9E721
:10B6F000D4F894130D68C4F890580968C4F89418E5
:10B70000282101FB0242C3F30A13E5E751F8042F95
:10B710009060CA6B01339060F6E54FF40071092325
:10B7200078E6012240210E2374E6012240210D23F8
:10B7300070E6012240210C236CE6012240210B23FC
:10B7400068E6012240210A2364E601224021E6E75F
:10B750000122402108235DE601224021072359E60A
:10B76000000000204C2E0020882B0020034BD3F833
:10B770007C0908B104F002BC01207047901A002037
:10B7800008B5FFF7F3FF0A4A18B9002382F85039C9
:10B7900008BD92F844390133DBB2072B82F84439F3
:10B7A000F3D8044BD3F89431C2F840390123EDE7C4
:10B7B000901A0020882B0020F0B5C54CD4F88009E1
:10B7C00085B0002861D094F85039013B082B44D84B
:10B7D000DFE813F009005D00DF004300AA0130013B
:10B7E00086014300E601FDF79DFE00210846FDF7B6
:10B7F00025FF0546FDF7A6FE012D29D1002684F878
:10B800004669FDF78FFE40F2AB110820FDF716FFE9
:10B8100005280AD184F84659FDF794FE94F8463974
:10B82000A3B1022384F85039CDE70128F4D10423D1
:10B83000D4F880093246694653F04CFD9DF8033038
:10B84000AB2B04BF022384F84639E5E784F850396E
:10B85000D4F88009022104F039F894F85039013BFA
:10B86000022B09D89B4BD4F84029D3F894319B1A6A
:10B87000C82B01D9FFF784FF94F85009042800F081
:10B88000A081A0F108035842584105B0F0BDFDF772
:10B8900049FE94F84659AA1E55425541AD0700216C
:10B8A0003720FDF7CBFE29462920FDF7C7FE0546C8
:10B8B000FDF748FE002DCBD194F84639022B17D165
:10B8C000FDF730FE29463A20FDF7B8FE0423064670
:10B8D0002A46D4F88009694653F0FCFCFDF732FE95
:10B8E00016B1FFF74DFF6EE7009D2DBAC5F38075C9
:10B8F00084F84759FDF716FE00210920FDF79EFE4A
:10B9000010B1FDF71FFEA3E773481021FDF74AFEB3
:10B9100006460028F5D101217F204FF0C5FD012802
:10B920000546EED1022130464FF0BEFD50B1012850
:10B93000E7D116213A204FF0B7FD01308002C4F85C
:10B94000540918E004212C204FF0AEFD03210746D6
:10B950004E204FF0A9FD0C21064636204FF0A4FDE5
:10B960000236431CB340BD40A3FB05355B0A43EAE6
:10B97000C553C4F85439FDF7E5FDFDF7D3FD0021AB
:10B980000A20FDF75BFE08B903234BE7FDF7DAFD5C
:10B99000A7E710216846FDF705FE00287FF458AFA1
:10B9A0009DF8003084F85A39BDF801305BBAA4F82C
:10B9B00058399DF8033084F85B39019BC4F85C3931
:10B9C0009DF808301A0903F00F0384F86539DDF893
:10B9D000093084F864291BBAC4F860399DF80D3029
:10B9E0009DF80E201B01DBB243EA121303F5FA6344
:10B9F00002F00F02A4F8663984F86829FDF7A2FD69
:10BA000094F847394BB1D4F88009022103F05EFF66
:10BA10000023C4F84C39042304E7FDF783FD4FF4F9
:10BA200000711020FDF70AFE0546FDF78BFD002D85
:10BA3000E9D056E794F83419D4F82C29D4F88009C1
:10BA4000802302EBC112002153F044FC94F83439F6
:10BA50000133DBB2042B84F834397FF4FEAE1F4A85
:10BA6000D4F880090223002153F034FC0123D4F8D8
:10BA700080090022694653F02DFC9DF8003003F048
:10BA80001F03052B15D1072384F85039114BD4F827
:10BA90003859D3F89431C4F84039002D3FF4DDAE65
:10BAA000D4F83C39D4F82C29D4F830190120A8470F
:10BAB000D3E6FFF765FED4F83859002D3FF483AE86
:10BAC000D4F83C39D4F8301900220120A8477AE68E
:10BAD000901A0020882B0020FC23002030760608D6
:10BAE00053F01EFC002862D0002384F84439D4F8B7
:10BAF0004C39012B0BD9013BC4F84C39D4F84839E7
:10BB00000133C4F84839082384F85039A5E607D131
:10BB1000FDF76AFD02287FF4A0AEFDF713FD9CE659
:10BB2000042384F85039F8E7D4F82C094FF4007155
:10BB3000FDF738FD0128054619D0022820D000283D
:10BB40007FF48BAEFDF7FEFCD4F8386984F84459D5
:10BB5000042384F85039002E3FF47FAED4F83C39EA
:10BB6000D4F82C29D4F830192846B04775E6164B7E
:10BB7000D3F89421D4F8403964339342BFF46DAEC6
:10BB8000FDF7E0FCFFF7FCFDD4F83859002D3FF439
:10BB90001AAE0022D4F83C39D4F83019104695E793
:10BBA00053F0BEFB18B1FDF7CDFC0423ACE7064B08
:10BBB000D3F89421D4F84039FA339342FFF491AE8C
:10BBC0004BE6012061E600BF882B00202DE9F34100
:10BBD000284C05460E4690461F4694F85039042BD3
:10BBE0000DD0082B07D1D4F84839AB4219D0FDF756
:10BBF000FBFC0228F1D0012002B0BDE8F081FDF786
:10BC000091FC94F8473953B969021820FDF716FDE5
:10BC100038B1FDF797FCFFF7B3FD0320ECE72946A9
:10BC2000F3E794F85039D4F88009082B14BFFE23A9
:10BC3000FC23FF228DF804208DF8053001AA022391
:10BC4000002153F047FBD4F88009802332460021BD
:10BC500053F040FB012384F834390623C4F82C69DF
:10BC6000C4F83059C4F83889C4F83C7984F850399C
:10BC70000020C1E7901A002070B51C4C94F8503990
:10BC8000042B05460E4610D1FDF74CFC0021372051
:10BC9000FDF7D4FC31461720FDF7D0FC90B1FDF73D
:10BCA00051FCFFF76DFD032002E0082B01D00120BD
:10BCB00070BDD4F84839834214D0FDF795FC0228B2
:10BCC000F5D1E1E794F8473973B969021920FDF716
:10BCD000B5FC0028E3D1082384F85039C4F84C6936
:10BCE000C4F848590220E3E72946EFE7901A0020FC
:10BCF000034BD3F8280908B143691847704700BFC0
:10BD0000901A0020034BD3F8280908B1836918471B
:10BD1000704700BF901A0020002110B5084604F0BB
:10BD2000F7FCFFF7EFFF40B90F4B104A03F6A801ED
:10BD3000C2F82819D3F8A8389847002403E0012056
:10BD4000013407F0E7FBFCF7CDFB10B9B4F57A7FBF
:10BD5000F5D10121002004F0DBFCB4F57A7F4FF02F
:10BD6000FF3018BF002010BD00000020901A0020F6
:10BD7000034BD3F8280908B1C3691847704700BFBF
:10BD8000901A002038B50D461446FFF7F1FF0368FE
:10BD90002B604FF400732360002038BD034B1B78E9
:10BDA000032B14BF4FF4807080207047C04E0020DA
:10BDB00008B50B4A68B1816811B10723937008BDBB
:10BDC000FFF7ECFFC2E90311C2E90100117504237A
:10BDD000F4E702F58051012381F8B4315370EEE7A6
:10BDE000C04E002010B502784368022A0B4A06D1E3
:10BDF000D2E9802102EB410202EB532010BD016920
:10BE0000D2F81802D2F8104218400239D2F80C3297
:10BE1000400A04FB01001844F0E700BFC05E0020A8
:10BE2000064B1B78022B0BBF030AC0F3D413C0B21E
:10BE300000F07F000B601060704700BFC04E002014
:10BE400090F91A305A1C0AD003F58172124B03EB99
:10BE50000213DA7922F00102DA71FF23837690F976
:10BE60001B104B1C16D00C4A01F5817102EB01131B
:10BE700002EB0112DB79D179C3F34503012B86BFB5
:10BE800003F1FF3303F03F03002363F34601FF2375
:10BE9000D171C376704700BFC04E002008B5FFF7D0
:10BEA0007DFF034BD3F810325843400208BD00BF5A
:10BEB000C05E00200378022B09D10E4BD3F820225C
:10BEC0004368B3EB422F2CBF01200020704700696C
:10BED00070B1094B1B78032B0EBF084B80B24FF695
:10BEE000F773984294BF0020012000F001007047D2
:10BEF0000120FAE7C05E0020C04E0020F7FFFF0FD0
:10BF00004368F7B5C3F308020A44B2F5007F04465C
:10BF10000D4604D22B446360012003B0F0BDFFF74F
:10BF20008FFF0378022B01D16368F3E7154BD3F839
:10BF30001022B5EB422F4FEA422706DCD3F8183225
:10BF400046681E407342AB4201DD0020E5E7AB19B5
:10BF5000BB4210D30169007E01AA52F08BFB01287D
:10BF6000F3D123696361019B236163683B449B1B9D
:10BF7000EF1B6360BD192046FFF79CFF0028CBD163
:10BF8000D2E700BFC05E002070B504460E461546DD
:10BF9000FFF7B6FF20B10DB12046A847012070BDC4
:10BFA00094F82800022320B9C4E90B5684F82830FD
:10BFB000F5E71846F3E738B5174D05F58054014607
:10BFC00094F8E00130BB49B191F828302BB94422F4
:10BFD00004F5DC7059F064F8012038BD44220F48A4
:10BFE0005AF080F94FF6FF73A4F8D231032384F896
:10BFF000D0312B780948022B18BF032384F8B831BD
:10C00000D4F81C32C4F8DC31102384F8D1314FF05D
:10C0100015FCE1E70020E0E7C04E0020786000203A
:10C02000044A92F8B411012309B982F8B431024AE2
:10C0300053707047C05E0020C04E00202DE9F74FBE
:10C0400012F002098A461546019304D018B9FFF789
:10C05000E7FF02200CE0684AD2F808625EB1D2E93C
:10C06000831404FB0611884205D3FFF7D9FF002093
:10C0700003B0BDE8F08F4FF0FF31604EDFF880B1C4
:10C080008C468E46884600243368B77B984221D17F
:10C09000002F46D0D2F89810594E0131C2F89810AE
:10C0A00004F581721201B1502146554C01F581769B
:10C0B00004EB06129279042AC9D801A757F822F096
:10C0C00057C10008ADC100086FC00008ADC100082D
:10C0D000C1C100080FB3012F10D104F581770BEB1C
:10C0E0000717FF79FB0709D417F07E0F06D1FF0968
:10C0F00015D1B76847453CBFA446B8460134082C63
:10C1000006F11006C0D100290CDABEF1000F20DACA
:10C11000BCF1000FABDB614604E02146EEE7A6462A
:10C12000ECE72146364E41F2180406EB0117385170
:10C13000D2F898400134C2F8984041F21C02BC5039
:10C1400001F58172170106EB0212F45100245460CC
:10C15000ABE77146E6E715F0010213D0294BD3F89F
:10C160002839002B83D0284F5D68284A002307EB2D
:10C170004121A84700283FF47AAF04EB06140223BC
:10C18000A37174E704EB0610019B90F807C0EF1051
:10C1900067F3C71C032B80F807C02BD94FF6FF723B
:10C1A000934228BF134604EB06129380B9F1000FA7
:10C1B00006D004EB011000F580501830FCF7B4F9FC
:10C1C0006A0741BF04EB0612D37943F00103D37130
:10C1D000EB0608D504EB0614E379C3F345020132FC
:10C1E00062F34603E371084B03EB4123CAF80030C6
:10C1F00001203DE71346D6E7C05E0020D85E002050
:10C20000C04E0020901A0020D84E0020AD970008A4
:10C210007FB50F4D01AA0C4602A9FFF701FE05F5F7
:10C220008053029ED3F800020322002303A9304466
:10C23000FFF704FF012808D12978039B019A0229FE
:10C240000CBF23F8124043F8224004B070BD00BF79
:10C25000C04E00202DE9F04FD1F8009085B0164671
:10C26000074601AA48460D4602A9FFF7D9FD374AFD
:10C270000299D2F8003201EB0308019B013B9C19A3
:10C28000FFF78CFDA4EB09040444A2F5805AB4FB2B
:10C29000F0F408EB04092B68B342A9EB080103D3BF
:10C2A000012005B0BDE8F08FDDF804B00BEB06040B
:10C2B000E41AFFF773FD844228BF0446BBF1000F68
:10C2C0001AD1A0428CBF0B220A220B46404603A97A
:10C2D000FFF7B4FE0128E4D19AF800102B68039A06
:10C2E000022903F1010358460CD0A0420CD242F8B7
:10C2F000203001300133F8E70B22E6E722F8103056
:10C3000001300133A042F9D32B68A3EB0B03234484
:10C31000012F2B6014D1B34212D102290BBF04F1BB
:10C32000004404F1804304F1FF3403F1FF330BBFF9
:10C330004FF6FF734FF0FF3122F8143042F823100C
:10C34000002308F101080193A5E700BFC05E0020AB
:10C350002DE9F04F85B00546FFF720FD0C46174646
:10C36000814601AA206802A9FFF75AFD6B1E012B26
:10C3700066D9019B4BB94E46DFF8C880012D8CBFB2
:10C3800000250125A8F5805A1BE0FFF749FE022091
:10C390002BE0D8F87831C3B1D8F89411914214D178
:10C3A000D8F81022013B500203EB4223B3FBF0F319
:10C3B0000B44B3FBF6F206FB12320AB133449B1A6C
:10C3C00023602268BA42E4D32BE0DDF808B0D8F845
:10C3D00000020023092203A95844FFF72FFE012879
:10C3E00006D00228D3D00028EBD105B0BDE8F08FED
:10C3F0009AF80010019A022907D00329C7D1039B9C
:10C4000053F8223023F0704302E0039B33F81230DC
:10C41000D4F800C0B3FA83F35B09AB4204D167459B
:10C42000E3D827600320E0E732440CEB0603914594
:10C430002360E0D80BF10103029300230193C0E7CE
:10C44000012699E7C05E002037B50446C0690D4655
:10C4500010B9012003B030BD0023032201A9FFF76A
:10C46000EDFD0128F6D1B4F92030002B17DB019A3D
:10C47000012D4FEA431102EB431316D0022D12D0C7
:10C48000E268DA612278032A04D100221A775A7707
:10C490009A77DA77626A5A83110C9982D9E7FFF7A3
:10C4A000BFFD0220D6E7E5205054A268E9E738B581
:10C4B000044694F83430052B2FD8DFE803F0072723
:10C4C000353C444D022084F83400F2E7294DD5F87C
:10C4D000082204F1300102320120FFF739FF012860
:10C4E00005D00238C0B2012817D80520EBE7D5F8EF
:10C4F0001012E268236BC5F8143202EB4122E260AD
:10C50000E26A2361002ADED16362DCE7206B4FF030
:10C51000FF31FFF77DFE012801D0002038BDE36A1E
:10C52000002BCFD10320CEE7D4E90B01FFF770FE3B
:10C530000128F7D0F1E700212046FFF785FF012809
:10C54000EBD10420BFE794F82830082B04BF002368
:10C5500084F828300120E1E794F82830082B04BF44
:10C56000002384F82830034B012283F8B5210220F0
:10C57000D4E700BFC05E00202DE9F341044694F8E3
:10C580003830032B0ED8DFE803F00611767F032046
:10C5900084F83800F3E72046FFF789FF0128F7D039
:10C5A0000228F4D0002002B0BDE8F081237865684D
:10C5B000DFF8E480022B1CBF374BD3F8183220463B
:10C5C00018BF1D40FFF70EFCC5F34F252D1A064678
:10C5D000ADB20023022201A93046FFF72FFDAF19AB
:10C5E0000128BFB2DFD101984FF40072002159F049
:10C5F00079FEE3692BB363681BBB019B4FF02032CC
:10C600002E211970C3F80120C3F80520A3F80920D2
:10C61000606A58834FEA104C102083F8201083F88A
:10C620002110D872C3F82220C3F8262083F82A20CC
:10C63000E26BA3F814C022FA00F199865A8783F8B6
:10C640002B00D8F810124B1E9F4208D24FF40071F5
:10C650002046FFF755FC51F02DFF0136B9E7C1EB3D
:10C66000C151490201F500712046FFF749FC51F024
:10C6700021FF02208CE7002384F82830236C0BB1C3
:10C680002046984701208EE7236C002084F828007C
:10C6900003B19847022086E7C05E002010B504462B
:10C6A00094F83830032B53D8DFE803F00631434DBC
:10C6B000022384F83830F3E72649D1F89421226127
:10C6C000FFF7ECFBE3680344E360FFF767FB10440C
:10C6D000C1F89401FFF7E2FBD1F878311B1AC1F8D9
:10C6E0007831FFF7DBFBD1F87C311B1AC1F87C31C4
:10C6F0002263FFF753FBE36A1044606313B962627D
:10C700000123D6E7FFF74AFB121A2263F8E7124823
:10C710000021FFF799FE0128CAD0431EDBB2012B8E
:10C7200006D894F82830062B04BF002384F828305C
:10C7300010BD626B04F130010120FFF78BFD012871
:10C74000EBD10323B5E700212046FFF77DFEE4E7A8
:10C750000220E2E7C05E0020306000202DE9F743B0
:10C7600006460C464FF6F77596F83C30042B73D806
:10C77000DFE803F0290736416300032086F83C0018
:10C78000F2E73A4FDFF8EC8007F580593B78306BE1
:10C79000032B4FD140454BD801A94EF061FE012833
:10C7A00057D1306B0021FFF733FD012851D1019B98
:10C7B0003363D9F81422013B934294BFC9F8143271
:10C7C000C9F81422E2E7610001F0FE013046FFF7EC
:10C7D0003BFE01280CD1736B002B18BF0220CDE764
:10C7E000726B06F130010020FFF734FD0128C4D040
:10C7F00002282ED131E01E48F26AD0F89431C0F8F8
:10C8000094219B1AD0F810225343D0F8782102EBE0
:10C810004322C0F87821D0F87C2102EB4322C0F8F3
:10C820007C21002100F5B870FFF70EFE0128DFD152
:10C830000420A3E783B2AB42ADE796F82830042B7F
:10C8400004BF002386F82830B36B0BB130469847FD
:10C85000012003B0BDE8F083022096F82830042BB5
:10C8600004BF002386F82830F3E700BFC04E002045
:10C87000C05E0020F7FFFF0F70B50378027E023B19
:10C88000012B04461CD8237E990622D42046FFF7AC
:10C89000D7FA237E1A070AD51E4D95F89801C31FB3
:10C8A0005842584151F006FE002385F89831002384
:10C8B000237084F82830E36A53B1BDE8704018470C
:10C8C00012F0060FDFD00121FFF7BEFD0128DAD0FC
:10C8D00070BDE2691049002318010858824211D145
:10C8E0000E4903F5817201EB0213DB79C3F34503B3
:10C8F000012B0BD8002301EB0212D17963F346011F
:10C90000D171C3E70133082BE6D1BFE7013B03F048
:10C910003F03F0E7C05E0020D85E0020C04E00203C
:10C9200010B580B1027872B190F828206AB9D0E9C8
:10C93000012494422CBF84608260032280F8282066
:10C94000C162FFF799FF012010BD0020FCE7B1F99B
:10C9500004300F2B2DE9F34104460D4616460BD14A
:10C960004FF40071FFF7CCFA18B9002002B0BDE80F
:10C97000F0814FF6FF73AB802046FFF733FA94F94E
:10C980001B20531C074624D0244B41F2180103EB13
:10C99000021041588F4212D1183303EB4223019306
:10C9A000019A72B1AB8801331BB202EB4312AB8028
:10C9B00020463260FFF716FA28600120D6E7FFF71D
:10C9C0002FFB2046FFF776FA0028CED000233360F5
:10C9D000F3E72046FFF76EFA80460028F1D1381EB3
:10C9E00018BF012051F066FD4346112201A93846C7
:10C9F000FFF724FB0128E4D1094A019B9B1A48BF99
:10CA000003F2FF13B3F5805F4FEA632203D3FFF70E
:10CA100007FB4FF0FF32E276C2E700BFC04E0020B6
:10CA2000D84E00202DE9F0414FF0FF31304A314C13
:10CA30000D460023107804280ED103F5817004EB15
:10CA40000010C079C60707D4681C52F80A0C01D040
:10CA5000884201D201461D460133082B02F1100223
:10CA6000E8D1002D41DB234CDFF8988005F5817774
:10CA700004EB07132E01998841B1D8F828392BB15E
:10CA8000A01941F218029B688058984741F2180398
:10CA90002644F058D8F828396BB1174ED3F80C80DB
:10CAA000164A002306EB4521C04720B1022810D0CA
:10CAB0000020BDE8F081124BD3F89C2004EB071452
:10CAC000013AC3F89C200322A271012283F8A0201E
:10CAD000EEE706F6E87604EB0714D6F89C30013B47
:10CAE000C6F89C300123A371E2E70120E1E700BF13
:10CAF000E65E0020C04E0020D84E002005980008B9
:10CB0000C05E0020901A002070B5124D124BC5F87F
:10CB1000B83840F20112002385F81432A0F84421FD
:10CB2000C0F85C3105F6B8020D23C0E95422044672
:10CB300085F8C418C0F8583100F5A27151F0F7FE1D
:10CB400005F5FA7220461F23BDE87040012151F01F
:10CB500087BF00BF882B00205553425370B50B7818
:10CB600013F06002044638D0202A1ED14A78FE2AEB
:10CB700005D0FF2A1DD051F0D9FD022016E04A88C9
:10CB8000AAB9CE88012E12D11A0610D5314DD5F88A
:10CB900020329B699847C0B285F8C80838B1324640
:10CBA00005F6C801204651F097FE002070BD2046D2
:10CBB000E1E74A88002AFAD1C9880029F7D11B0683
:10CBC000F5D4244A82F81412012182F8F0111F23AF
:10CBD00002F5FA7251F044FFE7E74B780A2B24D0B4
:10CBE0000B2B25D0012BE0D191F904600D79C068A1
:10CBF000002E22DA05F07F0152F08CF929462046FA
:10CC000051F0A2FD2946134D02234022204651F047
:10CC1000C5FD95F8F031022B12D18121204651F04B
:10CC200053FD002385F8F031BFE70B490122BAE735
:10CC3000084B4A8883F8C928B7E752F055F9DDE771
:10CC4000002EB2DA012BB0D001212046FFF75CFFA5
:10CC5000ABE700BF882B00205134002010B50B4AF1
:10CC600092F81432022B044607D0033B012B02D862
:10CC70000021FFF749FF002010BD92F8011251F08A
:10CC80000DFF0028F7DA01212046F2E7882B00206B
:10CC900070B5314C94F8146205461EB1012E50D087
:10CCA000002070BDD4F8F831C4F8BC38D4F8FC3199
:10CCB000C4F8C038B0F8B4331F2B0DD1D4F8F42128
:10CCC000264B9A4208D194F80112012904D894F80D
:10CCD0000232013B0F2B0AD92021052051F06AFBBB
:10CCE000022384F8F0312846FCF7F4FAD8E751F033
:10CCF000D5FE0028F7DB94F81432013B022BCFD984
:10CD0000B4F8CA1821B3D4F8FC3184F8C468994245
:10CD100028BF1946D4F8C0385B1AC4F8C0380423B9
:10CD200084F8143240F20113A5F844310C4BC5E9E4
:10CD30005616C5E9543305F5A271284651F0F7FDA2
:10CD4000AEE794F8011251F0A9FE0028A8DA3146A6
:10CD50002846FFF7D9FEA3E7882B0020555342430E
:10CD6000BE3E0020F0B59C0827010E46154600EB9C
:10CD70000414A04206F1100605F1100508D103F0D5
:10CD8000030339443A4404EB83039C4223D1F0BDAE
:10CD900084469CED006A16ED045AD0ED016A56ED0A
:10CDA000037A90ED027A56ED025A26EE056A66EE97
:10CDB000A76AD0ED037A05ED046A16ED016A45ED28
:10CDC000036A27EE257A67EE867A103005ED027A3F
:10CDD00045ED017ACDE7F4EC017AB1EC017A67EE2A
:10CDE000877AE2EC017AD0E74A09012350F8222041
:10CDF00001F01F018B40134214BF01200020704737
:10CE000010B54C09012250F8243001F01F018A406E
:10CE1000134340F8243010BD80EA0120082241F27B
:10CE2000210103B2002BB5BF81EA4303400098B251
:10CE300080B2013AF5D1704738B50C468D18AC4236
:10CE400000D138BD14F8011BFFF7E6FFF7E74840B3
:10CE5000082243B2002BBBBF5B0083F0D503400028
:10CE6000D8B2A8BFC0B2013AF3D1704738B50C466A
:10CE70008D18AC4200D138BD14F8011BFFF7E7FF55
:10CE8000F7E770B5066805460C460020B44203D3A8
:10CE9000731C2B60307070BD14F8011BFFF7D7FFB7
:10CEA000F4E7DFED0A7AC0ED020A20EE270AB7EEBA
:10CEB000007AC7EE007A00230360C0ED017A70EEBD
:10CEC000A77A80EEA77A80ED037A7047DB0FC9401E
:10CED00090ED017AD0ED007AC0ED020A30EE877A4B
:10CEE000C0EE876A30EE677AE6EE877AB0EE670AC0
:10CEF000C0ED007A7047012303700023C36483648C
:10CF00000365036443644365836283657047DFEDB3
:10CF1000157A80ED010AF4EEE70AF1EE10FAC0EDA1
:10CF2000020A80ED031AC0ED051A18DDB4EEE70A17
:10CF3000F1EE10FA08DC9FED0C7A80ED047A80EDBA
:10CF40000F2AC0ED0E2AD6E781EE007AC0EE207AD5
:10CF5000F0EE006A77EE877A86EEA77AEDE7002397
:10CF60008360E8E7BD378635000000000F29A8BFC1
:10CF70000F21012970B5B8BF01214C0001340026F2
:10CF80000460A40005468160466022463146803038
:10CF900059F0A8F92246314605F58070BDE8704089
:10CFA00059F0A0B9FDEEC07A17EE903A2033402B2D
:10CFB00043D8DFED237A9FED237AB4EEE70AF1EE52
:10CFC00010FA28DCDFED207A9FED1E7AB4EEE70A36
:10CFD000F1EE10FA22D4DFED1D7AB4EEE70AF1EE9D
:10CFE00010FA1EDD30EE670A37EEC00A60EE007AF6
:10CFF000DFED176A9FED177AA7EEA67ADFED166AC6
:10D00000E7EE876A9FED157AA7EEA67A20EE276AEB
:10D01000A6EE070A704730EE470ACEE730EE070A61
:10D02000D4E79FED0F7AB4EEC70AF1EE10FA44BFD1
:10D0300030EE270A37EE400AD8E79FED0A0A70471C
:10D04000DB0F4940DB0FC940DB0F49C0DB0FC93F95
:10D050009A7C2E36FAAF4FB93587083CA4AA2ABE6F
:10D06000DB0FC9BF00000000DFED027A30EE270AB7
:10D0700098E700BFDB0FC93F10B51C46334BB3FB2D
:10D08000F2F399429FED325AF0EE404AF7EE005A21
:10D0900053D207EE901A9FED2F7ADFED2F6AF8EE4C
:10D0A000677AF8EE002A67EE877A07EE102AB8EE64
:10D0B000477A27EE267AC5EE876A87EEA64AB0EE53
:10D0C000440AFFF76FFFF0EE403AB0EE440AFFF774
:10D0D000CBFF74EEA44A012C83EEA43A1CBF35EEBC
:10D0E000C04AF6EE006A33EE257A12BF64EE266A75
:10D0F000F0EE656A20EE224A86EE876AC4EE074AA1
:10D1000060EE227A75EEC35AC7EE876AC5EE877A5B
:10D11000F0EE465AC0ED005AC0ED014A80ED026AB9
:10D12000C0ED036AC0ED047A80ED065A80ED055A21
:10D1300080ED085A80ED075A10BDF0EE454AB0EE7A
:10D14000456AF0EE456AF0EE457AE3E720A1070074
:10D1500000000000DB0FC940BD378635B0EEE06A45
:10D16000F0EEC07AB4EEE76AF1EE10FAF0EE406A43
:10D170004BDCB5EE400AF1EE10FA4BD0B4EEE76AA4
:10D18000F1EE10FAF0EE675A41D5B0EE465A85EE50
:10D19000257ADFED225A9FED225ADFED224AA7EED3
:10D1A000255ADFED215AE5EE075A9FED205AA5EEEC
:10D1B000875ADFED1F5AE5EE075A9FED1E5AE7EE3C
:10D1C000054AB7EE005AA4EE875AB1EE657A87EEAB
:10D1D000050AB4EEE76AF1EE10FA48BFDFED167A01
:10D1E000F5EEC00A48BF37EEC00AF1EE10FA48BFAC
:10D1F000DFED127AF5EEC06A48BF37EEC00AF1EEF5
:10D2000010FA48BFB1EE400A7047F0EE465AB0EE51
:10D21000675ABCE79FED0A7ABBE700BF39094E3D6C
:10D22000E3B59EBE69A2163E88FA16BE45FE7FBFD4
:10D23000A7DFA8B499FB243FDB0FC93FDB0F4940B0
:10D240000000000044F25063984203DDA0F50C405A
:10D25000A0387047034B9842BCBF00F50C40A0308B
:10D26000704700BFB0B9FFFF48F69F43984203DD07
:10D27000A0F50C40A03870470028BCBF00F50C405A
:10D28000A030704791ED005A08B5B0EE450AFFF79F
:10D29000EBFEF0EE405AB0EE450AFFF783FE91ED4B
:10D2A000015AF0EE404AB0EE450AFFF7DDFEF0EE1F
:10D2B000403AB0EE450AFFF775FE91ED023AB0EE46
:10D2C000405AB0EE430AFFF7CFFEB0EE404AB0EE50
:10D2D000430AFFF767FE25EE806A63EEC07A24EE0C
:10D2E000847AC0ED017AF0EE467AE5EE077A25EE13
:10D2F000843A64EE806AC0ED037AF0EE437AE5EE9C
:10D30000667AA5EE067AE5EE436A23EE844A64EE79
:10D31000E34A65EEA35A80ED004A80ED025AC0ED63
:10D32000047AC0ED054AC0ED066A80ED077AC0EDCB
:10D33000085A08BD034600F1400100221A615A61F3
:10D340009A61DA6110338B42F8D11022002158F033
:10D35000C9BF91ED007AD0ED047AE7EE077AC0ED0F
:10D36000047AD1ED006A91ED017AD0ED057AE6EE0E
:10D37000877AC0ED057AD1ED006A91ED027AD0EDA1
:10D38000067AE6EE877AC0ED067A91ED007AD0ED66
:10D39000077A77EE877AC0ED077AD1ED016A91EDD1
:10D3A000007AD0ED087AE6EE877AC0ED087A91ED42
:10D3B000017AD0ED097AE7EE077AC0ED097AD1ED6E
:10D3C000016A91ED027AD0ED0A7AE6EE877AC0ED35
:10D3D0000A7A91ED017AD0ED0B7A77EE877AC0ED7B
:10D3E0000B7A91ED007AD1ED026AD0ED0C7AE6EE7F
:10D3F000877AC0ED0C7AD1ED026A91ED017AD0ED19
:10D400000D7AE6EE877AC0ED0D7A91ED027AD0EDD5
:10D410000E7AE7EE077AC0ED0E7A91ED027AD0ED42
:10D420000F7A77EE877AC0ED0F7A91ED007AD0ED22
:10D43000107A77EE877AC0ED107A91ED017AD0ED0F
:10D44000117A77EE877AC0ED117A91ED027AD0EDFC
:10D45000127A77EE877AB7EE007AC0ED127AD0EDC5
:10D46000137A77EE877AC0ED137AD1ED017AD1ED98
:10D47000006A91ED027A67EEA77AE6EEA67AE7EE09
:10D48000077A90ED007AA6EEA77A80ED007AD1EDCA
:10D49000016A90ED017AA6EEA77A80ED017AD1EDCE
:10D4A000026A90ED027AA6EEA77A80ED027A90EDFC
:10D4B000037A77EE277AC0ED037A70472DE9F043BF
:10D4C000034685B000F11007054600261C46AC4611
:10D4D00012E0F8EC016A1EED047AD4ED007AE6EE73
:10D4E000C77AC4ED007A98450EF1100EF1D10434DC
:10D4F000BC420CF1040C03D0A7F11008E646F2E799
:10D5000001361C46B646BEF1040F1DD000EB0E1CC2
:10D51000A84604F1100907E0FCEC016A18ED047A52
:10D52000E6EEC77AC4ED047ACC45D4ED047A08F16E
:10D530001008F1D1D3ED006A87EEA67A0EF1010E44
:10D5400084ED047A6446DEE7042E03F1140305F14A
:10D55000040507F11007B9D100230093019302934A
:10D5600003936C4600231427F2EC017A00EB0315B9
:10D5700007FB030C6E466545C4ED007A1FD10133ED
:10D58000042B04F10404EFD104AD103100F140028A
:10D5900075ED017A00EB03170E461446BC4241EDCF
:10D5A000017A13D152ED016A87EEA67A013BA2F10E
:10D5B000140221ED017AEBD105B0BDE8F083F5EC62
:10D5C000016AB6EC017AE6EEC77AD4E7F4EC016AB8
:10D5D000B6EC017AE6EEC77AE0E71FB50C460246E4
:10D5E00069461030FFF76AFFDDED007AB6EE007A8B
:10D5F00067EE877A0120C4ED007ADDED017A67EEEF
:10D60000877AC4ED017ADDED027A67EE877AC4EDA0
:10D61000027A04B010BDF8B510EE100A10EE904A70
:10D6200052F032FA064620460F4652F02DFA3246A4
:10D6300004460D463B463046394652F07DFA2246B6
:10D64000064601F100472B462046294652F074FA5F
:10D6500002460B4652F0BAF802460B4630463946AF
:10D6600052F094FB41EC100B53F0CAFB51EC100B41
:10D6700052F05AFD00EE100AF8BDB5EEC00AF1EE08
:10D6800010FA08B506DB53F0E3FCB4EE400AF1EE05
:10D6900010FA01D79FED010A08BD00BF000000008D
:10D6A0002DE9F041044626461C3004F1640250ED99
:10D6B000017AB1EC010A77EE807A40ED017AFBF74E
:10D6C00050F918309042F2D12C4F6268D7F894315B
:10D6D00025699B1AA2680135934225612BD904F173
:10D6E0003008F36A012BC3BF03F1FF3307EE903A12
:10D6F00096ED0A7A9FED220AC4BFF8EEE77A87EE2C
:10D70000270AFFF7BAFF4645D4ED057A15D0F4EEA7
:10D71000C07AF1EE10FA06F11806E2D5237B4BBB76
:10D72000D7F89421626000222361A261E362226340
:10D730006364A264E365BDE8F081F4EEC07AF1EEC3
:10D7400010FAEBD407EE905AD4ED066AF8EE677A39
:10D75000022386EEA77AD4ED0C6A84ED067A86EE73
:10D76000A77AD4ED126A84ED0C7A86EEA77A84ED5E
:10D77000127A00E003232370DDE700BF882B00202E
:10D780000000000070B52DED028B0378012B0446DC
:10D790003CD10569254E25B9426812B9D6F89421C5
:10D7A000426094ED068A30EE088A013584ED068ADF
:10D7B000256104F11C00FBF7D4F86268D6F89431B7
:10D7C0009B1AA268934221D9E36A012BC3BF03F1DC
:10D7D000FF3307EE903A94ED0A7A9FED150AC4BF25
:10D7E000F8EEE77A87EE270AFFF747FFD4ED057AD0
:10D7F000F4EEC07AF1EE10FA0ED5237B4BB9D6F8D1
:10D800009421626000222361A261E362BDEC028B7D
:10D8100070BD03232370F9E707EE905AF8EE677A9C
:10D82000022388EE277A84ED067AF3E7882B00201E
:10D830000000000008B52DED028BF0EEC08AB0EEBE
:10D84000408AB7EE000A30EE680AFFF716FF9FED38
:10D850000E7ADFED0E7AE8EE877A9FED0D7AA7EE6D
:10D86000A87ADFED0C7AE7EE287AB5EEC08ABDEC37
:10D87000028BF1EE10FA20EE270A44BFDFED067AA4
:10D8800037EEC00A08BD00BF306E99BC2716983D20
:10D89000843459BEA40DC93FDB0F494060EEA00A95
:10D8A000E0EE000AB0EE600AE7E660EEA00AE0EE05
:10D8B000000AE1EE010AB0EE600ADEE62DE9F74F5C
:10D8C00090469DF83020002A0CBF4FF0200A4FF000
:10D8D000300A0D9A1C1E05460F46BABF64424FF02F
:10D8E000010B4FF0000B12F8011B01B14CB9BBF159
:10D8F000000F2DD1264636B9A1464FF0FF340D9EBC
:10D900000FE0013CEFE7BD4202D251462846C04736
:10D91000013EF0E7BD4203D201922846C047019A7A
:10D920001646324612F8011B0029F3D10D9BA9EBD4
:10D9300003094E44BBF1000F06D0A146B9F1000F18
:10D9400009DC002CA8BF3619304603B0BDE8F08FC3
:10D950004FF00009D3E7BD4202D251462846C047E6
:10D9600009F1FF39EAE70FB437B50C4D06ABD5F82E
:10D97000D01853F8042BD5F8CC08019351F000FDD2
:10D980000446D5F8240203F0BDFD0028F9D0204656
:10D9900003B0BDE8304004B0704700BF882B0020C2
:10D9A0000EB403B503AB084953F8042BCDE900309E
:10D9B00001A851F0E5FC019B00221A7002B05DF84D
:10D9C00004EB03B0704700BFB58900080CB430B554
:10D9D0002C4CD4F8D438A5B01BB9D4F8D838002BC7
:10D9E00039D094F8DC38994206D9012303FA00F0C3
:10D9F000D4F8E03818422ED0D4F894114FF47A734A
:10DA000004A8B1FBF3F203FB12131F49FFF7C8FF91
:10DA100004AB0344289A1D490393054629AB03A888
:10DA2000029351F0ADFC039B591C03910A2119701C
:10DA3000039B591C0391002119700246D4F8D408A5
:10DA400090B103685B6A03B19847D4F8D45804AC2A
:10DA500014F8011B21B925B0BDE8304002B0704771
:10DA6000284603F025FDF3E7D4F8D838002BF2D090
:10DA700015440222009204A9AA18FD202AF02CFBCA
:10DA8000E9E700BF882B0020B7200708658700085A
:10DA9000174A38B5D2F8E458033005EB9003B3F5D4
:10DAA000007F19D802F6E804C2F8E438114A02EB04
:10DAB000810120F0030051F8102CC3F500730244DB
:10DAC00041F8102C9B000C4A0421002004EB850433
:10DAD000FFF77CFF204638BD0021084A0846FFF7C3
:10DAE00075FF074A136843F0007313600024F1E7E1
:10DAF000882B0020803C0020C3200708E72007086F
:10DB0000C06D01202DE9F0470368214F0546002430
:10DB100057F83420934213D11E4E06EB84094FEA86
:10DB20008408D9F828A2BAF1000F21D10721642076
:10DB3000FFF7AEFF0146C9F8280260B9164A04E0B3
:10DB400001340E2CE4D1154A00210520FFF73EFFD9
:10DB50000020BDE8F0876422514658F0C3FBD9F895
:10DB6000283207EBC407C3E90073DB615B63DB6446
:10DB700046446879D6F82832182404FB0032002184
:10DB80001046C2E90311956011750430E1E700BF4A
:10DB9000AC750608882B00201A210708F520070815
:10DBA00003685A1C026019700368090A5A1C026053
:10DBB0001970704703685A1C0260197003685A1C78
:10DBC00002600A0A1A7003685A1C02600A0C1A7072
:10DBD0000368090E5A1C02601970704738B5044674
:10DBE0000068154657F05CFA23682B44236038BD63
:10DBF00003685A1C02601878704703685A1C026058
:10DC00001A4612F8021B0260587841EA0020704759
:10DC1000026810B5531C0360134613F8021B03601F
:10DC2000D31C5478036093781B0443EA04230B430A
:10DC3000111D0160D07843EA006010BDD1E90032C7
:10DC40009A4206D05A1C0A6008B11B780370012062
:10DC5000704700207047D1E900239B1A012B10B5B3
:10DC60000446084604DDFFF7C8FF2080012010BDF0
:10DC70000020FCE7A0F16103192B98BF2038704702
:10DC800038B505460024284651F092FDA04200D840
:10DC900038BD2B5DA3F16102192A9CBF203B2B5597
:10DCA0000134F0E730B50A440546914201D1002025
:10DCB00011E015F8013B11F8014BA3F141001928BF
:10DCC000A4F1410098BF2033192898BF2034181BB5
:10DCD00001D1002CE9D130BD6FF00042E2E710B570
:10DCE0000388827803F003010C24013A04FB01222B
:10DCF0001149847901EB4202A3F5FA63B2F8F220EC
:10DD000040F2B5519B0801FB0323C278013A13444A
:10DD10000279182101FB0323427900893C2101FB90
:10DD20000322064B234401FB02334FF47A72002195
:10DD3000C3FB020110BD00BF4075060880436D386B
:10DD4000F8B519460446002310464FF47A7252F093
:10DD500049FB244B3C25034493FBF5F005FB1033B2
:10DD600090FBF5F105FB110060711820A37191FB88
:10DD7000F0F300FB131140F2B550217193FBF0F169
:10DD800000FB1133B3F5896F4FEA810526DA40F2C3
:10DD9000DA218B4224DCB3F5B77FB4BF0020012029
:10DDA000114E182101FB00660B2136F811709F42BD
:10DDB00001DD0139F9D105F5FA65054425804D1CD1
:10DDC000A5700C2505FB00110848228100EB4101DC
:10DDD0000133B1F8F2105B1AE370F8BD0320DFE7FE
:10DDE0000220DDE780BC92C732760608407506083F
:10DDF000F0B5294D07460E460FCD8DB06C460FC4C9
:10DE00000FCD0FC495E80F0084E80F0017F003034F
:10DE10003FD1642197FBF1F201FB127242B94FF43A
:10DE2000C87297FBF2F302FB1373003B18BF012388
:10DE30007A1EC3F11D03002A019340F26D131146AF
:10DE400007FB03F3B8BFB91C03EBA1036FF0630139
:10DE500092FBF1F10B444FF4C87192FBF1F21344C1
:10DE60002533072493FBF4F2C2EBC2029B1A013E56
:10DE70006D46002155F8040F01310344B14293FB74
:10DE8000F4F2C2EBC202A3EB0203F3D1C01A0DB04D
:10DE9000F0BD0123CCE700BF94760608084BD3E918
:10DEA0001E1251EA020309D0064BD3F894315B18D5
:10DEB00042F10002C0E900320120704700207047A3
:10DEC000803C0020882B002037B505466846FFF7C8
:10DED000E5FF044638B1DDE900232846FFF730FFAF
:10DEE000204603B030BD40F2011328806B80A8802B
:10DEF000A8712881F4E737B50546FFF7E5FF04462A
:10DF000050B1074B0DF10602B3F88030ADF8063082
:10DF1000294628464DF014FA204603B030BD00BF14
:10DF2000803C00202DE9F041044686B094F8303062
:10DF3000042B13D8DFE813F0150005005D00E9009D
:10DF40003601DFF8688204F11C0701AA3946404611
:10DF5000FEF7FDFC01280CD002282AD006B0BDE84F
:10DF6000F08192484DF06AFC4FF6FF732384012341
:10DF70003CE0019D0DB12B7863B98C48FDF760FF43
:10DF8000237EDD0618D54DF059FC4FF6FF73238430
:10DF900002232BE0EE7A3007D7D40B2204F13101B3
:10DFA000284656F0F9FF0028CFD1637E7340D9068A
:10DFB00004D57E48FDF744FF042317E0AA8A6B8B43
:10DFC00043EA02437A4A6362D2F81022EB69A36003
:10DFD0005202B3FBF2F102FB113109B113445B1A97
:10DFE0007248E3606676FDF72BFF032384F8303038
:10DFF0009CE76F4E96F8E031002BAFD104F11C087E
:10E0000006F5DC7701AA41463846FEF7A0FC012858
:10E0100059D1019D002D38D02B78E52B01D0002B54
:10E02000F0D1644BEB1A48BF03F2FF13B3F5805FE6
:10E030004FEA632003D3FDF7F3FF4FF0FF305E4953
:10E0400001EB0010FAF770FA01F5D070FDF7F8FE59
:10E0500020220021284658F045F9D4F831302B60B1
:10E06000D4F835306B60B4F839302B8194F83B30FC
:10E07000AB72637EEB7203A8FFF73DFF38BB6FF016
:10E080007E032B7447236B743AE096F8B831022B69
:10E0900092D096F8E031002B8ED10922C6E97D336B
:10E0A00086F8E02186F8F031D6F8CC2186F8EC31FC
:10E0B0003E48D6F81432C6F8E421C6F8E831FEF737
:10E0C0005BFA01289ED002283FF476AF46E79DF820
:10E0D0000E209DF80F3043EA4213BDF80C20A2F247
:10E0E000BC7243EA42232B829DF811309DF8122026
:10E0F0005B0143EA52039DF8102043EAC223EB81FF
:10E100002B8A2B83EB89EB826FE7237E9A0608D557
:10E11000E0690023112202A9FDF790FF01287FF496
:10E120001DAF20464DF08AFB2269237E9AB91B075A
:10E1300008D51F4B93F89821002A7FF40FAF0722D0
:10E1400083F89821002384F82830E36A204606B03B
:10E15000BDE8F041184703F0F70213F004032276FC
:10E160000AD0E26AA1680023204684F8283006B06D
:10E17000BDE8F041FDF708BF122AE3D1E26AA263CD
:10E18000626A84F83C3004212046C4E90B22C4E9C9
:10E19000023384F828106363636206B0BDE8F0417F
:10E1A0004DF04CBB0020E36A2070D0E7786000207F
:10E1B000C05E0020D84E0020D85E00202DE9F3413B
:10E1C00003780446002B76D090F82830013B082BCA
:10E1D00071D8DFE803F00509475B4C6170666B009E
:10E1E00002B0BDE8F0419DE6344B4568D3F81072AB
:10E1F000D3F818327F021D40216B2046FDF75AFEEE
:10E2000005EB01084745064626D880B1D4E901321E
:10E210009A422CBFA260A360002384F82830E36AEE
:10E22000002B48D0204602B0BDE8F04118472169D4
:10E23000207E01AA50F01EFA01283CD123696361B7
:10E24000019B236163683B445B1B6360236BDB1BA7
:10E250002B4423633546CFE70028D7D163680B44AE
:10E260006360D3E702B0BDE8F041FEF705BB0121D2
:10E27000FEF774FA01281ED1216C0023204684F891
:10E28000283002B0BDE8F041FEF74ABB002102B0E1
:10E29000BDE8F041FEF762BA02B0BDE8F041FEF71A
:10E2A000FDB902B0BDE8F041FEF701B902B0BDE82A
:10E2B000F041FEF761B902B0BDE8F081C05E002018
:10E2C000F0B50124B0FBF4F58D4203D200261CB951
:10E2D0001C70F0BD4C43F5E7B0FBF4F5B4FBF1F76F
:10E2E00004FB15002EB9002D03DC8C420CD33C46F8
:10E2F000EDE7092D08DD002A0CBF572437242C44F4
:10E3000003F8014B0136F2E73024F8E703463038D2
:10E31000C2B2092A0FD9A3F16102052A02D8A3F1DA
:10E3200057007047A3F14102052A02D8A3F1370034
:10E3300070474FF0FF30704770B50446944208466E
:10E340001546B4FBF2F602D33046FFF7F5FF05FBA6
:10E350001644024B1B5D00F8013B70BD3F210708CE
:10E36000B5EEC00ADFED2D7AF1EE10FACCBF30EE3B
:10E37000270A30EE670ADFED2A7A20EE270A30B549
:10E38000FDEEC07A87B017EE904A054684EAE47045
:10E39000002303A9A0EBE470CDE9003302934DF014
:10E3A0003DFA002CB4BF2D23202303A88DF80030A4
:10E3B00051F0FEF9012822D130238DF8013043F2CB
:10E3C0003003ADF8023003A9684658F043FE6846B2
:10E3D00051F0EEF9C41EE4B222466946284656F0D2
:10E3E0005FFE00232B550F49284658F033FE0DEBF6
:10E3F0000401284658F02EFE284607B030BD0228FA
:10E4000005D130238DF801308DF80230DBE7032889
:10E4100004BF30238DF80130D5E700BF6F12033AF7
:10E4200000007A446D58070830B50278202A034668
:10E4300000F10100F9D0092AF7D02D2A4BD103466B
:10E44000BFEE000A9FED3C7A1A46F2EE046A1346CC
:10E4500012F8010BA0F13001CCB2092C41D92E28C1
:10E460000BD1F2EE046A1146B0EE666A0B4611F863
:10E47000012B303AD0B209283CD91A7802F0DF02D9
:10E48000452A53D15A782D2A3FD102330120013B2E
:10E4900000220A2513F8011F3039CCB2092C3AD9D1
:10E4A000B2F59A7F1346DFED256A28BF4FF49A73C1
:10E4B0001A46F7EE007A072A30D8DA086FF007011B
:10E4C00001FB0233F2EE046A63BB88B3C7EE276A2E
:10E4D00020EE260A30BD2B2A08BF0346B7EE000AFD
:10E4E000B0E707EE901AF8EEE77AE7EE267AB0EE9C
:10E4F000677AACE707EE902AF8EEE77AC7EEA65AFD
:10E5000066EE866A37EE257AB0E72B2A14BF013310
:10E5100002330020BBE705FB0212BBE767EEA67AD9
:10E52000083AC8E767EEA67A013BCDE7F7EE007A36
:10E5300067EE276ACCE700BF0000000020BCBE4C9D
:10E5400070B5034610F8012B202AFAD0092AF8D01A
:10E550002D2A0ABF034601254FF0FF35591E00241E
:10E560000A2611F8010FFFF7D1FE092802D905FB91
:10E5700004F070BD06FB0404F3E710B50023802807
:10E5800004D893420AD2C854581C10BD934205D0F7
:10E5900060F07F04CC54C0090133F0E74FF0FF3046
:10E5A000F3E7F8B5144D2B787E2B23D101222946B1
:10E5B0000020FEF741FC114F6C1C228862B1A31DA4
:10E5C000BB4217D2A618BE4214D2052A12D9214640
:10E5D000FEF732FC3446F0E702222146FEF72CFC1F
:10E5E0006388074AC31A0434641B5842A2F81A42CB
:10E5F0005841F8BD0020FCE70040000800800008FA
:10E60000803C00202DE9F04F724BDFF8DCB18FB079
:10E61000A3EB0B02CDE901234FF0030810220021E8
:10E620000AA857F05FFE019B0993029B08936A4B6F
:10E63000CDF81CB01A69002ABFBF684A5A6002F1BF
:10E6400088325A600124F322DA604FF000097E23F9
:10E65000224604A907A88DF83440CDF830908DF8F3
:10E660001030FAF759FA4845C0F2A180224604A9B1
:10E670004846FEF7E1FB5A4CADF81200594B9C425C
:10E680003CD30024022205A907A8ADF81440FAF7EC
:10E6900043FAA042C0F28B80BDF81200022205A905
:10E6A000FEF7CAFB0222ADF812000DF1120107A815
:10E6B000FAF732FAA0427ADB0B9880B1079B089AEE
:10E6C0000344934273D80AABC0F1040221461844B4
:10E6D00057F008FE0AA907A8FAF77AF90C900C9BE4
:10E6E000002B64DB9DF8342022B13B490A6942F0DB
:10E6F00000420A61B3FA83F35B0959E062888DF83E
:10E700001990C2F30B06B31DADF814302388C3F380
:10E710000B011B0B8DF818301304ADF816101ED426
:10E72000062205A907A8FAF7F7F900283FDBBDF88C
:10E730001200062205A9FEF77FFB676805463246F0
:10E74000394607A8FAF7E8F9002830DB324639469F
:10E750002846FEF771FBADF8120014348EE700274F
:10E760003D460135EDB2062205A907A88DF81950DE
:10E77000FAF7D2F900281ADBBDF81200062205A923
:10E78000FEF75AFB616882463944324607A8039176
:10E79000FAF7C2F900280ADB039932465046FEF721
:10E7A0004BFB032DADF812003744DAD1D5E7002337
:10E7B000B8F1010808D0002B3FF430AFFFF7F1FEAD
:10E7C00020B10FB0BDE8F08F002BF7D1052005F088
:10E7D000FBF900BF00800008003C024023016745B0
:10E7E000208207087087070800400008034AD2F813
:10E7F0001C3223EA0003C2F81C327047803C002020
:10E80000034606490648884201D300207047028823
:10E81000C2F30B029342F9D01430F4E77087070873
:10E820002082070870B544880B460546C4F30B04E4
:10E8300022460021184657F055FD2969084A9142A1
:10E84000034607D3074A914205D22246BDE87040ED
:10E8500056F026BC19B1BDE870401846084770BD97
:10E86000708707088B8C070810B4B0F90240428803
:10E87000002C0B4641685DF8044BBEBFC2F30B028F
:10E88000DBB203FB0211CDE730B5094B094CA342C3
:10E8900000D330BDB3F902205988002A06DA5A683D
:10E8A000DD68C1F30B0100FB01222A601433EEE79F
:10E8B000208207087087070830B50246014400200F
:10E8C00012F8015B082480EA050343F3000323F0F8
:10E8D000730383EA5003D8B2631E13F0FF044FEAB8
:10E8E0005505F0D19142EBD130BD2DE9F04F87B005
:10E8F000CDE903230025804601910095039B404606
:10E90000EC0003EBC50AFBF7DBF8002800F097806A
:10E91000002201214046FBF7BDF80290002800F0DC
:10E920008E8098F804309A0706D4029A049B104609
:10E930001D7007B0BDE8F08FF0214046FBF7CAF824
:10E9400000287CD0039BA4F108024FF0000B0126A5
:10E95000134434465F460593019BB3B3082C34D867
:10E9600004F1FF3943FA09F909F001094946404623
:10E97000FBF767F8002862D0002201214046FBF730
:10E9800089F8024600285AD098F8041001F0600C6B
:10E99000BCF1600F4FEAD11037D0019B1BB1082C9E
:10E9A00001D88145C1D120B31AF807103143760050
:10E9B000013416F0FF060AF80710E4B2CCD1013793
:10E9C000FFB2082F21D00126C6E75DB1009BA3420C
:10E9D00008D9059BDA5D164214BF4FF001094FF0CC
:10E9E0000009C3E7009B1B1BD3F1000949EB030996
:10E9F000BCE7880940EA511111F0010F1AF807101D
:10EA000008BFA34621EA0601D1E7402C11D907210E
:10EA100050460292FFF750FF9AF80740029A84424C
:10EA200007D10135EDB2BBF1000F3FF47FAFCDF858
:10EA300000B0049B1B78AB423FF660AF76E7002244
:10EA400074E700BF0000000090F83C20034602F08D
:10EA5000FF0012B1002283F83C2070474FF480532E
:10EA6000838170474FF40063838170474FF40063E4
:10EA7000838170474FF40063838170474FF40063D4
:10EA8000838170474FF40063838170474FF40063C4
:10EA90008381704710B5064A0423002152F8044BC5
:10EAA000844208BF42F8041C013BF7D110BD00BFEF
:10EAB000E8600020324BF0B5188ADC8BB3F928509F
:10EAC000B3F92270B3F918E0B3F93060001B9C8BE6
:10EAD0006043B3F9264005EBE035E40294FBF5F41E
:10EAE00004EBE034A4F57A60B3F91650DC6200FB65
:10EAF00000FC4FEA2C3C45430CFB07F700FB0EFEE5
:10EB0000ED12B3F9200005EBE725B3F914700CFB07
:10EB100000F0001405EB8705B3F81AC05B6B00EB3F
:10EB20006E30B54002300235A3EBA50580104CF2E3
:10EB3000503300F5004033416B430CFB00F04FEACB
:10EB4000D03055BF5B00B3FBF0F3B3FBF0F35B00D9
:10EB500071B1181240F6DE3540436843094D001488
:10EB60005D4300EB254000F6CF6003EB20130B6004
:10EB700022B10A235C430834241114600120F0BD43
:10EB8000E860002043E3FFFF012070470120704749
:10EB90002DE9F74F604E9046B38FB26BB6F94CC07B
:10EBA000B6F94A70B6F948B0C3EB22155B00C3EB67
:10EBB000E203B6F93E206D435343B6F940202D13CE
:10EBC0005543AD1305EBE325B36D0093A5F5FA307E
:10EBD000B6F946307565894680FB001EDA1703FBDF
:10EBE0000EF401FB0244A3FB01321444B6F94420A5
:10EBF00082FB00A21B0A120343EA046342EA1A5290
:10EC00004FEA0A3A13EB0A0342EB2422B6F842A079
:10EC100002F500420192A3FB0A23019A0AFB023A81
:10EC20004FEAEA734FEA6A0253EA6A0A4FF00004B5
:10EC30005ED087FB00704FEAEC7A0CFB0EFE4004BE
:10EC400001FB0AEE40EAD730ACFB011C7F047F18C1
:10EC50000099F4444CEB0000C1F5801C0CF000411D
:10EC6000E71941EA5C014FEACC7CBCEB070C40F6AB
:10EC7000354400EBCB0061EB0001ACFB040C04FB62
:10EC800001C151F0AFFB84460746430BB6F9520071
:10EC90004A1343EAC14300FB02FEC41703FB04EE20
:10ECA000A0FB03407044624303FB0022A4FB034328
:10ECB0001A44B6F95030640E44EAC2144FEAE37EB7
:10ECC00003FB01F0E4190EFB0C00A3FB0C373844E6
:10ECD0004FEAD34343EA403341EB6262E41842EB2C
:10ECE000E042B6F94E30240A44EA026404EB03140D
:10ECF000B9F1000F02D0240AC9F80040B8F1000FA2
:10ED000005D005EB850580352D12C8F8005001208F
:10ED100003B0BDE8F08F00BFE860002031B10A4BBE
:10ED2000D3ED1E7AFDEEE77AC1ED007A52B1064BC3
:10ED30009FED067AD3ED1F7A67EE877AFDEEE77ACC
:10ED4000C2ED007A01207047E86000200000C84250
:10ED50002DE9F74FCDE90012574AB2F88E30D2F8BC
:10ED60008010B2F88A60B2F890701B02C91AB2F82B
:10ED70008C306EEB0E0EA3FB010403FB0E44B2F8C5
:10ED80008830C00940EA44601B04C018A6FB013566
:10ED900006FB0E55B2F886604FEA132343EA05637B
:10EDA0004FEAC6364FEAE41444F100049B19A7FB6E
:10EDB000012607FB0E664FEAD25242EA46224FEA8C
:10EDC000252545F10005F61512F5FA6C46F1000B04
:10EDD000BCF5FA6F7BF1000750DA02FB06F8A2FBE4
:10EDE00002794FF0050A09EB4809A7FB0A780AFBEC
:10EDF00009884FEA570949EAC879BF08B0EB090901
:10EE000047EA887764EB6804DF1B3B462B4F65EBD2
:10EE1000A805BC454FF0FF377BEB0707484622DAD1
:10EE200040F6AC57D21946F100065643A2FB0272D7
:10EE300002EB46024FEAC208FE00BE1B48EA5778C2
:10EE400062EB0808361844EB08044FF00B08304614
:10EE5000A7FB087608FB02627F0847EAC277DF1B40
:10EE60003B4665EB620501FB0EFEA1FB011202EBC6
:10EE70004E02C90F41EA4201BCEB010C009A9AB163
:10EE80000D4AD2F89410A1FB033201FB05225B0D61
:10EE900043EAC2231B1A4FEA625262EB0402DB0B05
:10EEA00043EA4243009A1360019B0BB1C3F800C0D0
:10EEB000012003B0BDE8F08FE860002024FAFFFFD6
:10EEC00001207047B0F900305943084B994208DBE4
:10EED000B1F5000F07DA0029B8BFFF31081200B200
:10EEE00070470348FBE747F6FF70F8E701FF7FFF35
:10EEF0000080FFFF064B0022C3F89820C3F89C2037
:10EF0000C3F8A0200022C3F8A4200120704700BF4E
:10EF1000E8600020104B1A68104BD3F8A410521A66
:10EF2000FA2A16D8D3ED267AFDEEE77A17EE902A64
:10EF3000D3ED277AC286FDEEE77A17EE902AD3ED5D
:10EF4000287A0287FDEEE77A17EE903A4387012090
:10EF500070470020704700BF1C2D0020E860002093
:10EF600090F85F3230B53BB990F85D1290F85E32A0
:10EF70000124DAB2914200D830BDB0F8665204FAEA
:10EF800003F22A43A0F866220133F2E743790246EE
:10EF900013F0010006D0D2E90731D2685B1A013ABA
:10EFA00003EA020070474379024613F0020007D0DB
:10EFB000936A516A1269013B5B1A013A03EA020043
:10EFC000704710B5437913F0010304460ED0FFF7E4
:10EFD000DDFF034650B1226A6369E1689B5C013240
:10EFE000B2FBF1F001FB1022DBB22262184610BD29
:10EFF00043799B070AD5436A8269D154436A0269FF
:10F000000133B3FBF2F102FB1133436270474171EC
:10F01000704781717047D0E90920131A584258414E
:10F020007047024BD3F8A8305B681847E8600020AF
:10F03000024BD3F8A83008309B681847E8600020DE
:10F040000120704701207047012070470120704760
:10F050000120704731B10C4BD3ED2B7AF8EEE77AF3
:10F06000C1ED007A7AB1084BDFED086AD3F8B03011
:10F07000A3F5D543333B07EE903AF8EEE77A87EEF7
:10F08000A67A82ED007A7047E86000200000C8424E
:10F090000120704701207047094A30B505460A240F
:10F0A00000201368AB4205D1D3688B421EBF431CBE
:10F0B000D160D8B2013C02F11402F2D130BD00BFE0
:10F0C0009C0500207047054B40F2FF7203EBC00324
:10F0D0009142A8BF11469980704700BF503D002063
:10F0E000112807D8044B03EB8003D3F8B4300BB1DD
:10F0F0009B681960704700BFE860002008B5FFF703
:10F10000EFFFBDE808401EF0D7BF0C4A13787BB173
:10F110000B4B93F8FC1059B193F8FD1059B150689E
:10F120000021FA2883F8FD10A8BF4FF0FF30704788
:10F130006FF0010070476FF002007047F010002080
:10F14000E86000200B4B93F8FE206AB193F8FF2093
:10F150006AB1002283F8FF20074B9868B0F5967FCC
:10F16000A8BF4FF0FF3070476FF0010070476FF09D
:10F1700002007047E8600020F0100020024BD3F836
:10F1800000315B68184700BFE8600020024BD3F8ED
:10F1900000319B68184700BFE8600020024BD3F89D
:10F1A0000031DB68184700BFE8600020014BD868D9
:10F1B000704700BFF0100020044B93F8043113B1E6
:10F1C000034B186970476FF001007047E86000203A
:10F1D000F0100020014B5869704700BFF01000206C
:10F1E0002DE9F041062592F9007086B06B43144674
:10F1F00012F80580A0EB080EA0EB070CBEF1000F83
:10F20000B8BFCEF1000EBCF1000FB8BFCCF1000CBE
:10F21000E645B8BF541905F10605B8BF4FFA88F79F
:10F22000AB421646E4D11A4433786588BB420BD111
:10F2300073884D1BCB1A002DB8BF6D42002BB8BF91
:10F240005B429D42C8BF34460636B242ECD1637978
:10F25000049323790393638802932378054ACDE9C5
:10F260000013034603210120FEF7B0FB204606B041
:10F27000BDE8F081F82107084B1EDBB2062B9CBFCE
:10F280001C4AD25C1C4BF0B5A3F1580488BF4FF464
:10F290008072002808BF1C46234687B013F9087BFC
:10F2A0001888C8B9154B93F80501A3790593A3886D
:10F2B0000493A378039323880091CDE90123104A96
:10F2C000104B0321002818BF13460F4A0120FEF7F8
:10F2D0007DFB204607B0F0BD161AD51B002EB8BF27
:10F2E0007642002DB8BF6D42AE42BCBF1C4647B24D
:10F2F0000833D5E70077060864110020E860002095
:10F30000193E0708F56C07083122070808B50068A0
:10F310004EF033F8024BC3F88000012008BD00BF57
:10F32000E860002008B500684EF027F8024BC3F8EB
:10F330009400012008BD00BFE860002038B51446E5
:10F340000D46002943D0344B9FED347AD3ED427AF9
:10F35000B3F92421F8EEE77A06EE102AC7EE876AA1
:10F36000B3F92021D3ED437AF8EEE77AB8EEC66A16
:10F37000C7EE875A07EE102AD3ED457AB3F91C2160
:10F38000B8EEC77AB8EEE70AA6EE867AD3ED467AEB
:10F39000F8EEE77AE6EE877AA6EEA70A07EE902A5D
:10F3A000B3F92221B3F91E3106EE102A07EE103A06
:10F3B000B8EEC66AB8EEC77AF8EEE77AA6EE867AB5
:10F3C000E6EE877AA5EEA70A51F0ECFE28600CB3B2
:10F3D000114BDFED126A93ED437AB3F91021B3F9C3
:10F3E0001231B8EEC77A07EE902A87EE260A07EEAA
:10F3F000103AB8EEC77AF8EEE77A20EE070AB6EED2
:10F40000007AA7EE870ADFED067A20EE270A51F090
:10F41000C9FE2060012038BDE86000200000F04AED
:10F420000000C842094B10B553F8304007EE901A5F
:10F430005CB1F8EEE77A94ED047A94ED030AA7EE56
:10F44000870A51F0AFFEA368186010BD503D002040
:10F4500010B50C4B0C4C1B68D4F828011B1AFA2B66
:10F4600006D9042018F020FD002084F82C0110BDDE
:10F4700011B1D4F830310B6012B1D4F834311360CB
:10F480000120F4E71C2D0020E86000202DE9F04168
:10F490000C4DDFF834802C686B6901271C400CB9D7
:10F4A000BDE8F081B4FA84F3C3F11F0307FA03F651
:10F4B00008EB830324EA0604D3F83801036898476D
:10F4C0006E61ECE7003C0140E8600020F8B583681D
:10F4D0001C686379DB0724D5A57994F85C3205F0C4
:10F4E00001073D46F3B1E06B43681A68D36AC3F382
:10F4F0004E03536294F86D32012B07D094F86132B9
:10F5000023B1B4F868320133A4F8683285F0010100
:10F510004BF0EAFF0023A4F866324FF08073C4F882
:10F520005C32F8BD94F85F62012E04BF94F85D323E
:10F5300084F85E322046FFF713FD4EB9012384F8AC
:10F540005F3287EA0301E06BBDE8F8404BF0CCBFC7
:10F55000002384F85F323946F5E7F0B52DED028BD4
:10F5600083B00E46154647F0B7FF002869D022F059
:10F570005DFC354B354C1B6803F00203002845D079
:10F58000002B59D0324F0DF1060023F02BFBD7F89A
:10F590006425BDF806309FED2F7A9B1A07EE903A4E
:10F5A000F8EEE77AF0EE408A67EE877A9FED2A0A56
:10F5B00027EE800AFDF758FD07F5AF6797ED008A43
:10F5C000A0EE688A40F0C8FF54ED2E0AD0ED057A0F
:10F5D000B0EE480A70EEA70AFEF760F97EB1DFEDE3
:10F5E0001F7A9FED1F7A20EE000A20EE270AC0EE58
:10F5F000077A9FED1C7A77EE877AC6ED007A0DB117
:10F60000194B2B6003B0BDEC028BF0BDA3B134F9F4
:10F610009C3C01EE103A34F99E3C00EE903A34F9ED
:10F62000A03C00EE103AB8EEC11AF8EEE00AB8EECF
:10F63000C00AFEF73AF9D1E754F8843C93ED330A57
:10F64000CCE79FED0A0AC9E7686E0120E07100204F
:10F65000E86000200AD7233C35FA8E3CCDCC9C3F95
:10F6600000409C4682E6C5473313904300000000EB
:10F6700070B50446012027F0B7FB58B103684BB1C1
:10F680001C4A237992F83D10994231D092F83C20DF
:10F690009A422DD0184B5E68730612D500212720A0
:10F6A000FAF7B4FB002105462620FAF7AFFB1DB19F
:10F6B0002A6823689A421BD018B1026823689A42CC
:10F6C00016D0F5030CD521680C4B0A22186881422C
:10F6D00002D1D868C0010BD4013A03F11403F5D16B
:10F6E0002079112804D0A0F121035842584170BD5F
:10F6F0000120FCE750030020686E01209C050020DB
:10F7000000684DF07EBB08B5202157F0B2FC0346DF
:10F71000184623B10278202A03F10103F8D008BD6E
:10F7200070B50D461446FFF7EEFF0646A0B1FEF792
:10F7300007FF40F634039842A8BF1846B0F5617F32
:10F74000B8BF4FF46170A0F561731922B3FBF2F3F7
:10F750002B702378013323703046FFF7D4FF064621
:10F76000A0B1FEF7EDFE40F634039842A8BF18465C
:10F77000B0F5617FB8BF4FF46170A0F561731922D5
:10F78000B3FBF2F36B70237801332370304670BD06
:10F79000144B53F8200070B508B3134D0C2202FB34
:10F7A000005212F97F3C591C1AD012F8770CB0B1F4
:10F7B000E9188C2411F82C6C12F8781C0020142203
:10F7C00063435C1805EB4404013A34F8284C314497
:10F7D00010FA84F0F5D11423B0FBF3F080B270BDC1
:10F7E0000020FCE7E8600020E071002038B503202D
:10F7F0000D461446FFF7CCFF07EE900A8DB19FED42
:10F800000B7AF8EE677AF0EE006A67EE877AB8EE68
:10F81000047AA7EEA67ADFED067A67EE277AC5EDC1
:10F82000007A0CB1034B236038BD00BF6740533AE8
:10F8300000007A443313904310B5427A044632B143
:10F840000146406851F80A3B98470023637210BD97
:10F8500010B4447A621C0444D2B24272A172037A98
:10F86000934202D85DF8044BE6E75DF8044B70471D
:10F87000EEE710B503681A79022A044602D1987A95
:10F880004DF06CFD00232371236010BDF0B50D4BCE
:10F890000D4E0446B34201D30020F0BD5879884292
:10F8A0000DD11D79A54200D04CB9D879904206D12E
:10F8B00018680779AF4202D105689D42EDD00C333C
:10F8C000E8E700BFA00100085C03000837B5034665
:10F8D0000079022830D11B4A93F91030009214228B
:10F8E0005343194C194AE358934227D0A2F5784262
:10F8F000934225D002F5806293421DD101F10802A6
:10F900000DEB02011A8811F8085C22F04002120483
:10F91000120C14211A8001FB00441A88E16822F0BD
:10F92000380231F825101204120C0A431A801A8882
:10F9300092B242F040021A8003B030BD0020DDE7F1
:10F940000120DBE700010203B0000020003001408D
:10F95000C36910B5044623B909211420FEF798F8AD
:10F96000E061E06910BD10B504460068FFF7F0FFE4
:10F970008378DBB1B0F90A3007EE903AF8EEE77A17
:10F98000C4ED057AB0F90C3007EE903AF8EEE77A5C
:10F99000F1EE677AC4ED047AB0F90E3007EE903AD2
:10F9A000F8EEE77A0120C4ED067A10BD1846FCE7B0
:10F9B00010B504460068FFF7CBFF8378CBB1B0F9F0
:10F9C000043007EE903AF8EEE77AC4ED047AB0F925
:10F9D000063007EE903AF8EEE77AC4ED057AB0F912
:10F9E000083007EE903AF8EEE77A0120C4ED067A87
:10F9F00010BD1846FCE710B504460068FFF7A8FFE5
:10FA00008378CBB18388DBBA07EE903AF8EEE77AD9
:10FA1000C4ED047AC388DBBA07EE903AF8EEE77AD1
:10FA2000C4ED057A0389DBBA07EE903AF8EEE77A7F
:10FA30000120C4ED067A10BD1846FCE710B5006839
:10FA40000C46FFF785FF0346807840B15B89222290
:10FA5000DBBA93FBF2F303F26D132380012010BD98
:10FA600038B500680D461446FFF772FFD0F8013034
:10FA700007EE103ACDB1D0F80530DFED176A9FEDF3
:10FA8000176A07EE903AF8EE677A77EEE67A77EE45
:10FA9000A77AC7EE866AF7EE007A76EEE77ADFEDB0
:10FAA000106A67EEE67AC5ED007A9CB1DFED0D7A5B
:10FAB000DFED0D6AB8EEC77A27EE277AC7EE267A11
:10FAC0009FED0A7A77EEC77A9FED097A77EE877A0B
:10FAD000C4ED007A38BD00BF9AC9CC449AC94C46DF
:10FAE0000E76D7450000484300E0FF44000048423E
:10FAF0003393884337B500680D461446FFF728FF57
:10FB0000D0F805309FED237A07EE903AF8EE677A49
:10FB1000F2EE046A77EEC77A9FED1F7AD0F80130D3
:10FB200067EE877AB3EE097A67EE877A07EE103AC6
:10FB3000F4EEE67AF1EE10FA06DCFAEE046AF4EE80
:10FB4000E67AF1EE10FA0CD517EE900A4FF09CFF12
:10FB5000124ACDE9000104210320FDF737FF03B06D
:10FB600030BD2DB1DFED0E6A67EEA67AC5ED007AE5
:10FB7000002CF4D0B8EE477ADFED0A6ADFED0A7A9E
:10FB8000E7EE267A9FED097A77EE877AC4ED007A60
:10FB9000E5E700BF00000046000080387B22070830
:10FBA0000AD778430319C83D000048C233938843FD
:10FBB0000379022B0DD190F9103014225343064AD9
:10FBC000D3581A89920746BF1889C0F3C010012084
:10FBD00070470020704700BFB00000200368DB6B57
:10FBE00013B504462BB923685B6B3BB9FF23E38253
:10FBF00002E098470028F6D102B010BD214601A8C6
:10FC000098470028F2D0BDF80630013B9BB2EEE7E2
:10FC1000036810B59B680446984701236374FF236B
:10FC2000A37410BD036810B504461B689847236889
:10FC300020469B689847E37C0133E37410BD03685A
:10FC400010B504465B689847236820469B68984730
:10FC5000E37C013BE37410BD2DE9F34104461846F3
:10FC600016460D461F464FF0A3FD2368E673284451
:10FC70000022A0730092D3F8148032463B462946F6
:10FC80002046C04702B0BDE8F08130B5046885B0B9
:10FC9000E469089D34B10DB90DF10F050095A04739
:10FCA00005B030BD2046FBE703685B6A1847036870
:10FCB0009B6A184710B5037B04460BB1437B13B90D
:10FCC0002046FFF7F4FF23682046DB68BDE81040BC
:10FCD000184703685B6C03B11847704738B5044692
:10FCE0008B6801600D4698470B4B236100232375F9
:10FCF0002B6B13B1204698472075084B93F820339F
:10FD00001BB1237D23F0010323750023E3822046EA
:10FD1000BDE8384062E700BF0001FF00E07100204D
:10FD200003681B6803B11847704703685B6803B139
:10FD30001847704703681B6A03B118477047036888
:10FD40005B6A03B11847704730B40468029DA46A27
:10FD50001CB10295A44630BC604730BC704730B43B
:10FD60000468029DE46A1CB10295A44630BC604759
:10FD700030BC704703685B6C03B118477047036879
:10FD80009B6C03B11847704703689B6F03B118471A
:10FD900070470368D3F8803003B118477047036891
:10FDA000D3F8843003B1184770470368D3F888301C
:10FDB00003B11847704721B10B68D3F88C3003B1F9
:10FDC00018470020704738B5094C052303FB004451
:10FDD000A13C0025013514F8010FEDB24DF043F9B7
:10FDE000052DF7D1BDE8384000204DF03CB900BFEB
:10FDF0000777060810B5441E14F8010F00B910BDAE
:10FE0000FFF7E1FFF8E7FFF741BBFFF73FBBFFF765
:10FE10003DBBFFF73BBBFFF739BBFFF737BB18B163
:10FE200003689B6803B11847002070470C4B93F898
:10FE3000212370B506460D468AB9D3F8244374B120
:10FE400023681B685BB12046FFF7E9FF38B12368E0
:10FE50003246196820462B46BDE87040084770BD01
:10FE6000E07100200120704718B103689B6803B15E
:10FE70001847002070470B4B70B5D3F8284306464F
:10FE80000D4674B123681B685BB12046FFF7ECFF99
:10FE900038B123683246196820462B46BDE87040C9
:10FEA000084770BDE0710020034620B1026812B11E
:10FEB000D26902B1104793ED017A084BB8EEC77AC8
:10FEC000D3EDCC6AF6EE007AE7EE267AFDEEE77A1D
:10FED00017EE900A00F30B00704700BFE07100209E
:10FEE000034620B1026812B1126A02B1104793EDC5
:10FEF000027A084BB8EEC77AD3EDCD6AF6EE007AF7
:10FF0000E7EE267AFDEEE77A17EE900A00F30B0093
:10FF1000704700BFE0710020034628B102681AB1A3
:10FF2000516A09B19369184793ED037A074BB8EE0C
:10FF3000C77AD3EDCE6AF6EE007AE7EE267AFDEECA
:10FF4000E77A17EE900A00F30B007047E07100208B
:10FF50004FF47A7300F50060584340F6FF7390FB4E
:10FF6000F3F000F57A70B0F5FA6FA8BF4FF4FA60BD
:10FF7000B0F57A7FB8BF4FF47A70704730B103683C
:10FF800082881B691A4214BF01200020704710B1FB
:10FF9000036882881A83704710B1036882885A8385
:10FFA000704773B50C46054600B30668104B06F162
:10FFB0003F4202F57E0203EB922393F8AA024BF034
:10FFC0000BFCAB88009304F003038DF80430C4F3FA
:10FFD00081038DF805306946C4F300133046640987
:10FFE0008DF806308DF80740FAF7B4FA02B070BD0C
:10FFF00000770608F7B50C4615460746A8B306680D
:020000040801F1
:100000001B4B06F13F4202F57E0203EB922393F86D
:10001000AA024BF0E1FBB8880090B0FA80F3C3F17C
:100020001F0303F00702C3F3CC0306EB8303920024
:10003000196A0F27974021EA07011962196A95404A
:100040000D431D6204F003038DF80430C4F38103F3
:100050008DF805306946C4F30013304664098DF805
:1000600006308DF80740FAF775FA03B0F0BD00BF0F
:100070000077060838B50409013C032C00F00F0294
:1000800019D80E4D05EB4403B3F8B01241FA02F350
:1000900013F001000ED001239340013B03EA01005D
:1000A000254457F0DBF895F8B832034404480C2295
:1000B00002FB030038BD0020FCE700BF0077060804
:1000C0001C7500202DE9F04F542204460021BE4843
:1000D00091B056F007F9BD49621E0846033412F884
:1000E000013F5D1E052D88BF0023944240F8043B6C
:1000F000F5D1B64A002352F8040B012800F05A81CA
:100100000133042BF7D1002351F8042B022A00F00D
:1001100047810133042BF7D10320FEF7BBFC0420F9
:10012000FEF7B8FC0520FEF7B5FC0620A64EDFF86A
:10013000B882FEF7AFFC34464FF01A0B4FF0000ABE
:1001400008F52F79277B57B3384694F90D50FFF700
:1001500091FF28B105238371002380F807B0037253
:100160001321FFF71EFF002319F83310B94240F0A6
:10017000DE8008EBC303D3F8C032954A236118230D
:1001800003FB0525D5F8E8302375591C0723A37513
:100190000123C5F8E810637585F8E4309A440BF143
:1001A000010B5FFA8BFBBBF1200F04F10C04C9D1EA
:1001B000BAF1000F00F0B880864DDFF830820027DA
:1001C0002B7C002B00F0A88068794BF005FB287988
:1001D0004BF002FBD5F808A05046FAF733F92C682B
:1001E000D5F81490CDF80C800023CDE90C33CDE97F
:1001F0000E330493069304F14C030293EB680193CE
:10020000142303FB09F34FF4806205934FF400635A
:10021000CDE907234FF400514FF48073CDE9091362
:1002200050464FF4003301A90B934BF0E7F9DAF88D
:100230000030694A43F00103CAF800305168674B47
:100240000B4043F4403353606268B9F1010F22F070
:100250004072D4BF0023012322F4807242EA0322B9
:100260006260A2685E4B134043F00203A360E26A3F
:1002700009F1FF3322F47002DBB242EA0353012298
:10028000E362304694464FFA87FE437D6BB390F9A4
:100290000D30734529D1037C90F81690092B4CD969
:1002A000A3F10A01D4F80CA001EB41014FF0070BB8
:1002B0000BFA01FB2AEA0B0A09FA01F141EA0A01E9
:1002C000E160062A48D8511ED4F8349001EB810130
:1002D0004FF01F0A0AFA01FA29EA0A0903FA01F1A2
:1002E00041EA090161630132D2B20CF1010CBCF1A7
:1002F000070F00F10C00C8D1A36843F40073A3609A
:10030000A36843F48073A360A36843F00103A36070
:10031000A36843F08043A3600137032F05F118055C
:1003200008F58C787FF44CAF11B0BDE8F08F013345
:10033000102B7FF419AF00231FE7216903EB430B58
:100340004FF0070A0AFA0BFA21EA0A0A09FA0BF136
:1003500041EA0A012161B4E70C2A10D8D11FD4F870
:10036000309001EB81014FF01F0A0AFA01FA29EAE5
:100370000A0903FA01F141EA09012163B3E7A2F195
:100380000D01D4F82C9001EB81014FF01F0A0AFAFD
:1003900001FA29EA0A098B4043EA0903E362A2E76A
:1003A000104B212203F8682C13F82C2C013203F88F
:1003B0002C2CB1E60B4B112203F8742C13F82C2CC7
:1003C000013203F82C2C9EE660710020E8600020CA
:1003D000F0100020C411002000230140E030FCFF99
:1003E000FDF7FFC0E071002000770608B87100201B
:1003F0002DE9F04F85B0B04D0293B04B9D4220D215
:100400006C798C4240F070812C79844202D00028B3
:1004100040F06A81EC79944240F066812C6884B1A6
:100420001C220021201D55F05DFF25602B792371D2
:10043000AA79A2600192012B2A7AE26006D0022BEF
:100440000DD00024204605B0BDE8F08FE87AFFF714
:1004500011FE6B7A2374AB7AA0616374F2E7E87AD9
:10046000FFF708FE95F90980A06184F81080A87A4A
:10047000FFF700FE07466061002800F03181142379
:100480008F4E03FB08F3F218F558002D00F0288179
:10049000937C002B40F0CB8092F8089048464BF0BC
:1004A0009BF909F01F024FEA59190123A9F102092A
:1004B0009340B9F1030F08D8DFE809F07872026CB5
:1004C00080490A6922EA03030B61142303FB0863D2
:1004D00008F101095879FFF7CDFD5FFA89F9034664
:1004E00020B140F60A32C28080F80890142202FB44
:1004F00008620393D079FFF7BDFD039B824620B1CC
:1005000040F60A52C28080F80890142202FB08626A
:1005100003939079FFF7AEFD039B834620B140F62D
:100520000A42C28080F80890142202FB086292F806
:100530000990019A12F0040201924A463CD04A21E5
:100540001846FFF757FD4A462A215046FFF752FD4D
:100550004A460A215846FFF74DFD142303FB086362
:1005600093F804A0BAF1000F06D05046FFF782FDC1
:100570004A460921FFF73EFD534B9D4223D103F527
:1005800084335A6A42F480525A625A6A22F4805280
:100590005A6225E04B494A6922EA03034B6194E71A
:1005A00048490A6A22EA03030B628EE745494A6A10
:1005B00022EA03034B6288E70A211846FFF71AFD77
:1005C0004A460A21C1E7414B9D423ED103F5003323
:1005D0001A6A42F480421A621A6A22F480421A624B
:1005E000019B002B65D1012202212B880A4303F4D1
:1005F0004153134343F445732B80AB8B23F40063C7
:100600001B041B0CAB8307232B822B889BB243F06C
:1006100040032B80BAF1000F04D05046FFF72AFDAB
:10062000FFF7B5FC142303FB08660123B374029B98
:10063000BB710E23FB71002338463B720921FFF783
:10064000B0FC3846FFF7A3FCFCE6214B9D4209D1E4
:1006500003F5FE331A6A42F400421A621A6A22F45F
:100660000042BCE71B4B9D4209D103F582335A6A15
:1006700042F400525A625A6A22F4005288E7164B3A
:100680009D4209D103F568435A6A42F480125A62C6
:100690005A6A22F480127BE7104B9D42A0D103F5E9
:1006A00064435A6A42F400125A625A6A22F40012EF
:1006B0006EE70022114698E7A00100085C030008DD
:1006C000B0000020003802400030014000380040F7
:1006D000003C004000340140005001400054014003
:1006E0002046FFF7C6F8ACE60C3587E6074B03EB70
:1006F0008003D3F83C333BB19A881B6859690A429E
:1007000001D05A8370471A83704700BF00770608EC
:10071000064B03EB8003D3F83C332BB11A689B885C
:1007200009B9138370475383704700BF00770608E9
:100730000A4B10B5D3F8884524B1094A0321204655
:10074000F9F792FB20460021F9F7E4FB2046054922
:10075000BDE8104040F62B424AF07ABFE07100201D
:10076000009F2400B49B002038B5104CD4F8885565
:1007700025B10F4A64212846F9F776FB0021284667
:10078000F9F7C8FB6B681A68B2F844306FEA434364
:100790006FEA53439BB2A2F8443013889BB243F0F4
:1007A00001031380012384F88C3538BDE0710020EB
:1007B000009F2400DFF8B0C12DE9F84F9CF88CE5CC
:1007C000BEF1000F40F0CC80DCF8889599F810302D
:1007D000002B40F0C5809CF890359CF891259CF842
:1007E0009255ACF88EE50CF29450F0463C26817898
:1007F000C778C1F1FF0189B2002900F0AD80C1F1D5
:10080000FF0179430488B4FBF6FA0912BAF1050F27
:1008100020D8DFE80AF0030D647283917A1A6243EC
:10082000B2FBF6F252FA81F2CDB2D2B23B460FE001
:10083000B4FBF6F306FB13439BB2C3F13C037A1AF5
:100840005343B3FBF6F353FA81F3CDB2DBB23A462E
:100850004FF0010E1F0247EA024747EA050B00214D
:100860000127C1F1170A07FA0AFA08EB01041AEA8C
:100870000B0F04F12A0408BFBA46A4B2394F01F1A4
:10088000010118BF4FF0020A182947F824A0E7D148
:1008900008F118081FFA88F8B8F5406F00F1040055
:1008A000A5D18021ACF89417BEF1000F05D08CF8CB
:1008B00092558CF891258CF890354FF44063ACF844
:1008C0008E359CF89637002B4AD0484640F62B418F
:1008D000F9F744FC4846BDE8F84FF9F771BCB4FBA2
:1008E000F6F206FB12427D1A92B25543B5FBF6F5BD
:1008F00055FA81F5CBB2EDB2A9E7B4FBF6F206FBEF
:10090000124292B2C2F13C027C1A6243B2FBF6F28E
:1009100052FA81F2CBB2D2B23D4699E7B4FBF6F57A
:1009200006FB15447B1AA4B26343B3FBF6F353FAF8
:1009300081F3CAB2DBB2EFE7B4FBF6F306FB134375
:100940009BB27C1AC3F13C03CAB26343B3FBF6F318
:1009500053FA81F1CDB269E73D463A463B4677E727
:10096000BDE8F88FB49B0020E0710020F8B5134B70
:10097000D3F88845054604B393F88C15C9B9E068E7
:1009800066688268136823F0010313603268777920
:100990000B4E938936F817609BB223EA06039381C6
:1009A000217413889BB243F0010313800177FFF792
:1009B000DBFE2046F9F7A4FB0560F8BDE0710020DE
:1009C0004075060838B5104CD4F8880550B194F835
:1009D0008C353BB194F89737032B04D1F9F790FB92
:1009E0006423036038BD022B4FF0000503D1F9F7F3
:1009F00087FB0560F6E784F88C55FFF799FE002821
:100A0000F0D184F89607EDE7E07100200346806B93
:100A10009B7903F00103994201D0FFF7B8BAFFF7C1
:100A2000BBBA10B5837913F0010F03F0200204461E
:100A3000C36B13D05B68002A1A7A08BF4221606B2F
:100A400018BF0221FFF7D6FA012184F86012A4F83A
:100A50005C12E06BBDE81040F9F768BB5B68002AE8
:100A600008BF22211A7AEAE7036C806B23B15B6826
:100A700001211A7AFFF7BEBA0121FFF792BA2DE9D8
:100A8000F04183681C686679B1072FD594F86152EC
:100A9000C5B194F962528DB1B4F864124B08A4F850
:100AA0006432204601F00101FFF7B0FFA379013D58
:100AB0006DB2580684F8625218D5BDB9002384F887
:100AC000613213E0A36A626A94F860129A4225D1F7
:100AD00061B9A3791A0709D5236CA06BD3B15B6800
:100AE0001A7AFFF787FA2046FFF79BFFF10740F1DC
:100AF000818094F85C32002B7CD194F85D32013314
:100B0000DBB2092B84F85D3235D12046BDE8F041D7
:100B1000FEF726BA1946FFF744FAE4E75A1CA06923
:100B2000A262C35C2069A7795B0043F40073A4F858
:100B300064320A23824228BF002284F862320123F1
:100B4000A26284F8613299B13B0711D5D4F83C8098
:100B500029464046F9F7EAFAD8F80430606B1A7A69
:100B60002946FFF747FA84F860522046FFF77CFFDA
:100B70007D068ED4BAE70A2B3CD194F85F322BB9AC
:100B8000B4F8663243F00103A4F86632B4F86602A2
:100B9000820501D4C3071AD4B4F86A320133A4F829
:100BA0006A3294F85F5201239D42A4F85C3221D14D
:100BB000A179E06B002384F85F3201F001014AF073
:100BC00093FCE06B2946BDE8F041F9F7AFBAE36A60
:100BD000C0F3470013B1216B9847E2E7E36962690C
:100BE000D054E369E2680133B3FBF2F102FB113345
:100BF000E361D6E7BDE8F081F8B51E4B46681A6898
:100C000004461346B3FBF1F0B0F5803F2ED281B21B
:100C10002046F9F729F923681F687C7974B165B219
:100C200003212846F9F70CF9002D07DB6109124A68
:100C300004F01F040123A34042F82130BC7974B1B1
:100C400065B203212846F9F7FBF8002D07DB61099F
:100C5000094A04F01F040123A34042F821303268FE
:100C600013889BB243F001031380F8BD012BCBD94D
:100C70005B08C7E70001002000E100E08160C06B75
:100C8000BAE7002ABCBF80185242002BBCBFC9186B
:100C90005B420028BCBF121A0020F0B5841800295E
:100CA000A4F11D04BCBF5B180021002CC8BF121B9F
:100CB000CC180F3C002CC8BF1B1B0B4E02440B442E
:100CC0003C274FF0200C90420CDC06EB40050C4614
:100CD00004E007FB04FE013425F80EC09C42F8DD59
:100CE0000130F0E7F0BD00BF7879002008B5114B66
:100CF0001A6C42F080521A640F4A012111620F4AA5
:100D0000FF215162CA215162532151625B6FDB00A6
:100D100009D400210120FAF73FF9BDE8084008494D
:100D20000020FAF739B90020FAF746F9044B984247
:100D3000EFD108BD0038024000000E4200280040FC
:100D400076614E6938B50C4605461946046014B103
:100D50002046F9F789F8BDF810102046F9F7DAF8BF
:100D600063681A68B2F844306FEA43436FEA53434A
:100D70009BB2A2F8443013889BB243F00103138066
:100D80002046F9F7BDF90023A860036038BD2DE9BE
:100D9000F04F85B006469DF83CA0039289469846E0
:100DA000FCF7B0FE834648B1214C94F8582B082A32
:100DB00009D9204A00210420FCF708FE0025284616
:100DC00005B0BDE8F08F531C5C21DFB284F8587B7E
:100DD00004F65C3501FB024402FB01550022C4F815
:100DE0005C2B84F8602B3079FFF744F9044620B17E
:100DF000022280F80690C2710772BDF83830009365
:100E0000039A434659462846FFF79CFFBAF1000F64
:100E100005D0327A02212046FFF7ECF8CFE72046D2
:100E20001121FFF7BEF82046FFF7B6F8C7E700BF6D
:100E3000E07100209D22070830B51E4B2DED028B7E
:100E40001C68B4FBF1F303F57F4383B0FF331B0C45
:100E5000B4FBF3F40023B4FBF1F5019200932246B6
:100E6000ABB20221F0EE408AB0EE608AFFF78FFF4E
:100E7000E0B107EE904AB5EE408AF1EE10FAF8EED6
:100E8000677A0ABF07EE105A68EE270AF8EE470A9B
:100E90009FED097AC0EE876A0123037127EE667A17
:100EA000C0ED046AA8EEA77A80ED037A03B0BDEC2A
:100EB000028B30BD0001002000007A440023064967
:100EC00010B51C46984200DC10BD51F833200AB121
:100ED000926814600133F5E7503D002013B50F4CC4
:100EE0008DF80700D4E90423A16853438B4212D044
:100EF0006368E0680DF10701184454F0D1F86368A5
:100F000022691344A268B3FBF2F102FB1133636060
:100F100063690133636102B010BD00BF283D00204A
:100F20000F4B1B78062B14D8DFE803F004131607C9
:100F30000A0D10004FF4C87070470A4B588870476C
:100F40004FF47A6070474FF4FA5070474FF47A507C
:100F500070474FF47A7070474FF4FA60704700BFE3
:100F6000043D0020903E00202DE9F04F2DED028B36
:100F7000A54FA64D3B78DFF8D0B299B0002403937B
:100F8000AA462646A946DAF800804046F8F700FF50
:100F9000584490F8982E022A6FD0032A76D0012A5E
:100FA00009D1DAF80C2022F0807222F0080242F017
:100FB0000402CAF80C205046FEF75AFB70B91422FE
:100FC00002FB0692D16801F00C02042A06D14046C9
:100FD000FEF762F80134E4B20444E4B201360A2EAA
:100FE0000AF1140ACFD18A4EA6F1C8084046FEF78E
:100FF0003FFBC0B9D8F80C104A0714D501F00C0318
:10100000042B10D0039B9C4247D221F0080141F0F1
:101010000401D8F80000C8F80C10FEF73DF80134C0
:10102000E4B20444E4B208F11408B045DED14FF054
:1010300000094C464E46C8462846FEF719FBA8B3A1
:10104000744A434601210420FCF7C0FC08F1010862
:10105000B8F10A0F05F11405EED13E780C2E40F3DD
:101060008F8001238BF8A63E6B4A0C2300933346F6
:1010700000210420FCF7AAFCA7E0DAF80C2022F0FB
:10108000807222F0040242F0080292E7DAF80C20A3
:1010900022F00C0242F080728BE721F00401D8F8B4
:1010A0000000C8F80C10FDF7F7FFBCE7E9684B0734
:1010B0000AD5039B9E4207D221F008012868E96007
:1010C000FDF7EAFF0136F6B2EA6810071AD528687C
:1010D00005A900239C420DDC0823EB6018AB03EB51
:1010E000890209F1010A082142F8245CD146FDF782
:1010F000D3FFABE751F804CFDCF800C0604501D066
:101100000133E7E751071AD528680EA900234B459C
:101110000DDB0423EB6018AB04F1010A03EB84043C
:10112000042144F8485CFDF7B7FF54468EE751F8B8
:1011300004CFDCF800C0604501D00133E7E7D301FC
:1011400084D5286805AA00239C4202DC0EAA00234D
:101150000EE052F8041F096888423FF477AF01336C
:10116000F2E752F8041F096888423FF46FAF013379
:101170004B45F6DB4FF08071E960FDF78DFF65E7C9
:10118000264B1979264B0329197035D90B1F022BD1
:1011900034D8FFF7C5FE234A234B9FED197B80B25D
:1011A000B3FBF0F3136000235360204B83ED007B0F
:1011B0001F4BCBF8A83E1F4B13F81130002B45D125
:1011C0001D4A02210420FCF701FC1FF0ADFF9BF833
:1011D000AC3E0446002B40F0BE80184A0221042099
:1011E000FCF7F4FB9BF8A60EB0FA80F0400919B0AA
:1011F000BDEC028BBDE8F08F114BDAE7114BD8E75D
:101200000000000000000000646E01209C0500202A
:1012100064060020D8220708F0220708903E00202C
:10122000043D0020103D002040420F00183D0020EA
:10123000C7F00008C47606081C230708982307088F
:1012400025F40008C5F00008E0710020A64217DC74
:10125000754F9FED768A0DF114080024A642B4DD87
:10126000734B58F8045F5B68C3F3007A714B1B78CB
:10127000062B6CD8DFE803F0621B220B2B2B2B0014
:1012800003238BF8A63E6C4A00943346F0E6FFF742
:1012900047FEDFED6A0A01465246B0EE600A284674
:1012A000FFF7CAFD47F83400002845D125E0FFF7D5
:1012B00037FEDFED630A01465246EEE7FFF730FEE8
:1012C000DFED600A9FED600A01465246E7E7052B15
:1012D0001DD05E4A5E49062B18BF0A46CDF804A011
:1012E0004FF0000A2846CDF800A014230221FFF792
:1012F0004EFD054668B947F8340005238BF8A63E35
:10130000544A234600210420FCF760FB5DE7524A63
:10131000E4E700F1140319460068039312224AF02F
:1013200097F9039B30B118464822514654F0DAFF32
:1013300001232B7147F8345001348FE7FFF7F0FD9C
:101340009FED3A0A01465246F0EE480AA7E700230D
:1013500047F83430D1E712280BDD02238BF8A63E84
:101360003E4A12230093002103460420FCF72EFB83
:1013700038E79BF8B63E012B0CD0022B0ED0384B31
:10138000CBF8BC3E9BF8B63E002B38D0022B09D0E0
:10139000344A23E74BF066FA334BF1E74BF062FA3D
:1013A000324BEDE74B46122BB8BF12239BB29C4247
:1013B00027DC4C45A8BF4C462D4FDFF8B880DFF83E
:1013C00070900EAE0025A542BFF60CAFD9F80420F0
:1013D000BBF8B03EB8FBF3F3C2F300720192BBF866
:1013E000AE2E00920321234A56F8040F9BB2FFF75A
:1013F000CEFC014670B147F8040B0135E3E74B46DC
:10140000D4E704208BF8A60E1B4ACDF800902346A3
:101410000021ABE705238BF8A63E184A2B46042093
:10142000FCF7D4FADEE600BF503D00206F12833A8D
:10143000686E0120043D00203A23070800000000E8
:101440006F120339ACC5A737ACC5A736001BB70070
:10145000C0C62D0073230708808D5B00B2230708E8
:10146000E1F00008DE230708B9E00208FDF00008FB
:101470009C61002040420F001A24070850240708EE
:10148000034AD2F8BC2E12B1112800D81047704779
:10149000E071002040B101380023FF2803F1010270
:1014A00003D840EA032080B2704740081346F4E7AF
:1014B00003681B68184703685B68184703689B68E4
:1014C000184703681B6A70B506460C46154683B17B
:1014D000BDE8704018473046FFF7F0FF0028FAD00B
:1014E00014F8011B3046FFF7E3FF2B1B002BF2DC47
:1014F00070BD0D44F9E7E4E70368DB68184703684B
:101500001B69184703685B6918470368DB6A03B106
:101510001847704703681B6B03B118477047164B99
:101520001B6813F0100F154B05D0B3F8C02E12F046
:10153000040F18BF002093F8DA2E72B1D3F8DC2E16
:10154000CAB1926838B1B3F8E01E0D4BB3FBF1F3AA
:101550005B101360704710607047D3F8E42E93F867
:10156000E83E0BB980F001002AB11368928808B1F7
:101570001A8370475A837047C06D0120E0710020C4
:1015800040420F00BFF34F8F0549064BCA6802F473
:10159000E0621343CB60BFF34F8F00BFFDE700BF96
:1015A00000ED00E00400FA0508B572B600224FF025
:1015B000FF31930003F1604303F561430132082AD0
:1015C000C3F88010C3F88011F3D1FFF7DBFF08B533
:1015D0000120F9F7F1FC012809D10021F9F7DCFC21
:1015E000034B1A6882F308885B689847FEE708BDDA
:1015F0000000FF1FEFF31183102282F312880949C4
:101600000A6801320A604FF0E02207499069C1F888
:10161000EC0E0020C1F8F00E1269DBB283F31188E2
:10162000704700BF1C2D0020E0710020074A084BC6
:101630005168D3F8F43E58434FF47A73B0FBF3F09B
:1016400053685B1A8342FBD9704700BF001000E06B
:10165000E071002010B504464FF4FA70FFF7E6FF82
:101660006069BDE81040FEF792BC90F910302DE99A
:10167000F0411646142253430D4A52F80380836802
:1016800013F0020504460F4602D140694BF05EFE9E
:10169000394640464DF05CFE314640464DF058FE1E
:1016A00015B92046FFF7D6FF0120BDE8F08100BF45
:1016B000B00000207FB50379012B0D460AD0022B24
:1016C00019D18368DB0758BF01F07F0104B0BDE882
:1016D0007040CAE781688DF80F2001F001010DF11B
:1016E0000F0200920191417C90F910002A46F9F70F
:1016F00007FC04B070BD0020FBE700682E22F42137
:10170000D8E7044B00681A8E9201343202F0FC02D2
:10171000F421CFE7E860002008B53122F421006809
:10172000FFF7C8FF012008BD006801225821C1E76A
:10173000006801224821BDE7006802220821B9E7BC
:10174000006801220821B5E710B5044600222121D6
:101750000068FFF7AFFF2068FC222021FFF7AAFFF7
:10176000206840222421FFF7A5FF20680C222321B6
:10177000FFF7A0FF206800222221FFF79BFF012036
:1017800010BD10B5012204460B210068FFF792FF3F
:1017900020B120681D220921FFF78CFF00F0010015
:1017A00010BD044B0246D3F8F80E08B1802181E742
:1017B000704700BFE071002010B5B020FFF7F1FFC7
:1017C0004020FFF7EEFF0020FFF7EBFF1020FFF7B0
:1017D000E8FF4FF48064013C0020A4B24BF043FCCE
:1017E000002CF8D110BD10B50446A1F15000C0B2D4
:1017F000FFF7D7FF04EB4400400004EB440400F083
:101800000E00FFF7CEFFC4F3C3001030BDE8104058
:10181000C7E708B55038C0B2FFF7C3FF0020FFF795
:10182000C0FFBDE808401020BBE738B500221F23E9
:1018300035210120FEF7DCFD3C4BC3F8F80E10B952
:101840000024204638BDAE20FFF7ABFF0446002839
:10185000F6D0D420FFF7A5FF8020FFF7A2FFA82035
:10186000FFF79FFF3F20FFF79CFFD320FFF799FF73
:101870000020FFF796FF4020FFF793FF8D20FFF732
:1018800090FF1420FFF78DFFA120FFF78AFFC820EB
:10189000FFF787FFDA20FFF784FF1220FFF781FFB1
:1018A0008120FFF77EFFCF20FFF77BFFD920FFF7D6
:1018B00078FFF120FFF775FFDB20FFF772FF402074
:1018C000FFF76FFFA420FFF76CFFA620FFF769FF6B
:1018D000AF20FFF766FFA620FFF763FFAE20FFF7FC
:1018E00060FF2020FFF75DFF0020FFF75AFFB020C8
:1018F000FFF757FF4020FFF754FF0020FFF751FF8D
:101900001020FFF74EFF4FF48065013D0020ADB27F
:101910004BF0A9FB002DF8D18120FFF742FFC82032
:10192000FFF73FFFAF20FFF73CFF8AE7E0710020A1
:1019300008B5FFF7BFFE014B187008BDF01000207E
:101940002DE9F0411E4690F91030154614225343FC
:101950000E4A52F8038083689A0704460F4602D461
:1019600040694BF0F3FC394640464DF0F1FC3346FC
:101970002A46002140464DF083FCA3689B0702D411
:101980002046FFF767FE0120BDE8F081B00000208F
:10199000F7B50779012F16460AD0022F15D18468B2
:1019A000E40758BF41F0800103B0BDE8F040C7E74D
:1019B000826802F00102CDE900620A46417C90F99A
:1019C0001000F9F79DFA03B0F0BD0020FBE707B562
:1019D00052BAADF80420022301AAFFF7D9FF024B47
:1019E000187003B05DF804FBF010002010B50A4C2D
:1019F000002384F8FC3E84F8FD1E84F8FE2E0323A9
:101A000004F6FC62FF21FFF7C3FF00280CBF6FF054
:101A10000C00002010BD00BFE071002010B50B4C81
:101A2000002384F8FC3E130A84F8FD1E84F8FE3E71
:101A300084F8FF2E042304F6FC62FF21FFF7A8FFC1
:101A400000280CBF6FF00C00002010BDE0710020DA
:101A5000024A0068002351219AE700BFDC81002080
:101A60002DE9F0411E4690F91030154614225343DB
:101A70000E4A52F8038083689A0704460F4602D440
:101A800040694BF063FC394640464DF061FC3346FB
:101A90000022294640464DF0F3FBA3689B0702D481
:101AA0002046FFF7D7FD0120BDE8F081B0000020FF
:101AB000F7B50779012F16460AD0022F15D1846891
:101AC000E40758BF41F0800103B0BDE8F040C7E72C
:101AD000826802F00102CDE900620A46417C90F979
:101AE0001000F9F733FA03B0F0BD0020FBE713B59F
:101AF000062304466A4600680221FFF7D9FFB8B101
:101B0000BDF9003007EE903ABDF90230F8EEE77A01
:101B1000C4ED077A07EE903ABDF90430F8EEE77AA3
:101B2000C4ED087A07EE903AF8EEE77AC4ED097A48
:101B300002B010BD13B5022304466A4600680321B3
:101B4000FFF7B6FF10B9002002B010BD9DF90130BB
:101B5000002BF8DA206807236A461221FFF7A8FF56
:101B60000028F0D09DF902209DF8013043EA0223BD
:101B700013EB430348BF03339B1007EE903A9DF9E4
:101B800004209DF8033043EA022313EB4303F8EEED
:101B9000E77A48BF03339B109DF90620C4ED047A11
:101BA00007EE903A9DF8053043EA022313EB430316
:101BB000F8EEE77A48BF03339B10C4ED057A07EED1
:101BC000903AF8EEE77AC4ED067ABDE738B50446F8
:101BD0000068FDF7BDFE0C230546021D194620686E
:101BE000FFF766FFA870B8B1B5F9043007EE903A78
:101BF000F8EEE77AC4ED077AB5F9063007EE903AC9
:101C0000F8EEE77AC4ED087AB5F9083007EE903AB5
:101C1000F8EEE77AC4ED097A38BD38B504460068B5
:101C2000FDF796FE0D230546C21C0C212068FFF728
:101C30003FFFA870B8B1B5F90A3007EE903AF8EE58
:101C4000E77AC4ED077AB5F90C3007EE903AF8EE72
:101C5000E77AC4ED087AB5F90E3007EE903AF8EE5F
:101C6000E77AC4ED097A38BD13B503230C46006842
:101C700001AA2221FFF71CFF30B1BDF9053003EBAB
:101C800083031B12E633238002B010BD13B5062375
:101C900004466A4600681F21FFF70AFFD0B1BDF86D
:101CA0000030DBBA07EE903ABDF80230F8EEE77A82
:101CB000DBBAC4ED047A07EE903ABDF80430F8EED2
:101CC000E77ADBBAC4ED057A07EE903AF8EEE77AE8
:101CD000C4ED067A02B010BD13B5062304466A4669
:101CE00000682521FFF7E4FED0B1BDF80030DBBA73
:101CF00007EE903ABDF80230F8EEE77ADBBAC4EDB1
:101D0000077A07EE903ABDF80430F8EEE77ADBBACE
:101D1000C4ED087A07EE903AF8EEE77AC4ED097A56
:101D200002B010BD13B502230C46006801AA1D21A4
:101D3000FFF7BEFE98B1BDF80430DFED0A6ADBBAEA
:101D400007EE903AB8EEE77AC7EE267A9FED067A6C
:101D500077EE877AFDEEE77A17EE903A238002B0AD
:101D600010BD00BFCFF7534100007A4370B506683D
:101D700005463046FDF7ECFD0E230446021D3B21CF
:101D80003046FFF795FEA070B8B1A389DBBA07EE25
:101D9000903AF8EEE77AC5ED077AE389DBBA07EE09
:101DA000903AF8EEE77AC5ED087A238ADBBA07EEB7
:101DB000903AF8EEE77AC5ED097A70BD07B50223CF
:101DC000006801AAF621FFF773FE20B1BDF80430C8
:101DD000024A5BBA138203B05DF804FBE86000209E
:101DE00007B50323006801AAF621FFF761FE80B161
:101DF0009DF805309DF8042007491B0243EA024381
:101E00009DF806201343B1F93020C2F10802D340F7
:101E10004B6303B05DF804FBE860002073B5062354
:101E2000F7210068154D164C6A46FFF741FE15492B
:101E3000E8B19DF801209DF800309DF80360120183
:101E400042EA03329DF8023042EA13129DF8043050
:101E50008A651B0143EA06339DF80560C5F8FC2F2F
:101E600043EA16138B6344F8F83C02B070BDD5F812
:101E7000FC3F8B6554F8F83C8B63F6E7E07100207B
:101E8000D8820020E860002007B50323006801AA7B
:101E90001946FFF70DFEA0B19DF804309DF805101E
:101EA0009DF904201B0443EA01239DF80610002A33
:101EB000ACBF00224FF07F420B431343024AC2F8EB
:101EC0000C3103B05DF804FBE860002007B5032384
:101ED000006801AA0021FFF7EBFDA0B19DF80430D6
:101EE0009DF805109DF904201B0443EA01239DF889
:101EF0000610002AACBF00224FF07F420B43134371
:101F0000024AC2F8083103B05DF804FBE860002023
:101F100013B5044600680379022B0CBF432103214B
:101F200006236A46FFF7C4FD18B9E086A06302B035
:101F300010BDBDF800305BBAE386BDF802305BBA75
:101F40006387BDF804305BBA2387F0E713B500233D
:101F5000C38683630446062300686A460321FFF7AD
:101F6000A7FD78B1BDF8003003EB4303E386BDF96C
:101F700002305B4203EB43032387BDF8043003EBDD
:101F80004303638702B010BD07B5012301AAFF21F7
:101F90000068FFF78DFD03B05DF804FBF7B505465B
:101FA0000068FDF7D5FC00230370042304460DEB05
:101FB00003022868FF21FFF77BFD10B9002003B062
:101FC000F0BD286804236A46FF21FFF771FD002851
:101FD000F4D09DF804309B09023B012BEED9BDF8EB
:101FE0000420BDF80630BDF80050BDF8021052BA0A
:101FF00043F6FF77C2F30D02BA42DFD0002ADDD0EC
:102000005BBAC3F34A1340F2FF76B342D6D0002B3B
:10201000D4D06DBAC5F30D05BD42CFD0002DCDD0C3
:1020200049BAC1F34A11B142C8D00029C6D0561BE3
:10203000002EB8BF7642FF2EC0DC5E1A002EB8BF5D
:102040007642FF2EBADC01262A440B44324133414A
:102050002670C4F80520C4F80130B0E737B505464E
:102060000068FDF775FC00230370042304460DEBA4
:1020700003022868FF21FFF71BFD40B19DF80430E3
:102080009B0907D00B4A04210320FBF79FFC00208B
:1020900003B030BDBDF80420BDF8063052BA5BBABB
:1020A00092B2C3F34A1301212170C4F80520C4F889
:1020B0000130EDE77524070807B5022301AAFFF7F1
:1020C000F7FC044B1870BDF8040040BA80B203B0AE
:1020D0005DF804FBF010002038B515460C4A0B0AD9
:1020E00082F8FC3E82F8FD1E022302F6FC62FF210C
:1020F0000446FFF74DFC30B101232A46FF2120465C
:10210000FFF7D6FC10B96FF00C0038BD0020FCE7DB
:10211000E07100202DE9F041104D05F6FC681646EF
:10212000002485F8FD1E02234246FF21074685F85C
:10213000FC4EFFF72DFC18B96FF00C00BDE8F081E4
:1021400002234246FF213846FFF7B2FC0028F3D0B5
:10215000B5F8FC3E5BBA33802046EFE7E071002023
:102160002DE9F341744D0468DFF8D8810023064659
:1021700085F8FE302D27B9B218F8012B204601371B
:10218000FFF734FC882FF6D1402287212046FFF745
:102190002DFC00238DF806309DF80630002B6FD003
:1021A000012286212046FFF721FC002287212046BC
:1021B000FFF71CFC092208212046FFF717FC00222C
:1021C0000B212046FFF712FC002851D137680DF192
:1021D00006025E213846FFF79DFFBDF80630B3F5D5
:1021E000D77F00F0A58059D8512B00F09F804DD8A3
:1021F0001D2B70D01E2B00F09980306821214AF0F1
:1022000004FE34680DF10602DE212046FFF782FF4E
:10221000BDF806309FED497A2822C3F309035343E2
:1022200007EE903AF8EEE77A454A67EE877A0021A2
:10223000FCEEE77A82F8FC1E17EE903A6C2182F8E9
:10224000FD1E190E82F8FE1E190C82F8FF1E190AD7
:1022500082F8001F82F8013FFF2102F6FC6206238C
:102260002046FFF795FB306840228721FFF7BEFB31
:10227000B0FA80F0400985F8FE0002B0BDE8F081B8
:102280000DF1060120464AF051FE85E7AD2B4FD0F7
:10229000D62B01D0602BB0D121241DE040F2E132D9
:1022A000934247D00CD840F2D922934242D040F218
:1022B000E122934202D0B3F5E67F9ED164240BE085
:1022C00040F28F42934203D040F29152934294D114
:1022D0004FF4FA7400E00F2400288ED10A224B211B
:1022E0003846FFF783FB0F2260213846FFF77EFB5D
:1022F0000D2263213846FFF779FBB8226921384661
:10230000FFF774FB40F60D7278213846FFF786FB25
:1023100040F60E627A213846FFF780FB00287FF4F2
:102320006CAF214638464AF070FD66E71424D3E7C7
:102330003224D1E7C824CFE7E86000209A99893F8A
:10234000E0710020487A060837B5134D95F8FE3045
:102350000446FBB100680DF105014AF0E7FD9DF868
:1023600005307BB10DF1060220689621FFF7D2FE01
:102370000A22BDF80630B3FBF2F3084A936001234A
:1023800085F8FF3020680122862103B0BDE8304087
:10239000FFF72CBB03B030BDE8600020F010002038
:1023A00013B5022301AA044651210068FFF780FB00
:1023B000114AE8B1BDF804305BBA9BB2D360D36870
:1023C000B3F5C87F02DD4FF0FF33D3600B4B0C4AEF
:1023D000196852F8F43C32338B4207D242F8F41CAD
:1023E0002068084A00235121FFF7D2FA02B010BD3D
:1023F0006FF00103E9E700BFF01000201C2D002062
:10240000D8820020DC81002007B50223006801AAE1
:102410000021FFF74DFB0F4B83F80401B0B1BDF86D
:1024200004300D4A5BBA9BB2B3F5FA6F3FBF0A2185
:10243000B3FBF1F307EE903AF8EEE77A2BBF4FF0DB
:10244000FF33FDEEE77A1361C2ED047A03B05DF865
:1024500004FB00BFE8600020F0100020F8B5254C18
:1024600005460323006804F118020021FFF720FB52
:1024700000283CD0A77E04F1170603210023013970
:1024800009D19F42286817D06FF002036361BDE84D
:10249000F8404AF0B6BC16F8012F082053405AB253
:1024A000002ABBBF520082F007025B00D3B2A8BF74
:1024B000DBB20138F3D1E2E7238B5BBA9BB25A1E41
:1024C00092B24FF6FD718A4202D94FF0FF33DDE739
:1024D00007EE903AF8EEE77AF2EE046A87EEA67A13
:1024E000FDEEC77A17EE903A28686361CFE76FF088
:1024F0000103F9E7F010002013B502230C46006831
:1025000001AA0021FFF7D4FA60B15CB19DF8053053
:102510009DF90420DB0903EB830302EB820203EB4A
:102520004203238002B010BDF8B590F91030154673
:10253000142253430D4AD75883689A0704460E461F
:1025400002D440694AF002FF314638464CF000FFA1
:1025500001230022294638464CF092FEA3689B07CF
:1025600002D42046FFF776F80120F8BDB000002025
:1025700073B50379012B16460AD0022B15D1836857
:10258000DB0758BF41F0800102B0BDE87040CBE7E7
:10259000826802F00102CDE900620A46417C90F9AE
:1025A0001000F8F7D3FC02B070BD0020FBE713B5B4
:1025B00004466A4600680821FFF7DAFF9DF80030FC
:1025C000DB0602D4002002B010BD206806236A4654
:1025D0000021FFF76DFA0028F4D09DF801309DF836
:1025E00000209DF80410DFED496A1B0203EB024353
:1025F0009DF802201C021A449DF8033048BF02F1E6
:102600007F42090201EB034107EE902A9DF8053055
:10261000F8EEE77A0B44090248BF03F17F4387EEE7
:10262000A67A07EE903AF8EEE77A394BC7EEA63A6B
:10263000B3F96A20B3F97410D3ED196AD3ED187A9F
:10264000B8EEE66A06EE902AB3F96C2003EE101A93
:10265000B3F9681005EE902AB3F96E2004EE901AD3
:102660002C4905EE102AB3F9702011F8F01C04EE85
:10267000102AF8EEE44A1129F8EEE77AF8EEE66A55
:10268000F8EEE55AB8EEC55AB8EEC44AB3F972206E
:1026900064EEA34A67EE232A2CD1B8EEC33AA7EE24
:1026A000034AE4EE075AA5EE876AE6EE077A06EEDD
:1026B000102AB8EEC66A77EEA47AA7EE065AE5EEBF
:1026C000076AB3F95C20E6EEA27A07EE102AB3F9A6
:1026D0005E20C3ED1E7A07EE902AF8EEE77AB8EE98
:1026E000C77A67EEA37AF6EE006AE7EE267AC3EDC4
:1026F0001F7A68E7E7EE045AE7EE056AA5EE876AF7
:10270000E6EE077A77EEA47ADBE700BF00007848B0
:10271000E8600020D88200202DE9F34116460DF133
:1027200007021D4607468846FFF722FF9DF807402F
:1027300006EA0403AB4209D024EA06022A434146D2
:10274000384602B0BDE8F041FEF7B4BF02B0BDE8C4
:10275000F0811FB50446002300688DF807300DF1A5
:1027600007022721FFF704FF60B19DF807301B0720
:1027700008D52068062302AA2821FFF799F920B975
:10278000E086A063002004B010BDBDF90830002B26
:10279000B8BF03339B10E386BDF90A30002BB8BFE6
:1027A00003339B102387BDF90C30002BB8BF0333D4
:1027B0009B106387E7E71FB500210446C18681634C
:1027C0000DF107020068FFF7D3FE10B9002004B036
:1027D00010BD9DF807301B07F8D52068062302AA14
:1027E0000121FFF765F90028F0D0BDF808305BBA89
:1027F000E386BDF80A305BBA2387BDF80C305BBABC
:102800005B426387E3E730B5002585B00446C586A3
:1028100085630DF1070200680621FFF7A9FE10B9D4
:10282000002005B030BD9DF80730DB07F8D52068E3
:10283000062302AA2946FFF73BF90028F0D0BDF88D
:102840000830E386BDF80A302387BDF80C30638773
:10285000E7E707B50DF10702FFF78AFE034B187093
:102860009DF8070003B05DF804FB00BFF0100020E6
:10287000F8B5144E144F41F0010200210446FFF751
:1028800057F8356847F8EC5C13212046FFF7E1FF65
:1028900010F007000BD001220B212046FFF748F86B
:1028A000002220461146FFF743F8012008E057F8C0
:1028B000E82C002AE8D033689BB25B1B9A42E3D233
:1028C000F8BD00BF1C2D0020D882002010B50C469A
:1028D0000121FFF7BEFFC0F300132370C0F3C00354
:1028E000A370C0F380036370C0F38013C0F3C01003
:1028F000E370207110BD2DE9F8430F4650211446B6
:102900000546FFF7A6FF01304000C0B220804621F7
:102910002846FFF79EFF2C4E2378013080B2734388
:102920004FF47A78A08003F5FA734FF4FA69B3FB99
:10293000F8F25121B3FBF9F300FB02332846B3FB55
:10294000F8F3E360FFF7B8FBC2B2C0F30F202378BF
:102950008240013292B27343E28003F5FA73284653
:10296000B3FBF8F1B3FBF9F302FB01337021B3FBC6
:10297000F8F32382FFF76DFF01304000C0B26080A2
:1029800071212846FFF798FBC3B2C0F30F208340A4
:102990000133FA789BB2238112B1E2889B1A23811A
:1029A000A3782089734303F5FA734FF47A724FF4D6
:1029B000FA65B3FBF2F1B3FBF5F300FB0133B3FBB4
:1029C000F2F36382BDE8F883002F3A002DE9F04767
:1029D000DB4FDFF87483DFF874934FF4FA738AB037
:1029E000044600268921006847F8E83C88F8FC6026
:1029F000FFF72FFF40F00102D2B220688921FEF7D5
:102A000097FF324620688821FEF792FF2068012256
:102A10008021FEF78DFF20680122FF21FEF788FF4D
:102A2000324631462068FEF783FF91212068FFF788
:102A300010FF314607F8E40C01222068FEF778FF0A
:102A400032462068FF21FEF773FF3246206880215E
:102A5000FEF76EFF60212068FFF7FBFE40F01202D8
:102A6000D2B220686021FEF763FF20682022442153
:102A7000FEF7ADFF2068FF220121FEF759FF256810
:102A8000012280212846FEF753FF0122FF2128461C
:102A9000FEF74EFF324631462846FEF749FF062232
:102AA000FF212846FEF744FF83212846FFF7D1FE89
:102AB00040F00402D2B283212846FEF739FF0722F4
:102AC000FF212846FEF734FF012281212846FEF728
:102AD0002FFF012280212846FEF72AFF6B22942136
:102AE0002846FEF725FF324683212846FEF720FFC1
:102AF000D9F8006047F8EC6C83212846FFF7A9FE5F
:102B0000002800F04683012228468321FEF710FFAB
:102B100092212846FFF79DFE0022C0F3C71681468A
:102B200081212846FEF704FF06222846FF21FEF7F2
:102B3000FFFE83212846FFF78CFE832100F0FB0275
:102B40002846FEF7F5FE28460122FF21FEF7F0FE9B
:102B5000284601220021FEF7EBFE28460022FF2135
:102B6000FEF7E6FE284600228021FEF7E1FE06235E
:102B700003AAB0212068FEF79BFF20680122FF21F5
:102B8000FEF7D6FE206800224F21FEF7D1FE206816
:102B90002C224E21FEF7CCFE20680022FF21FEF7FA
:102BA000C7FE2068B422B621FEF7C2FE0025002E23
:102BB00018BF0C2609F07F092A460120C5F3C40C72
:102BC0000CF128035FFA85FE0DEB030C76451CF82B
:102BD0001C3C05F0070102D8914540F0E58200FA5F
:102BE00001F123EA01030CF81C3C0135302DE5D13D
:102BF000062303AAB0212068FEF7CAFE514B01222A
:102C00001870FF212068FEF793FE0022114620680D
:102C1000FEF78EFE20680022FF21FEF789FE206865
:102C200000220921FEF784FE206800221021FEF711
:102C30007FFE206800221121FEF77AFE2068012223
:102C40002421FEF775FE2068FF222521FEF770FE85
:102C5000206800227521FEF76BFE20680122FF210B
:102C6000FEF766FE20682C224E21FEF761FE2068EA
:102C700000224821FEF75CFE294620682022FEF74C
:102C800057FE20680022FF21FEF752FE29462068E9
:102C90000922FEF74DFE206800225421FEF748FE6F
:102CA000206804223121FEF743FE206803223221EE
:102CB000FEF73EFE206883224021FEF739FE2068A1
:102CC00025224621FEF734FE206800226021FEF70F
:102CD0002FFE206800222721FEF72AFE2068062208
:102CE0005021FEF725FE206800225121FEF720FE2C
:102CF000206896225221FEF71BFE206808225621EA
:102D0000FEF716FE2A4620685721FEF711FE2068BE
:102D100000226121FEF70CFE206800226221FEF7EE
:102D200007FE206800226421FEF702FE20680022D0
:102D30006521FEF7FDFD2068A022662108E000BFA6
:102D4000D8820020F0100020E86000201C2D002018
:102D5000FEF7EEFD20680122FF21FEF7E9FD206865
:102D600032222221FEF7E4FD206814224721FEF7DB
:102D7000DFFD2068FF224921FEF7DAFD20680022EE
:102D80004A21FEF7D5FD20680022FF21FEF7D0FD85
:102D900020680A227A21FEF7CBFD206800227B21E1
:102DA000FEF7C6FD206821227821FEF7C1FD2068CC
:102DB0000122FF21FEF7BCFD206834222321FEF70B
:102DC000B7FD206800224221FEF7B2FD2068FF22F5
:102DD0004421FEF7ADFD206826224521FEF7A8FD1F
:102DE000206805224621FEF7A3FD402211462068F7
:102DF000FEF79EFD206806220E21FEF799FD206851
:102E00001A222021FEF794FD206840224321FEF77C
:102E10008FFD20680022FF21FEF78AFD2068032233
:102E20003421FEF785FD206844223521FEF780FD20
:102E300020680122FF21FEF77BFD2068042231215A
:102E4000FEF776FD206809224B21FEF771FD206810
:102E500005224C21FEF76CFD206804224D21FEF76F
:102E600067FD20680022FF21FEF762FD2068002236
:102E70004421FEF75DFD206820224521FEF758FD24
:102E8000206808224721FEF753FD206828224821A8
:102E9000FEF74EFD206800226721FEF749FD2068FD
:102EA00004227021FEF744FD206801227121FEF703
:102EB0003FFD2068FE227221FEF73AFD20680022C5
:102EC0007621FEF735FD206800227721FEF730FDE0
:102ED00020680122FF21FEF72BFD206801220D2131
:102EE000FEF726FD20680022FF21FEF721FD206865
:102EF00001228021FEF71CFD2068F8220121FEF747
:102F000017FD20680122FF21FEF712FD2068012233
:102F10008E21FEF70DFD206801220021FEF708FD3D
:102F200020680022FF21FEF703FD20680022802197
:102F3000FEF7FEFC042220680A21FEF7F9FC256852
:102F400084212846FFF785FC842100F0EF02284603
:102F5000FEF7EEFC012220680B21FEF7E9FC256854
:102F600001A92846FFF7B2FC05AA01A92846FFF7E8
:102F7000C2FC9DF80430002B00F01C81089D05F672
:102F800084559DF80630002B00F01781089B03F252
:102F9000B22305EB43059DF8073023B1BDF824307B
:102FA00003F525731D449DF8083023B1BDF8263084
:102FB00003F226231D44E822206847F8E05C012143
:102FC000FEF7B6FC2068294649F0CCFF01222068B4
:102FD0001146FEF7ADFC20684021FFF749FC0028B0
:102FE00000F0DF80206801210222FEF7A1FC2068AA
:102FF0000021FFF73DFC002800F0D3802068DFF8B7
:10300000D491E8220121FEF793FC2068202244217C
:10301000FEF7DDFC256801A92846FFF757FC05AA45
:1030200001A92846FFF767FC502257212846FEF7E2
:103030007FFC082256212846FEF77AFC0822502100
:103040002846FEF775FCBDF824004FF47A7A48F262
:103050000E660AFB0060B0FBF9F080B2FEF71AFAC8
:10306000512102462846FEF7B2FC089B0AFB036684
:10307000574B9E429DBFB6FBF9F202F1FF32D2B22E
:10308000FF2246212846FEF753FC57F8E01C28464D
:1030900049F068FF01212846FFF7DBFB02220646C4
:1030A00001212846FEF744FC00212846FFF7E0FBFB
:1030B000324601212846FEF73BFC246801A9204640
:1030C000FFF704FC05AA01A92046FFF714FC4822DB
:1030D00011462046FEF72CFC082247212046FEF729
:1030E00027FC032232212046FEF722FC0722302152
:1030F0002046FEF71DFC0122FF212046FEF718FCAA
:10310000202230212046FEF713FC0022FF2120461A
:10311000FEF70EFC062220467021FEF709FCBDF8E2
:1031200026304FF47A7246F6440002FB03004DF25B
:103130008803B0FBF3F09DF8073080B21BB1BDF8F7
:103140001A30184480B2FEF7A5F9712102462046D4
:10315000FEF73DFC57F8E01C204649F003FF012133
:103160002046FFF776FB0222054601212046FEF7A6
:10317000DFFB00212046FFF77BFB2A46012120468A
:10318000FEF7D6FB642347F8E83C012388F8FC30BF
:1031900007E0D9F800309BB29B1BB3F5FA7F7FF6AE
:1031A000ABAC0AB0BDE8F0870B41DB0744BF01328E
:1031B000D2B21AE540F63635E3E69DF80530002B2D
:1031C0003FF4E9AE089B03F525731D44E3E600BF19
:1031D0001B280D011C0C0100F8B53B4F97F8FC3083
:1031E0000446002B37D0394D15F8DC6C012E33D056
:1031F000022E4FD07EBB006801228021FEF798FB93
:1032000020680122FF21FEF793FB206832463146F9
:10321000FEF78EFB15F8E42C20689121FEF788FB61
:10322000206801223146FEF783FB20683246FF21E9
:10323000FEF77EFB206832468021FEF779FB20688E
:1032400001223146FEF774FB214B1B6845F8EC3C2C
:10325000012305F8DC3CF8BD00680021FFF7F9FA0E
:10326000C20711D555F8E82C002AF4D0184B55F8B0
:10327000EC1C1B689BB25B1A9A42ECD2154B4FF0C8
:10328000FF325A600023E4E7114B1B6845F8EC3C21
:103290000223DEE700681321FFF7DBFA4307E1D0E2
:1032A0001E212068FEF708FF012206460B21206838
:1032B000FEF73EFB0A23B6FBF3F6064BB6B25E60A2
:1032C000012387F8FD30DDE7E8600020D882002088
:1032D0001C2D0020F010002010B5EFF311811023F9
:1032E00083F312884FF0E023C9B29C691A6912F483
:1032F000803F0D4A1EBF0120C2F8F00E9C690B4BA7
:103300001868D2F8F03E81F31188D2F8F41E4FF419
:103310007A72034402FB01F0001BB0FBF1F00021C4
:10332000E3FB020110BD00BFE07100201C2D002056
:10333000124B5B68C3F3080330B4EBB9EFF31183AE
:10334000D3B90F490F4B4FF0E0250A68AC69086804
:103350008242FAD1D3F8EC0E8442F6D8D3F8F41EA8
:103360004FF47A7303FB01F0001BB0FBF1F0002176
:10337000E2FB030130BC704730BCADE700ED00E07C
:103380001C2D0020E071002010B5074C14F8D70C5C
:1033900040B1FFF7CDFF54F8D03CC01AC0F5FA5049
:1033A00020EAE07010BD00BFD882002010B50446AE
:1033B00030B1036823B1DB6813B1BDE81040184792
:1033C000FFF7B6FFD4E904239042994134BF0120AE
:1033D000002010BDF8B506460D46FFF7A9FF0446CC
:1033E0000F46FFF7A5FF021B61EB0703B242AB419B
:1033F000F7D3F8BD38B50D460446FFF7C5FF011EEB
:1034000002DDC917FFF7E6FF064B2068002203F82C
:10341000D72C492113F8D63C2A46FEF749FB012058
:1034200038BD00BFD88200202DE9F341384C54F854
:10343000C83CC0F8363034F8C43C438714F8D83C54
:10344000012B064600F13608A4F1C8070CD0022B68
:1034500026D0A3BB0122022148F09FFA012304F8E1
:10346000D83C14F8C25C10E0FFF78EFF14F8C25C81
:1034700058B969463046FFF7BDFF9DF8003008B1E6
:103480009B0706D1002304F8D83C284602B0BDE8CB
:10349000F08107220321304648F07FFA0223F2E749
:1034A000FFF772FF0028DCD169463046FFF7A2FF24
:1034B0009DF80630054610B113F0080205D000252E
:1034C00004F8D85C04F8C25CDFE734F9C01C684635
:1034D000FBF7F8FC404234F9BE1CF0860DF1020007
:1034E000FBF7F0FC34F9BC1C308701A8FBF7EAFCC1
:1034F000D6F8363044F8C83C40427087B8F80430FB
:10350000BB80012304F8D82C04F8C23CBDE700BFFF
:10351000D882002010B50446013C00D210BD4FF403
:103520007A700021FFF756FFF6E738B505680446C4
:1035300000212846FCF7CAF9B62214212846FEF7D6
:10354000B9F86420FFF7E6FF812210212068FEF71A
:10355000B1F80120FFF7DEFF152120688022FEF779
:10356000A9F80120FFF7D6FF20680321BDE8384005
:10357000FCF7ACB938B50568044600212846FCF7CD
:10358000A5F9B6227E212846FEF794F86420FFF7BD
:10359000C1FF00227C212068FEF78CF86420FFF731
:1035A000B9FF04227D212068FEF784F86420FFF72C
:1035B000B1FF8C2240212068FEF77CF80120FFF744
:1035C000A9FF022241212068FEF774F80120FFF7CD
:1035D000A1FF20680221FCF779F94FF40063A38171
:1035E00038BD10B504464069FCF7D6FC0120FFF752
:1035F00091FF6069FCF7CBFCBDE810400A2089E729
:1036000073B50468B6227E2105462046FEF752F8BF
:103610006420FFF77FFF02212046FCF757F9204680
:10362000FFF7DFFF00227C212046FEF743F8012050
:10363000FFF770FF002259212046FEF73BF80120DA
:10364000FFF768FF5E238DF8073094F910301422DD
:1036500053433D4AD658A3689A0702D4606949F09B
:1036600075FE01230DF10702002130464BF008FEE4
:103670004FF4A473354A002130464BF001FEA36895
:103680009B0702D42046FDF7E5FF0A20FFF742FF23
:10369000012259212046FEF70DF80120FFF73AFFDD
:1036A0008C2240212046FEF705F80120FFF732FF6B
:1036B000032241212046FDF7FDFF0120FFF72AFFED
:1036C000234EA96B234A95F83500B6FBF1F103238D
:1036D00089B2FBF785FD4388B6FBF3F62E640279C9
:1036E000422142F0C0022046FDF7E4FF0120FFF72F
:1036F00011FF082243212046FDF7DCFF0120FFF7E0
:1037000009FF042258212046FDF7D4FF0120FFF7CE
:1037100001FF0A2253212046FDF7CCFF0120FFF7CD
:10372000F9FE00227C212046FDF7C4FF0120FFF7AF
:10373000F1FE06227D212046FDF7BCFF012002B0EC
:10374000BDE87040E6E600BFB0000020A37A06089E
:1037500040420F00EC7B0608F8B5816B0468294AEB
:10376000294FB7FBF1F10546062389B290F83500E1
:10377000FBF736FD00214388B7FBF3F706462F64BD
:103780002046FCF7A3F880226B212046FDF792FF2C
:103790006420FFF7BFFE032268212046FDF78AFF61
:1037A0006420FFF7B7FE01226B212046FDF782FF60
:1037B0000F20FFF7AFFE18221B212046FDF77AFFEE
:1037C0000F20FFF7A7FE18221C212046FDF772FFED
:1037D0000F20FFF79FFE32791A212046FDF76AFF7E
:1037E0000F20FFF797FE727919212046FDF762FF3F
:1037F0006420FFF78FFE20460321BDE8F840FCF768
:1038000065B800BFFE7B060840420F00F7B50523F0
:103810000468816B654A664FB7FBF1F1054689B2D2
:1038200090F83500FBF7DCFC00214388B7FBF3F789
:1038300006462F642046FCF749F8002276212046F0
:10384000FDF738FF0F224E212046FDF733FF0F20F2
:10385000FFF760FE72794F2102F00F022046FDF75C
:1038600029FF0F20FFF756FE7279502102F00F0258
:103870002046FDF71FFF0F20FFF74CFE5221FF22CD
:103880002046FDF717FF0F20FFF744FE95F835108F
:10389000072941D0474E96F80501FBF7EDFC054698
:1038A000012276212046FDF705FFAA780C2120464B
:1038B000FDF700FF2A790D212046FDF7FBFEAA79CE
:1038C000AB88120142EA1322D2B20E212046FDF744
:1038D000F1FE4FF4807196F80501FBF7CDFC05462B
:1038E000022276212046FDF7E5FEAA78520002F07A
:1038F000FE0203212046FDF7DDFE2A790421204641
:10390000FDF7D8FEAA79AB88120142EA1322D2B29F
:1039100005212046FDF7CEFE002276212046FDF748
:10392000C9FE032214212046FDF7C4FE0F20FFF735
:10393000F1FD002263212046FDF7BCFE6420FFF765
:10394000E9FD082265212046FDF7B4FE0DF10702CE
:1039500064212046FEF70CFE9DF8072022F010029D
:1039600042F06002642120468DF80720FDF7A2FE98
:103970000F20FFF7CFFD0DF106024D212046FEF787
:10398000F7FD9DF8062002F03F0242F040024D2173
:1039900020468DF80620FDF78DFE0F20FFF7BAFDBB
:1039A00003212046FBF792FF03B0F0BD227C0608FE
:1039B00040420F00E8600020F8B5816B04682D4A92
:1039C0002D4FB7FBF1F10546062389B290F835007B
:1039D000FBF706FC00214388B7FBF3F706462F648C
:1039E0002046FBF773FF80226B212046FDF762FE25
:1039F0006420FFF78FFD072268212046FDF75AFE5D
:103A00006420FFF787FD00226B212046FDF752FE60
:103A10006420FFF77FFD01226B212046FDF74AFE5F
:103A20000F20FFF777FD18221B212046FDF742FEED
:103A30000F20FFF76FFD18221C212046FDF73AFEEC
:103A40000F20FFF767FD32791A212046FDF732FE7D
:103A50000F20FFF75FFD727919212046FDF72AFE3E
:103A60006420FFF757FD20460321BDE8F840FBF72F
:103A70002DBF00BFFE7B060840420F009CE710B53B
:103A80007822044600210068FDF714FE0520FFF7A8
:103A900041FD202201212068FDF70CFE0520FFF7E3
:103AA00039FD002202212068FDF704FE6420FFF7A3
:103AB00031FD012010BD10B5072204460A2100681F
:103AC000FDF7F8FD0520FFF725FD242241212068A0
:103AD000FDF7F0FD0520FFF71DFDC0224221206803
:103AE000FDF7E8FD0520FFF715FD012010BD10B51D
:103AF0000122044610210068FDF7DCFD48B11420C6
:103B0000FFF708FD2068A022BDE810401121FDF755
:103B1000D1BD10BD13B5044600210068FBF7D6FEE9
:103B20000021204647F020FF1420FFF7F3FC0F216F
:103B3000204647F019FF0A20FFF7ECFC01AA0323F7
:103B40001021204647F03EF80A20FFF7E3FC9DF8DD
:103B50000420174B803223F8C02C9DF805208032BA
:103B600023F8BE2C9DF8062000218032204623F841
:103B7000BC2C47F0F9FE0A20FFF7CCFC0DF1030244
:103B800001230221204647F01DF801230DF1030215
:103B90000921204647F016F82046122147F0E4FE9E
:103BA00020680321FBF792FE012002B010BD00BF88
:103BB000D882002008B5006801220921FDF77AFDAE
:103BC000BDE808406420A5E480B506460A25012129
:103BD0000846FCF79DFD00210846FCF799FD771C7F
:103BE0004FF03208052457EA04030BD14FF47A70E2
:103BF000FFF790FC013DEAD101210846F7F7CCF927
:103C0000FDF7D2FC0120FCF771FD0020FCF76EFDF2
:103C10000120FDF784FC4046FFF77CFC0120FCF707
:103C200065FD0020FCF762FDFDF779FC4046FFF7DB
:103C300071FC44B1013CD6D14FF4FA70FFF76AFC35
:103C40004FF0FA08CFE7013FCDE737B505680446E6
:103C500000212846FBF73AFE15227E212846FDF773
:103C600029FD6420FFF756FC11227E212068FDF714
:103C700021FD0520FFF74EFC20680DF1070203210E
:103C8000FEF776FC9DF8073003F03C03142B02D0BE
:103C90000620FFF799FF0C2240212068244DFDF7F4
:103CA00009FD0120FFF736FCA16B224A94F835008C
:103CB000B5FBF1F1092389B2FBF792FA4388B5FB12
:103CC000F3F52564027920684221FDF7F3FC012019
:103CD000FFF720FC082241212068FDF7EBFC0120C2
:103CE000FFF718FC002243212068FDF7E3FC0120C8
:103CF000FFF710FC102251212068FDF7DBFC0120AA
:103D0000FFF708FC0A2253212068FDF7D3FC0120AD
:103D1000FFF700FC802256212068FDF7CBFC012034
:103D2000FFF7F8FB20680321FBF7D0FD03B030BD9F
:103D300040420F00407C0608F0B5816B0568514A8F
:103D4000514FB7FBF1F185B00446062389B290F8D4
:103D50003500FBF745FA00214388B7FBF3F7064629
:103D600027642846FBF7B2FD80226B212846FDF729
:103D7000A1FC9620FFF7CEFB032268212846FDF721
:103D800099FC9620FFF7C6FB03226B212846FDF71E
:103D900091FC0F200021FFF71DFB10226A2128460D
:103DA000FDF788FC0F200021FFF714FB00226C2197
:103DB0002846FDF77FFC0F200021FFF70BFB7279EF
:103DC00019212846FDF776FC0F200021FFF702FBA2
:103DD00018221B212846FDF76DFC0F200021FFF75C
:103DE000F9FA18221C212846FDF764FC0F20002157
:103DF000FFF7F0FA32791A212846FDF75BFC012023
:103E00000021FFF7E7FA03212846FBF75FFD206852
:103E1000062302AA4321FDF74BFED0B1BDF80830BE
:103E2000DBBA07EE903ABDF80A30F8EEE77ADBBA73
:103E3000C4ED077A07EE903ABDF80C30F8EEE77A59
:103E4000DBBAC4ED087A07EE903AF8EEE77AC4EDF3
:103E5000097AD4ED087AFDEEE77ACDED017A9DF985
:103E6000043001330CD1D4ED077AFDEEE77ACDEDC5
:103E7000017A9DF90430013302D10620FFF7A4FE38
:103E800005B0F0BDFE7B060840420F0018B1036884
:103E90005B6803B11847FF20704718B103689B683F
:103EA00003B118470020704770B450B106798E42B4
:103EB00007D34579954204D30368DB680BB170BC26
:103EC000184770BC704710B440B184798C4205D358
:103ED00003681B6913B15DF8044B18475DF8044B88
:103EE000704718B103685B6903B11847704718B190
:103EF00003681B6A03B118470020704730B50A46B3
:103F000058B1041D00F1140320686168154603C50B
:103F100008349C422A46F7D1012030BD10B50C462A
:103F200070B92D2300202375094B2061C4E90000DE
:103F3000C4E90200C4E90633302384F8203010BD00
:103F40000368DB6A002BECD098470028E9D0F6E73D
:103F5000906D070838B5054D441E14F8011F01B9CE
:103F600038BD55F8B80CFBF773FCF6E7D882002093
:103F700070B50E4C0E4605460D48FFF7EBFF334675
:103F80000C4954F8B80C2A464BF0FAF954F8B80C1E
:103F9000FBF752FC14F8B43C3BB1012304F8B33CEA
:103FA00014F8B23C013304F8B23C70BDD882002052
:103FB0009824070871F8000808B50648FFF7CAFFFB
:103FC000054B33F8B00C18B1BDE80840FFF7A2BAB2
:103FD00008BD00BF817C0708D882002010B5074CBF
:103FE00002460B4654F8B80C05494BF0C9F954F891
:103FF000B80CFBF721FCBDE81040DDE7D8820020BB
:1040000071F8000808B5FFF7A5FFBDE80840D3E741
:1040100010B504460948FFF79DFF2046FFF79AFFB9
:10402000074B13F8B42C3AB1012203F8B32C13F860
:10403000B22C013203F8B22C10BD00BF982407083F
:10404000D882002010B504460348FFF783FF2046BE
:10405000BDE81040D6E700BFA42407080CB48306CF
:1040600007B500D551B9049805A90191FFF7B6FF2E
:10407000012003B05DF804EB02B070470020F8E7C0
:10408000024B014653F8B80CFBF7E2BBD882002084
:104090000CB407B510F0400009D069B92320FFF730
:1040A000EFFF049805A90191FFF798FF012003B0E5
:1040B0005DF804EB02B070470020F8E70FB413B5C9
:1040C000094C0A4954F8B80C04AB53F8042B01937B
:1040D0004BF056F954F8B80CFBF7AEFB02B0BDE854
:1040E000104004B0704700BFD882002071F800086B
:1040F0000FB407B504A951F8040B0191FFF76EFF47
:1041000003B05DF804EB04B070470FB407B504A921
:1041100051F8040B0191FFF72BFFFFF74DFF03B0A0
:104120005DF804EB04B0704770B5C379164603F030
:1041300007028CB00446062A4FD8DFE802F00414C8
:1041400017191C1E49000D7813F0C00347D0402BEF
:104150003CD12946204614F0C9F8002859D00CB0AB
:10416000BDE87040AAE791F90050EDE70D88EBE754
:10417000B1F90050E8E70D68E6E791ED000A6846FE
:10418000FAF7EEF801462848FFF798FFF6B1E37911
:104190003F2B1BD8204614F001F800EE100A6846A9
:1041A000B8EEC00AFAF7DCF801462048FFF786FFB0
:1041B000204614F003F800EE100A6846B8EE400AF4
:1041C000FAF7CEF801461948FFF778FF0CB070BD3A
:1041D00015480CB0BDE8704070E70025B4E7042A2C
:1041E0000CBF134813482946FFF768FF002EEDD097
:1041F000E3793F2BEAD8204613F0D0FF054620464E
:1042000013F0DCFF02460C4829460CB0BDE87040B4
:1042100054E76946204613F08FFE08486A4629464F
:10422000FFF773FFD2E700BF7E2D07087D2D07083B
:10423000F52407080E5907086A7F0708A92407080C
:104240002DE9F04F8FB001F020034C4C00938146D4
:104250000F464FF000084A4B53F8B80CFBF7ECFA46
:1042600094F807B00BF038034B4549D1204613F0C2
:104270001FFFFAF7C5FA8568204613F045FF82460E
:104280002E18204613F07EFF0BF007020146062A87
:104290006CD8DFE802F0044045494E525E0015F844
:1042A0000A200978511A4A424A41009B03B13ABB9D
:1042B00002A92046019213F03FFE7B0615D5019A14
:1042C0009AB9304802A9FFF7F9FE2F4902A84BF02E
:1042D0000FFA00284CD115F80A30202B48D12B4872
:1042E0003146FFF7EBFEFFF767FE294802A9FFF70B
:1042F000E5FE002231462046FFF716FFFFF75CFE81
:1043000008F1010840F29223984504F10C04A2D16F
:104310000FB0BDE8F08F15F90A2091F90010C1E740
:1043200035F80A200988BDE735F90A20B1F90010EF
:10433000B8E755F80A200968B4E796ED007AD1EDA0
:10434000007AB4EE677AF1EE10FA0CBF0122002277
:10435000ABE72046019113F031FF0199421C304632
:1043600050F01AFEB0FA80F252099EE700229CE754
:10437000002231462046FFF7D7FEB4E7C47E060888
:10438000D8820020C62407082D7F0708FE2A0708C8
:10439000C724070838B50D46044613F0F3FE2A4635
:1043A00001462046BDE83840BEE6F8B5C47914F0B1
:1043B000C003064602D0402B15D0F8BD13F0FEFE18
:1043C00004F00704062C054604D10146BDE8F84078
:1043D00012488DE6304613F0E1FE2A460146BDE85C
:1043E000F8400F4884E613F071FF05460D480E4E65
:1043F0000E4FFFF7AFFD00242B79A34202D8BDE892
:10440000F840D9E514B13046FFF7A4FD2B683846D3
:1044100053F82410FFF752FE0134EDE7D1240708CA
:10442000E1240708F8240708082507087D2D070858
:1044300008B50548FFF78EFD044B53F8B80CBDE8EE
:104440000840FBF7F9B900BFA4240708D882002070
:1044500000485AE60A25070813460A46014601485D
:1044600053E600BF1625070820B10078B0FA80F0A7
:1044700040097047012070472DE9F04F87B003468F
:10448000FFF7F2FF054618B107B0BDE8F04FDFE7D0
:104490005D49DFF8A8A1DFF870B105AA184650F011
:1044A000D4FD2F4681462C46A8464FF0FF36B9F181
:1044B000000F12D14FFA86F9484622F071FC10B174
:1044C0004568002D79D1B8F1000F55D14F483146DC
:1044D000F9F749FA07B0BDE8F08F032D07D8DFE8F8
:1044E00005F0020E132D4846FAF72AF8064605AAEB
:1044F0005946002050F0A9FD01358146D7E74846CE
:10450000FAF71EF88046F2E74149484652F001FEAC
:1045100020B94049484652F0FCFD08B144F001047E
:104520005146484652F0F5FD28B93B49484652F0FD
:10453000F0FD0028DBD044F00204D8E748464BF0F9
:1045400037F9032816D199F80020382A12D199F8A2
:104550000120452A0CD04E2A0CD1002299F80230B5
:10456000312B03D0322B05D142F002021743BEE7B4
:104570000422F3E7FF22F9E7002C08BF03240023FD
:10458000E4B2CDE9008402971A461946484622F063
:104590006FFC054610B92148314699E7204842464C
:1045A0003146F9F7E0F931461E48F9F7DCF91E4BC0
:1045B000294653F8AC0C45F0BDFF1C483146F9F7CD
:1045C000D2F95CB16979A14208D019482246F9F7BD
:1045D000CAF92B68E1B29B69284698475FB1A9796F
:1045E000B94208D013483A46F9F7BDF92B68394665
:1045F000DB6928469847EB6A002BD4D00E48F9F7C0
:10460000B2F90023EB62CEE74E760708362507089D
:10461000FF410708735E07082F4507085E25070856
:104620007D2507080B260708D88200209A25070851
:10463000B2250708D2250708F525070833250708FE
:104640002DE9F04F85B00546FFF70EFF044630B167
:104650000021012005B0BDE8F04F46F01BB88649A7
:104660002846F9F739FB20B905B0BDE8F04F3DF019
:1046700099BC82492846F9F72FFB28B9012005B0DB
:10468000BDE8F04F3DF0EEBD7D492846F9F724FB2B
:1046900098BB7C4B93F9A32F83F89C0F03F5BC7157
:1046A00091F8D654012D09D0033D052D06D90CB142
:1046B00083F8A32F05B0BDE8F04FC9E691F8D754B1
:1046C000A52D00F1010013D1012A0ED16E4983F806
:1046D0009C2F002283F89D0F01F8A82C83F8A32FAC
:1046E00005B0BDE8F04F3DF005BE013A52B20124DD
:1046F000782801F11401D3D1D9E72846F9F720FF32
:10470000614B13F9A83C009303FA80F6772E834699
:1047100000F2A7802846FAF7F6FF0746002800F0C7
:104720008C80F9F70DFF0124C5B23846FAF7EBFF8C
:104730000746002800F08480F9F702FF0134019059
:10474000E4B23846FAF7DFFF804600287AD0F9F75E
:10475000F7FE01340746E4B24046FAF7D4FF81463B
:10476000002871D0F9F7ECFE01340290E4B248461B
:10477000FAF7C9FF8246002868D0F9F7E1FE013454
:104780000FFA80F9E4B25046FAF7BDFF82460028DE
:104790005ED0F9F7D5FE01340FFA80F8E4B2504646
:1047A000FAF7B1FF002855D00390F9F7C9FE039A34
:1047B0000FFA80FA1046FAF7A6FF0346002857D0F2
:1047C00004F0FD04F9F7BCFE042C7FF473AFC3B210
:1047D000012D03D9EA1E052A3FF66CAF23B1A52BA4
:1047E00002D0482B7FF466AF26480EB980F8A36F3D
:1047F000142202FB06020199C2F83C16A52B02996D
:1048000082F84E56C2F84076C2F84416A2F848968E
:10481000A2F84A86A2F84CA682F84F360AD1009B2D
:10482000194A01335B4402F8A83C90F8A33F0133D6
:1048300080F8A33F05B0BDE8F08F0446054674E755
:1048400001907EE7074687E7029090E781469AE766
:104850008046A4E75FFA88F382468046062CB7D0EC
:1048600028E70A487722214605B0BDE8F04FF3E576
:104870000134E4B2F2E700BF392607083F260708F3
:1048800095390708E8600020D882002044260708F0
:1048900010B50346FFF7E8FD30B1FCF793F8BDE82B
:1048A00010400748FFF7AEBB1846F9F749FE04462B
:1048B00080B2FCF75BF821460248BDE8104017E4DF
:1048C0004D2607085926070808B50346FFF7CCFD13
:1048D00040B10C4B0C48002223F8B02CBDE8084036
:1048E000FFF790BB1846F9F72BFE014638B1054B90
:1048F00023F8B00CBDE808400448FFF7F9BBBDE859
:104900000840A5E5D88200206B2607088126070805
:104910002DE9F04F834689B090460C461646002795
:104920004FF0190A4FF46179B8F1000F4BD030788D
:1049300025787178B378F278854242D165788D42D6
:104940003FD1A5789D423CD1E578A5EB020CDCF186
:10495000000545EB0C05CDE90632059112F0C6FBCA
:10496000079A069B059901911AFB02921AFB039381
:104970000392029343790093144A3B4629465846D2
:10498000FFF786FB207812F0B1FBE3780F4A1AFBA1
:1049900003930393A3781AFB039302936378019321
:1049A0004379009329463B4658460137FFF756FBAB
:1049B000282F04F1040406F10406B5D109B0BDE8BE
:1049C000F08F0025C7E74546DCE700BF98260708BB
:1049D000F7B50746FFF748FD044630B12E490022DF
:1049E000012003B0BDE8F04092E73846F9F7A8FD92
:1049F0002728054648DC8600781C8DF80740FAF722
:104A000082FE074690B1F9F79BFD031E0EDB234A99
:104A10002146DBB202F5AF6404EBC10CC8009CF880
:104A200005C09C4525D001313D29F5D13846FAF71E
:104A30006AFE044660B1F9F783FD1D2808D8184BBB
:104A4000334403F8A60C9DF8073001338DF8073086
:104A5000114FB11C0DF1070239442046FAF760FEF0
:104A60009DF80730042B02D0002347F8253003B00F
:104A7000F0BD0B4B0244334492F87C2503F8A72C7D
:104A800001238DF80730D1E706482722214603B0DD
:104A9000BDE8F040E0E400BF318200200077060866
:104AA000D8820020AE2707082DE9F04F3F4FDFF8EE
:104AB00004A189B0814690460C46164602F1300B9F
:104AC00094F9045000230C22394802FB03F10956E3
:104AD000A94266D00133042BF6D10C36B34504F15C
:104AE0000C04EDD109B0BDE8F08F96F90430D6F88A
:104AF00000E07279B179307A96F807C007939D4249
:104B00004DD1256875454AD16579954247D1A5793A
:104B10008D4244D1257A854241D1E579A5EB0C033C
:104B20005D425D4107EB820207EB8C0C07EB8000D6
:104B300007EB8101D2F86027DCF86037D0F8600716
:104B4000D1F860170493CDE900E203900291079B2E
:104B5000524629464846FFF79BFAE27994F9043019
:104B600007EB82022946D2F860270492227A07EBEB
:104B700082024846D2F860270392A27907EB8202AC
:104B8000D2F860270292627907EB8202D2F860279E
:104B90000192226800925246FFF760FA9DE70025D5
:104BA000C0E7B8F1000FA0D14546D6E70077060868
:104BB000D4820020AB2607082DE9FF410346FFF70A
:104BC00053FC30B145490022012004B0BDE8F0415A
:104BD0006AE718465E1CF9F7B3FC044640B222F0BF
:104BE00003F9054630B93E48214604B0BDE8F0411E
:104BF000FFF78BBA0068696801AB03C3A868186047
:104C00003046FAF780FD0446002853D003782B2B5A
:104C100005D02D2B43D0F9F793FC019009E0013426
:104C20002046F9F78DFC012303FA00F0019B0343B2
:104C3000019302262B4F4FF000082046FAF763FD40
:104C4000044628B3F9F77CFC274A002352F8041BDA
:104C5000884231D00133112BF8D1002307EB8302B6
:104C6000D2F86027904213D1B8F1020F26D0B8F1E4
:104C7000030F26D0B8F1010F14BF8DF809308DF85D
:104C80000A3008F101080136B8F1040FF6B2D4D1A8
:104C9000012E19D804B0BDE8F041FFF7D9BB0134AB
:104CA0002046F9F74DFC012303FA00F0019B23EAAB
:104CB0000003BDE70126BDE7DBB2CFE78DF80C307E
:104CC000DFE78DF80B30DCE701AB03CB2860186819
:104CD0006960A86004B0BDE8F08100BF04830020D3
:104CE000C826070800770608607E06082DE9F04F01
:104CF000834687B090460C46164600274FF0190AA7
:104D00004FF46179B8F1000F4DD0B078A5783378C1
:104D1000727896F803C096F804E07179854240D124
:104D200025789D423DD1657895423AD1E578654533
:104D300037D12579754534D165798D4214BF002569
:104D400001251AFB02921AFB0393CDE9010303929A
:104D50000091CDE904CE154A3B4629465846FFF757
:104D600097F923790593E378049363780F4A1AFB44
:104D70000393039323781AFB03930293A37801937D
:104D80006379009329463B4658460137FFF766F999
:104D9000142F04F1060406F10606B3D107B0BDE8EE
:104DA000F08F0025CDE74546DBE700BFDB2607088F
:104DB0002DE9F3478246FFF757FB064630B13E49DF
:104DC0000022012002B0BDE8F0478FE75046F9F716
:104DD000B7FB1328054663DC062747430AF10100A9
:104DE0008DF80760354CFAF78EFC04F15C0909EB8D
:104DF0000708064648B1F9F7A3FB03289FBFE3194C
:104E000083F8610001238DF807303046FAF77BFC08
:104E1000064668B1F9F794FB1D2809D8062303FB61
:104E2000054383F85E009DF8073001338DF80730A5
:104E30000DF1070241463046FAF772FCFAF763FCBF
:104E4000064668B1F9F77CFB3C2809D89DF8073085
:104E5000062202FB0542013382F85F008DF807301D
:104E60003046FAF750FC68B1F9F76AFB1D2809D8FB
:104E70009DF80730062202FB0544013384F86000E8
:104E80008DF807309DF80730062B11D0002349F824
:104E90000730A8F8043002B0BDE8F047FFF7D8BAF1
:104EA00007481322314602B0BDE8F047FFF7D4BAF5
:104EB00002B0BDE8F08700BF34830020D882002014
:104EC000AE2707082DE9F04F2DED088BDFF814A170
:104ED00097B0074690460C461546002694ED008A8A
:104EE000B5EE408AF1EE10FA73D0D4ED019A94ED4C
:104EF000029AD4ED038AB8F1000F40D095ED000A74
:104F000095ED01BAD5ED02AA95ED03AAB4EE408A5B
:104F1000F1EE10FA62D1F4EE4B9AF1EE10FA5DD197
:104F2000B4EE6A9AF1EE10FA58D1F4EE4A8AF1EE34
:104F300010FA0CBF4FF001094FF0000912A8F9F761
:104F40000FFAB0EE4B0A83460EA8F9F709FAB0EE55
:104F50006A0A05900AA8F9F703FAB0EE4A0A049023
:104F600006A8F9F7FDF9059B049A0390CDE900B373
:104F700002923346524649463846FFF789F8B0EE6A
:104F8000480A12A8F9F7ECF9B0EE690A81460EA8B2
:104F9000F9F7E6F9B0EE490A83460AA8F9F7E0F90D
:104FA000B0EE680A049006A8F9F7DAF9049B0390BA
:104FB000CDE901B3CDF80090334652460021384682
:104FC0000136FFF74BF80C2E04F1100405F1100523
:104FD00084D117B0BDEC088BBDE8F08F4FF000090D
:104FE000ACE700BFF9260708F8B50546FFF73CFA1D
:104FF000064660B1434991F882324FF4D67202FB03
:105000000311BDE8F8400022E83101205AE73E498B
:1050100005222846F8F746FE80B93A4A02F1D40341
:1050200092F882224FF4D67101FB02330022013044
:105030000C285A6103F11003F9D1F8BD2846F9F79D
:105040007FFA0B28044656D82846FAF75CFB06463A
:1050500000283DD0F9F7E8F92A4A92F882324FF455
:10506000D670611C434303EB01131A4482ED360AE8
:1050700001253046FAF747FB064670B1F9F7D4F937
:10508000204A92F882324FF4D670611C434303EBFE
:1050900001131A4482ED370A01353046FAF733FB23
:1050A000064668B1F9F7C0F9164A92F882324FF411
:1050B000D6714B4303EB04131A4482ED3C0A0135CD
:1050C0003046FAF720FB28B9BDE8F840FFF7C0B931
:1050D0000546CEE70B4E96F88272F9F7A5F94FF424
:1050E000D6737B4303EB04143444032D84ED3D0A53
:1050F000EAD1F11885E731460448BDE8F8400B22B3
:10510000FFF7AAB9D882002039260708AE2707087A
:105110002DE9F347DFF868A081460E4617464FF0A9
:105120000208002457B337F8243036F8241037F833
:105130000820994220D136F80850A91A4D424D4115
:10514000CDE900322946234652464846FEF7A0FFE5
:1051500036F80830019336F824300093524623463F
:10516000294648460134FEF779FF042C08F104086B
:10517000D8D102B0BDE8F0870025E1E73D46E7E77A
:105180000D270708F8B50446FFF76EF9054628B164
:10519000BDE8F8402A4900220120B9E72949204604
:1051A000F8F79AFDA8B9284B4FF47A714FF4FA62D8
:1051B000A3F8A812A3F8AA22A3F8AC12A3F8AE226F
:1051C000A3F8B012A3F8B222A3F8B412A3F8B6223F
:1051D000F8BD2046F9F7B4F90328064628D820463A
:1051E000FAF791FA044670B1F9F7AAF901270546D2
:1051F0002046FAF788FA10B1F9F7A2F937B9BDE8F5
:10520000F840FFF725B905460746F1E7A5F2EE227B
:1052100040F2DC539A42F2D8A0F2EE229A42EED843
:10522000094B03EB8603A3F8A852A3F8AA02CFE721
:1052300029460648BDE8F8400322FFF70DB900BF34
:105240008085002039260708D88200201E270708FD
:105250002DE9F04F91B0174607900C4615460026F1
:1052600004F115090DF1240B04224946584651F06A
:105270002DFF00238DF82830D4E90232082B72F17B
:1052800000010DF12C0A55D22F491A465046F8F765
:1052900087FB002F56D095F80080237843454ED1E8
:1052A000D4E90202D5E902139A4208BF884246D1E6
:1052B000227D2B7D9A4242D1042205F115014846F8
:1052C00051F0B8FE00283AD121692B69CB1AD3F1ED
:1052D000000949EB03091D4B059300230493B5F91D
:1052E00012300393B5F910300293194B194A0798FD
:1052F000CDE9008349463346FEF7CAFECDF814B027
:10530000237D0493B4F912300393B4F91030114A99
:105310000798CDE901A314F8203B00934946334692
:105320000136FEF79BFE082E05F1200598D111B03D
:10533000BDE8F08F08495046F8F732FBA9E74FF077
:105340000009C8E7B946D9E70E5907082A4A0708ED
:10535000BA62070831270708262707082DE9F74F03
:105360000446FFF781F8074630B16F49002201205B
:1053700003B0BDE8F04F6BE76C492046F8F7ACFC92
:10538000014638B968484FF4807203B0BDE8F04F69
:1053900050F0A8BF2046F9F7D3F883B2072B054693
:1053A00000F2B9802046FAF7AEF9824600284CD0C8
:1053B000F9F7C6F801240FFA80F95046FAF7A3F975
:1053C00068B14FF00008411E00F1100C464611F87C
:1053D000013F13F0DF0F3BD101270134E4B2FAF7AC
:1053E00092F9824600284CD0F9F7AAF801340FFA56
:1053F00080FBE4B25046FAF786F90346002842D013
:105400000190F9F79DF80134019B0FFA80FAE4B29C
:105410001846FAF778F90346002836D00190F9F7D4
:105420008FF80134019B42B2E4B218460192FAF7B8
:105430006AF9019A034650B30134E4B2032C28D828
:1054400003B0BDE8F04FFFF703B804468146B4E768
:105450006145C2D0A3F13002D2B2092A05D9A3F125
:105460006102052A07D8573BDAB2360146EA1876B8
:1054700042EA0818ABE7A3F14102052AADD8373B51
:10548000F2E78346B6E78246C2E70246CDE7284BFD
:10549000D4E71FFA89F10229D2D80BF2262189B26A
:1054A000B1F5E16FCCD80AF2262189B2B1F5E16FEE
:1054B000C6D8D4B2062CC3D8184601934AF078F95E
:1054C0000428BDD8002FBBD01A4A019B2DB202EB95
:1054D000451102EB4512184D81F8B892C1E9B0862A
:1054E000A1F8C8B2A1F8CAA281F8CC4202F5337281
:1054F000591E033311F8010F2C5C04F00304022C35
:1055000008BF203802F8010F087808B18B42F1D1AA
:1055100003B0BDE8F08F09480722394603B0BDE863
:10552000F04FFEF799BF00BF90850020392607088D
:105530002A4A0708D8820020218007085227070836
:105540002DE9F04FDFF8AC9087B0834690460C46CB
:1055500016460027B8F1000F49D0707A617AB6F983
:105560000AC0B6F90CE096F808A08142D6E90032EC
:105570003BD12168994238D16168914235D1B4F963
:105580000A10614531D1B4F90C1071452DD1257A3D
:10559000A5EB0A014D424D41CDE90032CDE9020CA7
:1055A000CDE904EA3B464A4629465846FEF770FDD7
:1055B000237A0593B4F90C300493B4F90A300393B9
:1055C000637A02936368019354F8103B00934A4650
:1055D0003B46294658460137FEF740FD112F06F19C
:1055E0001006B7D107B0BDE8F08F0025D4E74546D7
:1055F000DEE700BF5F2707082DE9F74F0446FEF7F7
:1056000033FF054630B14E490022012003B0BDE80A
:10561000F04F95E74B492046F8F75EFB30B94FF065
:10562000FF3003B0BDE8F04F3FF024BB2046F8F751
:1056300087FFC3B2102B834607D94348102229465F
:1056400003B0BDE8F04FFEF707BF2046FAF75BF85E
:105650000646E8B1F8F774FF012482463046FAF7AF
:1056600052F80646B8B1F8F76BFF01348146E4B250
:105670003046FAF748F8064600285AD0F8F760FF97
:105680000128804609D903B0BDE8F04FFEF7E0BE1F
:1056900004468246E2E78146EAE70134E4B2304656
:1056A000FAF731F80646002845D0F8F749FF00F52B
:1056B000B473B3F5347F0746E5D80134E4B230461D
:1056C000FAF721F80346002837D00190F8F738FFA1
:1056D00000F5B472B2F5347F0646D4D80134019B8C
:1056E000E4B21846FAF70FF8034640B10190F8F714
:1056F00027FF0134051E019B18BF0125E4B218469F
:10570000FAF701F808B10134E4B2062CBBD10F4B13
:105710004FFA8BFB03EB0B13C3E9EEA983F8C183AC
:10572000A3F8C273A3F8C46383F8C05303B0BDE801
:10573000F08F8046B3E70746C1E70646D1E700BFD2
:1057400090860020392607087F270708D882002086
:105750002DE9FF47DFF87090804617460D46164644
:105760004FF0000A77B3337829789942D6E90120BF
:1057700026D16968914223D1AC68211A4C424C4130
:10578000CDE9012000934A46534621464046FEF7A4
:105790007FFCAB6802936B68019315F80C3B009398
:1057A0004A465346214640460AF1010AFEF756FC96
:1057B000BAF1080F06F10C06D4D104B0BDE8F087A9
:1057C0000024DDE73C46E4E7902707082DE9F8438D
:1057D0000446FEF749FE054628B1BDE8F8432E49C8
:1057E00000220120B4E72D492046F8F775FA01465A
:1057F00028B9BDE8F8432848602250F073BD204620
:10580000F8F79EFEC3B2072B064606D92946244860
:10581000BDE8F8430722FEF71FBE2046F9F773FFE5
:10582000074628B3F8F78CFE051E18BF0125012492
:105830003846F9F768FF0746E0B1F8F781FE013412
:105840008046E4B23846F9F75EFF0746A0B1F8F7A4
:1058500077FE01348146E4B23846F9F754FF08B1C7
:105860000134E4B2032C09D0BDE8F843FEF7F0BDE3
:105870000446DDE78046E5E78146EDE7094B76B271
:105880000C2202FB063686F8C854C6F8CC84C6F84B
:10589000D094BDE8F88300BFA08700203926070810
:1058A000A5270708D88200202DE9F04FDFF8849063
:1058B00091B007468846164600240DF12C0A04EBE9
:1058C000840508EB050358F805001B790290514642
:1058D00002A88DF80C3044F08BFE4EB3731970594A
:1058E0001B790490052204A902A88DF8143051F008
:1058F000A1FB0DF1180BB0FA80F5594604A86D090B
:1059000044F076FECDF800B023464A462946384694
:10591000FEF7BEFB2346CDF800A04A46294638468E
:105920000134FEF79BFB802CC9D111B0BDE8F08F8C
:105930003546EFE7B42707082DE9F04F89B0054653
:10594000FEF792FD044630B163490022012009B000
:10595000BDE8F04FA8E72846F8F7F2FD7F28064695
:1059600000F3B2802846F9F7CEFEB3005A4A0393FB
:1059700006EB8603D118D450584B0C71CDE9014386
:105980000546A346A146A2462746A046029B05AA75
:1059900013F8010B029394460023AE4615F8011B41
:1059A00019B1884201D00A2B0CD120336B444FF03F
:1059B0000005884203F80C5C08D009B0BDE8F04F40
:1059C000FEF746BD0CF8011B0133E6E708F1FF3393
:1059D0000EF10105032B31D8DFE803F0591B026EED
:1059E0004FF0010C12F8011B61B33D48002310F881
:1059F00001EB8E455AD00133082BF8D139480023EA
:105A000010F801EB714553D10CFA03F349EA03098D
:105A1000E8E7012112F8013BA3B14E2B3CD0452B06
:105A20003CD0532B3CD0572B3CD0552B3CD0442B57
:105A3000F0D1052301FA03F31F43EBE705A8F8F7BC
:105A40007FFD834608F101085FFA88F8B8F1050F79
:105A50009CD10399244B019A3144581803F5A5634E
:105A60000B4402F00F0204F00F0444EA071442EA68
:105A70000B123F1180F8282580F829A580F82A9577
:105A8000DC701F7109B0BDE8F04F2FF067B805A8B2
:105A9000F8F756FD0190D5E70023CBE70123C9E7CE
:105AA0000223C7E70323C5E70423C3E79A46A5E714
:105AB0000133072BA4D195E705A8F8F741FD10287D
:105AC0000446A8BF0024BDE708487F22214609B04C
:105AD000BDE8F04FFEF7C0BC00880020A47E060899
:105AE000A97E0608B17E0608D8820020AE270708E6
:105AF0002DE9FF47DFF86C90804617460D461646A5
:105B00004FF0000A67B333882A889A4226D16C88FE
:105B10007288A21A54425441F2780292B278214615
:105B2000CDE90032404653464A46FEF7B1FAEB78DB
:105B30000293AB78019335F8043B00934A465346F1
:105B4000214640460AF1010AFEF788FABAF1100F21
:105B500006F10406D6D104B0BDE8F0870024DBE7E7
:105B60003C46E4E7BE2707082DE9F0410546FEF76D
:105B70007BFC044628B1BDE8F04124490022012005
:105B8000B6E72846F8F7DCFC0F28064636DC284640
:105B9000F9F7B9FD1E4FDFF884800546A036284688
:105BA000F8F7CEFC37F8023B98421FDC012C08EBDB
:105BB000860311D0022C12D0A3F8280528462C21E8
:105BC00051F057FA054668B10135012301346BB134
:105BD000032CE4D1BDE8F08183F82A05EEE783F8D1
:105BE0002B05EBE7A21E53425341EFE7094B00227E
:105BF00043F82620BDE8F041FEF72ABC21460648BE
:105C0000BDE8F0410F22FEF727BC00BF808A0020CC
:105C1000B87E060800880020AE270708D88200203A
:105C20002DE9F04FDFF8B49085B00646884614465B
:105C30004FF0000B062303FB0BF505F5307500272D
:105C400018F805A0002C44D0625DAAEB0200414286
:105C50004141CDE900725B464A4630460391FEF76A
:105C600017FA0399CDE9007A5B464A463046013778
:105C7000FEF7F4F9062F05F10105E1D10BF1010B57
:105C8000BBF1060FD6D1DFF854904FF4397518F8F0
:105C900005B0A5F5397AF4B1635DABEB0302574269
:105CA0005741CDE900A34A46062339463046FEF760
:105CB000EFF90623CDE900AB4A4639463046FEF7F8
:105CC000CDF9013540F2ED239D42E0D105B0BDE8AC
:105CD000F08F2146C6E72746EBE700BFD02707082D
:105CE0007FB50346FEF7C0FB044630B119490022D8
:105CF000012004B0BDE8704092E71749164E6A468D
:105D000018464FF0A2F901AD80B1032C03D1FEF784
:105D10009FFB04B070BDF8F713FC6A4645F8040B0E
:105D20003146002001344FF090F9EDE7032CEED11D
:105D3000DDE90145039E29463246E0B22FF06EF8B8
:105D40000028E4D0054833462A462146FEF7D0F91C
:105D5000DFE700BF008800204E760708D02707083D
:105D60002DE9FF47DFF89890804617460C46164607
:105D70004FF0000A002F41D0B6F90030B4F90010FE
:105D8000B6F90220B6F9040096F906C0994233D15B
:105D9000B4F9021091422FD1B4F9041081422BD1F1
:105DA00094F90610A1EB0C0569426941CDE9003276
:105DB000CDE9020C53464A4640460D46FEF768F9C7
:105DC00094F906300393B4F904300293B4F9023025
:105DD000019334F9083B00934A465346294640460E
:105DE0000AF1010AFEF73AF9BAF1120F06F10806B4
:105DF000C0D104B0BDE8F0870021D7E73D46DFE71A
:105E0000E427070830B585B00546FEF72DFB0446AC
:105E100010B32E490022012005B0BDE830409FE7B5
:105E20002D2B03D0A3F13002092A4AD8042C04DD1B
:105E300005B0BDE83040FEF70BBB2846F8F780FB05
:105E400004AB621C03EB440424F80C0C15F8013F6E
:105E5000303B092BFAD914462B78002BE0D1052CC6
:105E6000E6D1BDF80430BDF90450112BE0D8BDF9DE
:105E70000600A0F5FA739BB2B3F5FA6FD8D8BDF956
:105E80000810A1F5FA739BB2B3F5FA6FD0D8BDF93B
:105E90000A209042CCDC9142CADBBDF90C4004F1EF
:105EA0007D039BB2FA2BC3D8094B03EBC503A3F8C0
:105EB0001608A3F81818A3F81A2883F81C4805B088
:105EC00030BD202BB4D101352246C4E7EE8A002034
:105ED000D88200202DE9F04F80468FB017460C463F
:105EE00016464FF0000A23780793B4F902906378BE
:105EF0002068A2880893237994F905B00A90ADF838
:105F00002C200993B9F1000F3DD0002F40D030680C
:105F1000BDF828500C9080B2B288ADF8342085428C
:105F200031787378B6F9022096F804E02ED19145C5
:105F30002CD1BDF82C50BDF83400281A45424541FB
:105F4000CDE901320091CDE903EB124A53462946CF
:105F50004046FEF79DF8099B0E4ACDF810B0CDE9FA
:105F60000293089B0193079B0093294653464046A2
:105F70000AF1010AFEF772F8BAF1240F04F10604DF
:105F800006F10606AFD10FB0BDE8F08F0025D7E7C8
:105F90003D46E0E7F9270708034B9A780021101ADD
:105FA000997018BF012070475885002010B5114B1B
:105FB000014603F11C0253F8044B41F8044B934291
:105FC000F9D11B880B800B4900F11E0351F8044BDB
:105FD00043F8044B9142F9D111881980054B3C30AC
:105FE00053F8041B40F8041B9342F9D11B8803802B
:105FF00010BD00BFA09D0608104A117A537A0B43CA
:10600000D17C0B4351780B4391780B43D1780B43F0
:1060100011790B43917B0B43917E0B4392F8231034
:106020000B4392F82F100B4305D192F84100013831
:1060300018BF012070470120704700BF60CC0020CE
:10604000F0B589B0044649F0B3FB10F0FF020CD163
:10605000394B9978394B4FF4D67000FB0131012050
:1060600009B0BDE8F040FFF735BF354905222046AD
:10607000F7F718FEA0B9304B9A78304B4FF4D67131
:1060800001FB02332F4A15689488062606FB00F2AE
:106090009918013024289D508C80F7D109B0F0BDAB
:1060A00020462949284E01AA4EF0CFFF4FF0FF337A
:1060B000079302AD002478B1062C02D1FEF7C8F98F
:1060C000ECE7F8F73DFA01AA45F8040B3146002049
:1060D00001344EF0BAFFEEE7042CEFDD029B232BD8
:1060E000ECD8039E112EE9D8049D3C2DE6D8059CE2
:1060F00004F57A72B2F5FA6FE0D80698FF28DDD879
:1061000007994A1C402AD9D80B4A92784FF4D6777F
:106110007A43062707FB03220C4B134483F8D8006D
:106120000B4883F8D46083F8D550A3F8D64083F8A1
:10613000D910FFF785FFB1E7588500208084002043
:1061400039260708BE9D06084E760708AC83002056
:106150002A4A070870B5054608460E4649F028FB4E
:106160003146044602462846F7F79CFD60B92B5D90
:10617000A3F13002092A06D923F02003413B192B51
:1061800001D90134281970BD0020FCE72DE9F04F3A
:106190009BB091460E900F930C46154600260F9B20
:1061A0005A1C01D0B34266D1A446BCE80F0010AF20
:1061B0000FC7DCF800303B6023790993237C0B93F5
:1061C00094F911300C93A37C94F80C8094F813A0EC
:1061D0000A9207460D93B9F1000F5AD0AE46BEE8B9
:1061E0000F000DF1540CACE80F00DEF80020149BFA
:1061F000CCF80020534033F07F43864695F804B036
:10620000A96895F80CC0E87C3FD1099A5A453CD161
:1062100077453AD1E04538D10A9A8A4237D1AAEB7C
:106220000003594259410A9B1B4A0E98CDF81CA005
:10623000CDE90583099B03930D9B02930C9B01936E
:106240000B9B0093049733468B46FDF721FF0A9B77
:10625000114A0E98CDF81CA0CDE90583099B039344
:106260000D9B02930C9B01930B9B00930497334669
:106270005946FDF7F3FE0136402E04F1140405F1F2
:1062800014058CD11BB0BDE8F08F0021CBE7194677
:10629000C9E7CB46DBE700BF632A07082DE9F04FCB
:1062A000074687B016460C4615464FF0000BD4E95A
:1062B000009AD4F8088066B3A8688045D5E9002123
:1062C00025D1914523D1AAEB010359425941CDE98A
:1062D000019A114ACDF800805B4638460591FDF7DA
:1062E000D7FE05990C4ACDF800805B46CDE9019AAE
:1062F00038460BF1010BFDF7B1FEBBF1080F04F1BD
:106300000C0405F10C05D2D107B0BDE8F08F0021D7
:10631000DDE73146E6E700BF842A07082DE9F04FA4
:10632000A1B0174610900C4615460026A646BEE8BA
:106330000F000DF1480CACE80F0023680B939EE8AA
:106340000700238A0C93638A0D93A38A0E93E38A32
:1063500094F80480D4F808B094F80CA094F818903D
:106360000F938CE80700002F5CD0AE46BEE80F000C
:106370000DF1640CACE80F009EE807008CE8070004
:1063800095F818C029682879AB682A7BCC4547D195
:10639000804545D10B98884242D1924540D19B45DA
:1063A0003ED1169A1D9B9A423AD117991E9BCB1A41
:1063B000594259410F9B08930E9B07930D9B0693DF
:1063C0000C9B194A1098CDF80CA0CDE904B30B9B97
:1063D000CDF80090CDE9018333461191FDF758FEC9
:1063E00011990F9B08930E9B07930D9B06930C9B93
:1063F0000D4A1098CDF80CA0CDE904B30B9BCDF855
:106400000090CDE9018333460136FDF727FE042EC7
:1064100004F11C0405F11C0588D121B0BDE8F08F02
:106420000021C7E73946DCE7952A07082DE9F04F38
:10643000DFF864A0DFF864B085B0064689461546EB
:106440001F460024002F01DBA7421CD119F804804D
:10645000FDB12B5DA8EB03020AEB830351425B6A9B
:106460000093514123465A4630460391FDF710FEF2
:1064700003990AEB88085A46D8F82430009330462E
:106480002346FDF7EBFD01340E2CDBD105B0BDE852
:10649000F08F2946EDE700BFA09D0608B72A070840
:1064A0002DE9F0418AB004460D4649F081F910F01B
:1064B000FF000FD13D4B1A783AB94FF0FF333C49FA
:1064C00001200AB0BDE8F04160E66B1C6BD02B46A2
:1064D0000246F4E7374905222046F7F7E3FB38B9CF
:1064E00033484FF47E710AB0BDE8F04146F058BF22
:1064F00020463149304E6A464EF0A7FD01AD0024DA
:1065000078B1092C02D1FDF7A3FF4CE0F8F718F899
:106510006A4645F8040B3146002001344EF095FDE3
:10652000EEE7092CEFD101993F29ECD8DDF808E01E
:10653000BEF1010FE7D8DDF80CC00CF10103402BD0
:10654000E1D8049F382FDED8059E072EDBD8069DA4
:106550001A4A05F5742303F510739342D3D8079CA8
:10656000072CD0D8089800F5742303F510739342D4
:10657000C9D8099AFF2AC6D8114B4FF0140808FB56
:10658000013309B2D8650F4883F864E083F865C029
:1065900083F8667083F858605D6583F8604083F81F
:1065A0006720FFF77DFF0AB0BDE8F081248200205C
:1065B000B4CC0020392607084E76070880841E00D8
:1065C00060CC00202A4A07084FF0FF3168E770B519
:1065D00086B0044649F0ECF810F0FF0205D12249DC
:1065E000012006B0BDE8704058E62049052220464B
:1065F000F7F758FB38B91C4840F2FF3106B0BDE848
:10660000704046F0CDBE20461949194E01AA4EF001
:106610001CFD02AD002478B1042C02D1FDF718FF57
:106620001FE0F7F78DFF01AA45F8040B3146002063
:1066300001344EF00AFDEEE7042CEFD1029A072A4E
:10664000ECD80C4B0C480C2101FB0233039AC3F825
:106650005C25049AC3F85425059AC3F85825FFF71A
:10666000B6FF06B070BD00BFB4D1002039260708C0
:106670004E76070860CC00202A4A07082DE9F0432F
:106680008DB0044649F094F810F0FF0205D13E4960
:1066900001200DB0BDE8F04340E63C49052220460C
:1066A000F7F700FB38B938484FF47E710DB0BDE8FC
:1066B000F04346F075BE20463549354E01AA4EF0EE
:1066C000C4FC02AD002478B10A2C02D1FDF7C0FE53
:1066D00057E0F7F735FF01AA45F8040B31460020D3
:1066E00001344EF0B2FCEEE70A2CEFD1DDF8088061
:1066F000B8F1030FEAD8DDF80CE0BEF1010FE5D8E0
:10670000DDF810C0BCF1070FE0D8059F214A07F55E
:10671000742303F510739342D8D8069E072ED5D85C
:10672000079D05F5742303F510739342CED8089C9A
:10673000B4F5004FCAD20998B0F5004FC6D20A99F5
:10674000B1F5004FC2D20B9AB2F5004FBED2124B38
:106750004FF01C0909FB0833A3F8C6050F4883F85E
:10676000CCE583F8B8C5C3F8B47583F8C065C3F841
:10677000BC55A3F8C445A3F8C815A3F8CA25FFF76C
:106780007DFF0DB0BDE8F08314D200203926070844
:106790004E76070880841E0060CC00202A4A070835
:1067A0002DE9F04FA1B0CDE90C011546002414AE3F
:1067B0000D9A02EB441263010DF1400C02F1200E20
:1067C00010685168674603C708327245BC46F7D166
:1067D000002D00F081802B4418AF03F1200C1868C5
:1067E00059683A4603C2083363451746F7D19DF806
:1067F00040300B939DF860100B98BDF842709DF8E7
:106800004480BDF846909DF848A0BDF84AB09DF878
:106810004C30BDF84E2081425CD1BDF86210B942C7
:1068200058D19DF86410414554D1BDF866104945D2
:1068300050D19DF8681051454CD1BDF86A105945AA
:1068400048D19DF86C10994244D1BDF86E10914228
:1068500040D11CA914A8CDE90E3248F049FFDDE96A
:106860000E32B0FA80F14909CDE905B30B9B0093D4
:10687000CDE90726CDE9039ACDE90178174A0C98AE
:106880000B912346FDF704FC0B99BDF84E3007939E
:106890009DF84C300693BDF84A3005939DF848307A
:1068A0000493BDF8463003939DF844300293BDF83D
:1068B000423001939DF840300093084A0C980896A6
:1068C00023460134FDF7CAFB082C7FF471AF21B0D9
:1068D000BDE8F08F0021C7E72946D6E7CF2A070891
:1068E0002DE9F04190B0044648F062FF10F0FF023D
:1068F00005D14549012010B0BDE8F04150E74349BA
:10690000434F01AA20464EF0A0FB41496A464EF093
:106910009CFB06AE0024354600286ED0092C61D1C0
:106920003A4901AA00204EF090FB0646002869D0A3
:1069300048F03EFF044638B10F2828BF0F242246F6
:10694000314602A84EF0ACFB04F14003DDF818809C
:106950000DEB0304B8F1070F4FF0000304F8383CC7
:106960004DD8DDF81CE0BEF11C0F48D8DDF820C082
:10697000BCF1FF0F43D8099F1C2F40D80A9EFF2E61
:106980003DD80B9C1C2C3AD80C98FF2837D80D9971
:10699000022934D80E9AFF2A31D81E4B03EB481334
:1069A00003F2346303F8084C03F810EC23F80ECC20
:1069B00003F80C7C23F80A6C23F8060C03F8041C7B
:1069C00023F8022C02AC224603CAAA42186059607E
:1069D000144603F10803F6D10F48FFF781FF10B00A
:1069E000BDE8F081F7F7ACFD6A4646F8040B39467E
:1069F000002001344EF029FB8EE7092C90D0FDF7E2
:106A000027FDECE704469FE784D20020444B0708AB
:106A10004E76070860CC00202A4A070838B5064D94
:106A2000002455F834000134FDF794FAFDF7C4FA58
:106A3000352CF6D138BD00BFD89D060830B52748A3
:106A400085B0FDF787FAF4F791FE28B9244805B020
:106A5000BDE83040FDF7D6BAF5F754F908B921483A
:106A6000F5E7F5F785F90268037D81790446407CF6
:106A70000290207C0190608A009052081A48FDF72D
:106A80001DFBE51D0C3415F8010BFDF7F9FAA542C5
:106A9000F9D1164C1648FDF75DFA6378022B06D043
:106AA00007D9032B10D11348FDF754FA0CE0124814
:106AB000FAE704F580541148FDF74CFA94F8B43124
:106AC000022B06D0032B06D005B0BDE83040FDF701
:106AD00073BA0B48E8E70B48E6E700BF032B07084B
:106AE0000D2B07081B2B07082A2B0708C04E002078
:106AF000582B0708682B07086E2B07087B2B070805
:106B0000812B07089A2B07082DE9F3473549DFF851
:106B1000D49001AA4EF099FA4FF0000A4FF0FF35D9
:106B2000564654465746A84678B9BAF1040F3DD0A8
:106B3000BAF1050F44D0BAF1030F13D02A492B46FE
:106B40004246012043F032FE0EE0BAF1040F09D8AC
:106B5000DFE80AF0030D12171C00F7F7F1FC80467E
:106B600003281BD9FDF774FC02B0BDE8F087F7F7E6
:106B7000E7FC0546A828F4E7F7F7E2FC07463F28BC
:106B8000EFE7F7F7DDFC04463F28EAE70378482BF8
:106B900003D0562BE6D1012600E0002601AA494683
:106BA00000200AF1010A4EF050FABDE70F4BA9226E
:106BB00002FB085203EB4203B3F82467C6F34036E6
:106BC000A92303FB0855A401084B04F47C6407F0D7
:106BD0003F0703EB45033C4344EA4634A3F824470C
:106BE000C2E700BF4E76070884D3002060CC0020A7
:106BF0002DE9F3412649DFF8988001AA4EF025FAE5
:106C0000002504462F464FF0FF366CB9022F0BBF0C
:106C1000204920498D55334612BF2246334622462D
:106C20000120FFF703FC04E037B1012F12D0FDF77C
:106C30000FFC02B0BDE8F0812046F7F781FC0D287B
:106C40000646F4D801AA414600204EF0FEF901376D
:106C50000446DAE710482146F7F73EF805460028D3
:106C6000F0D00E482146F7F737F860B10C482146BE
:106C7000F7F732F848B10B482146F7F72DF800280E
:106C8000D5D10325DEE73D46DCE70225DAE700BF84
:106C90004E76070878800020AC2B07087949070852
:106CA000AD6B07088B7207082DE9F04F2DED028BB5
:106CB0004D484E4D9FED4E8A8BB0FDF719FA0027D7
:106CC000B946BA464B4B4C4A196800238B4227DB26
:106CD00001371D2F05F14805F4D14849484BD1E94A
:106CE0000021520942EAC1624649186809684FF416
:106CF0007A73B0FBF3F34448FDF7FAF90A2299FBE3
:106D0000F2F302FB139000909AFBF2F13F4802FB72
:106D100011A2FDF7EDF90BB0BDEC028BBDE8F08FD1
:106D200052F8040BA84201D00133CFE7AC6A4CB152
:106D300007EE904AB8EEE77AC8EE077AFDEEE77AFA
:106D400017EE904AAB6B0893D5E90C637609E96BB3
:106D500046EAC3665B090993089B4FEAE47B6143FB
:106D6000A4FB030C03FB0B1141F28833C01841EB69
:106D70000C014FF47A72002349F084FB099A804693
:106D800004FB02F1A4FB060C41F28833C01806FB99
:106D90000B1141EB0C014FF47A72002349F072FBA6
:106DA0002B6C0196042F4FF47A72B3FBF2F3069327
:106DB0004FF00A0318BF814490FBF3F203FB12006B
:106DC000CDE9042098FBF3F203FB1283CDE9022303
:106DD000089B00932A680E482346394618BFC244D0
:106DE000FDF786F974E700BFB12B0708C80800203B
:106DF00000247449706E0120C86D0120406E01208E
:106E0000486E0120506E01202D2C07084F2C0708DA
:106E1000F82B07081FB50A4B03930A4B02930A4B42
:106E200001930A4B00930A4A0A4B0B490B48FDF7A2
:106E30005FF90B490B4805B05DF804EBFDF758B955
:106E40002A4A07089E2C0708A72C0708B02C070819
:106E5000202007087D2C070833200708832C07080B
:106E6000BC2C0708CC2C0708F8B50C480C4E0D4F6D
:106E70000D4DFDF73DF90D4B1A68C2F500729200F9
:106E8000002422B156F824103846FDF731F90134B8
:106E9000222C02D055F82420F3E7F8BDD52C0708A2
:106EA000809F0608EB2C0708703C00206C34002003
:106EB00070B5124B93F86C2CD2B1192A94BF104BB9
:106EC00010491148114D124E98BF03EB82034FF049
:106ED000000498BFD3F86812FDF70AF9214655F867
:106EE000042B30460134FDF703F9082CF6D170BDB0
:106EF000BDE870400748FDF785B800BF60CC0020B2
:106F0000A09D0608F92C0708012D0708D0D80020FD
:106F1000192D0708282D07082DE9F84F054648F0D8
:106F200047FCDFF8EC800446D8F80090C0B9304840
:106F3000304D314FFDF70EF8012655F8041B59B1BD
:106F40000B783BB106FA04F313EA090F02D0384676
:106F5000FDF7B4F80134F0E7BDE8F84FFDF72CB8C1
:106F6000024626492846F6F79DFE78B92448214C6A
:106F7000214DFCF7EFFF54F8041B0029ECD00B78EF
:106F8000002BF8D02846FDF799F8F4E72B78DFF8C6
:106F900064B02D2B03BF013504F1FF344FF0010A1B
:106FA0004FF0000A00265BF8047B1FB9BDE8F84FDC
:106FB00043F002BB224639462846F6F773FEA8B9CD
:106FC0000120B040BAF1000F0AD0F7F70FFC0D48CE
:106FD000FCF7C0FF39460C48BDE8F84FFDF788B80C
:106FE00040EA0900C8F800000848F1E70136DAE78E
:106FF0003F2D070870A00608BC7C0708492D07082C
:107000004E2D07085A2D07087D2D0708632D070808
:107010009C3E00202DE9F84F054648F0C9FBDFF8FB
:10702000F4800446D8F8986CC8B93148314DDFF87F
:10703000D480FCF78FFF0127E3B205EB8302D2F87F
:10704000541341B107FA03F3334202D04046FDF72F
:1070500035F80134F0E7BDE8F84FFCF7ADBF024664
:1070600025492846F6F71EFE60B92448244C254DD4
:10707000FCF770FF54F8041B0029ECD02846FDF7FC
:107080001DF8F7E72B78DFF878B02D2B03BF01351B
:1070900004F1FF344FF0010A4FF0000A4FF00009ED
:1070A0005BF8047B1FB9BDE8F84F43F085BA224670
:1070B00039462846F6F7F6FDB8B9012303FA09F375
:1070C000BAF1000F0CD026EA03030F48C8F8983C29
:1070D000FCF740FF39460D48BDE8F84FFDF708B80A
:1070E00033430B48C8F8983CF2E709F10109D7E7A8
:1070F0003F2D0708A09D0608492D07084E2D0708BB
:10710000F4A00608BC7C07085A2D07087D2D070847
:10711000632D070860CC00202DE9F047814648F038
:1071200047FB494E0446376800BB4848484D494E26
:10713000FCF7C4FF4FF00C0808FB04F35A5D012371
:10714000013A93403B4206D020461CF0F3FA014638
:107150003046FCF7B3FF0134182CEDD117B93E4887
:10716000FCF7F8FEBDE8F047FCF726BF02463B49B6
:107170004846F6F797FD054678B93948FCF7EAFE28
:107180002C46344D20461CF0D5FA013401462846E1
:10719000FCF794FF1A2CF5D1E4E799F800302D2B79
:1071A00003BF09F1010904F1FF344FF0010A4FF068
:1071B000000A002528461CF0BDFA224680460146FA
:1071C0004846F6F76FFD002836D1BAF1000F1CD003
:1071D000182D17D0192D0AD1736822483360FCF797
:1071E000B9FE41462048BDE8F047FCF781BF1F4B80
:1071F0000C2202FB053393F890230123013A9340BC
:107200003B43EAE76FF07F43E7E7182D03D1C6F869
:1072100000A01748E3E7192D01D17760F9E7134B78
:107220000C2202FB053393F890230123013A93408B
:1072300027EA03033360ECE701351A2DBAD1BDE824
:10724000F04743F0B9B900BFB08000206B2D0708AC
:1072500030A106087C2D0708752D0708492D070861
:10726000812D07085A2D07087D2D0708A09D0608C7
:10727000632D07082DE9F341044648F099FA0428E4
:107280003DD1661E2546E71C16F8010FF6F7F2FC05
:10729000BE423070F8D1DFF87880271D15F8016BF9
:1072A000404631464FF0E5FE20B1314628464FF0CA
:1072B000E0FE20B102B0BDE8F041FDF7C9B8BD4223
:1072C000ECD1204622F07AF90F48FCF743FE0F4933
:1072D0000F48002311F8012F10F8014B08326A44BF
:1072E0000133042B02F8084CF4D1002309488DF82F
:1072F00004306946FCF7FCFE02B0BDE8F0810028CE
:10730000E2D0FDF7A5F8DFE78C2D070800D90020B3
:1073100068A206087E2D070808B504460648FCF753
:1073200019FE064B1868F8F787FA054B18681FF026
:10733000FBFE204606F050FF922D07082082002019
:107340002C820020034808B5FCF704FE0120FFF75B
:10735000E3FF00BF9E2D070808B50C4B93F8A02C47
:10736000012A12D193F8A53C062B0AD00A2B04D08F
:107370000748BDE80840FCF7EDBD22F0F1FB0548E9
:10738000F7E721F04FF90448F3E708BD60CC00208F
:10739000B72D0708C62D0708E02D070808B50A48CD
:1073A000FCF730FE094B1868F8F746FA084B002442
:1073B00083F8C44CC3F8044D064B1C7017F0E0FC76
:1073C0002046FFF7A9FF00BFF92D07082082002003
:1073D00060CC00200175002008B5214B214C1D68B0
:1073E000D4F8100D1FF0A0FE28461FF09DFED4F823
:1073F000100D41798B0704D4036841F002019B69A9
:10740000984700210846F9F783F900210120F9F790
:107410007FF9D4F8100DFAF74EF878B10121002069
:10742000F9F776F9D4F8100DFAF766F80146284610
:10743000FAF73EF800210846F9F76AF92846FAF704
:107440003AF80028E5D001210846F9F761F9284605
:10745000FAF752F80146D4F8100DFAF729F8D4E7F4
:107460002C82002060CC0020F7B50546FCF7FCFF1D
:10747000044620B103B0BDE8F040FCF7E9BF284660
:107480001E491E4F01AA4DF0E0FD2646254640B993
:107490000B2D18D901461A480B22FCF7DDFF03B06B
:1074A000F0BD44B1012C0AD001AA394600200134B4
:1074B0004DF0CBFDEBE7F7F743F80546F4E7F7F7B8
:1074C0003FF80646F0E7022C0ED1A6F57A73B3F525
:1074D0007A7F05D90B484FF4FA624FF47A71DCE7F2
:1074E000094B03EB45039E80074B084803EB45031C
:1074F0002946B3F90420FCF7FBFDD0E74E760708D8
:10750000AE27070833520708706E0120232E0708A4
:1075100070B50446FCF7A8FFC0B11F4B1E680136CA
:1075200030461CF007F934460546E8B901341A2CF8
:10753000A8BF002420461CF0FDF80546A0B9B442BF
:10754000F4D1BDE870401548FCF75CBD2046F6F765
:10755000F7FF04461CF0EEF8054628B9214610480E
:10756000BDE87040FCF7C4BD0B4B1C601BF07CFFFA
:107570002A460C482146FCF7BBFD192C9DBF0A4B3F
:107580000C2202FB04330020BDE8704098BF93F842
:1075900090031BF081BF00BF0C120020302E0708A3
:1075A000442E07085A2E0708A09D060870B51D49ED
:1075B00090B0052204464FF069FD70B91A4A13785D
:1075C0002BB901211170194A1370194A1370194807
:1075D00010B0BDE87040FCF715BD174903222046E6
:1075E0004FF054FDC0B9104E104D3378104C7BB1A4
:1075F0002B786BB12278114901A8F6F7D1F901A8CF
:10760000FCF783FD002333702B70237010B070BD26
:107610000B48FCF7F7FCF5E70A4810B0BDE87040EE
:10762000FCF773BD42370708248200202582002022
:10763000268200206F2E0708B6390708852E070816
:10764000C82E0708DC2E070870B5124E337890B0AC
:10765000A3B1114D2B788BB1104C1149227801A8A0
:10766000F6F79EF901A8FCF750FD0E48FCF74DFD1A
:10767000002333702B70237010B070BD0A48FCF7E4
:1076800069FC21F07FFFF6F7BDFF21F085FF0020A8
:10769000FFF742FE2482002025820020268200205F
:1076A000852E0708EB2E0708092F07082DE9F0475C
:1076B0008CB0074610F8013B202BFAD00025204C57
:1076C000DFF88480DFF88490DFF884A02E466946D6
:1076D000204610F031FC394668464FF01AFDE0B103
:1076E00069464046FCF7EAFC4946684648F000F81F
:1076F00000BB204610F046FD124B014600782028C2
:1077000014BF50461846FCF7D9FCFCF755FC204640
:10771000FCF74BFEFCF750FC0136013540F292239A
:107720009D4204F10C04D2D10EB942F045FF0CB0D9
:10773000BDE8F08700212046FCF72CFEE5E700BFFE
:10774000C47E0608FE2A0708CB2407082D7F0708F9
:107750007E2D07082DE9F04F2DED028B8FB00578B7
:10776000202D064600F10100F9D0304648F020F8FF
:10777000044618B1012822D12A2D20D199489A4DCA
:10778000DFF88482FCF73EFC002640F29227284670
:1077900002A910F0D1FB02A94046FCF78FFC01368C
:1077A00028462146FCF7F6FDFCF706FCBE4205F133
:1077B0000C05ECD10FB0BDEC028BBDE8F08F3D2184
:1077C00030464FF056FC002800F0058103469946EC
:1077D00013F8012D202AFAD0A9EB060901308046C2
:1077E000074610F8013B202BF9D07F4D4FF0000ADF
:1077F0005FFA89F940F2922B02A9284610F09CFB0F
:1078000002A847F0D5FF02A9024601903046F6F7DC
:1078100049FA754B044658BB019A4A4528D10C22B7
:1078200002FB0A33DB7903F00706062E2FD1404610
:10783000F6F726FA6D4902A847F05AFF20B16C49C5
:1078400002A847F055FFE0B998F80030222B18D174
:10785000404647F0ADFF08EB000313F8013C222B34
:107860000FD1821E08F10101284610F04BFDA1E75F
:107870000AF1010ADA4505F10C05BDD142F09CFE82
:1078800098E7404647F094FF41460246ECE713F084
:10789000C0030AD0402B6AD05648FCF7B9FB2846F3
:1078A000FCF783FDFCF788FB84E798F80030002B99
:1078B000F2D0514940464FF01CFC0446404647F088
:1078C00077FF8442E8D14046F6F7AEFD2846B0EE99
:1078D000408A10F063FC07EE900AF8EEE77AF4EEC7
:1078E000C87AF1EE10FAD7D8284610F067FC07EEF8
:1078F000900AF8EE677AF4EEC87AF1EE10FACBDB74
:10790000052E1AD118EE104A3C4902A847F0F0FEA5
:1079100048B93B4B93F8471DE2B2914203D0002C8B
:1079200045D183F8AB4D284610F02CFC052E43D8EA
:10793000DFE806F041414B4B4D4F042E12D13A4641
:1079400017F8013B202BFAD0092BF8D0013A00247C
:107950000A2112F8013F303BDBB2092BD4D801FBDE
:107960000434F6E74046F6F7EBFD0446CCE728463C
:1079700010F0ACFC90F804B0814627462346A2469E
:10798000BB4500D91BB1BAF1000F85D0BCE7D9F8CF
:107990000030414653F82700F6F79EF9002805BF4E
:1079A0003C46012300234FF0010A0137E8E701229A
:1079B00083F8AB2DB7E7047002A91248FCF77EFBF1
:1079C00000212846FCF7E6FCF4E60480F4E70460B6
:1079D000F2E70460F0E730460FB0BDEC028BBDE883
:1079E000F04F63E6102F0708C47E06082D7F0708B6
:1079F000222F07085C2F07082D2F07083B2F0708A9
:107A000060CC0020512F0708CB2407082DE9F8434C
:107A10002BF05CFD20B9BDE8F8434948FCF79ABA61
:107A20004848494C494E4A4FDFF87081FCF7EAFA62
:107A300000256378FF2BA94605F1010576D0227851
:107A4000FF2A73D029463046FCF752FB2378A178F1
:107A5000062B5AD8DFE803F004343A42594A520060
:107A6000072954D83B4B03EB8103D3F8D024384685
:107A7000FCF73EFBA1794046FCF73AFBE17936483A
:107A8000072997BF334B354A03EB8103D3F85425BD
:107A9000FCF72EFB324B334803EB091303F6FC597A
:107AA000B3F8FE1DFCF724FBB9F8021001F0030146
:107AB000012936D0022940D02B48FCF719FB33E0CE
:107AC0002A4A2B4B002908BF1A46D0E7062920D89E
:107AD000204B03EB8103D3F8F024C8E707291AD819
:107AE0001C4B03EB8103D3F80C25C0E7092914D8FC
:107AF000184B03EB8103D3F82C25B8E779B11D4A65
:107B00001D4B022918BF1A46B1E71C4AAFE71C4AB1
:107B1000ADE71C4AABE71C4AA9E71C4AA7E71C4A89
:107B2000A5E71C48FCF76EFAFCF746FA402D04F175
:107B300010047FF47EAFBDE8F8831748F2E700BF7A
:107B4000FB2F07082A30070854DA00203A300708CC
:107B50004E300708A09D0608763007089B2F0708BF
:107B600060CC002087300708BE300708962F070832
:107B70008B2F0708DD2F0708EB2F07086C2F07084E
:107B80007F2F0708A32F0708B32F0708C22F070866
:107B9000CF2F07089C300708AC3007085D30070876
:107BA0002DE9F04F2DED028BA3B0BF4B0393BF4BDC
:107BB0000293BF4B0193BF4BBF4AC049C0480093DB
:107BC000C04BC14CC14DC24FFCF792FAC149C248EB
:107BD000FCF78EFAC14BC24819684FF47A73B1FBB7
:107BE000F3F1FCF785FA06A8F6F76EF906A916A8D0
:107BF00045F0E2FB16A9BB48FCF77AFA22F01EFA20
:107C00006423B0FBF3F103FB110094F8FD3005EBA6
:107C1000830382B2D3F87435009394F8FC30B248F1
:107C200089B2FCF765FAB14BB1481968B14BB1FBA9
:107C3000F3F1FCF743FAD7F81C80002605F28459CB
:107C400004F1FE0A05F5B46B0123B34013EA080FF3
:107C50000BD059F8263043B11AF806205BF82610ED
:107C600053F82220A448FCF729FA0136072EEBD15D
:107C7000FCF7A2F9A1489F4EFCF7C4F909A8F2F756
:107C8000AEFC09999E48B1FBF6F1FCF731FA0A996E
:107C90009C48B1FBF6F1FCF72BFA0B999A48B1FB23
:107CA000F6F1FCF725FA0C999848B1FBF6F1FCF7D0
:107CB0001FFA22F0CFFB05EB8000D0F8C815059124
:107CC00022F0D2FB05EB8000D0F8C88522F0DCFB67
:107CD00005EB8000D0F8C89522F0FAFB05EB800098
:107CE000D0F8C8A522F018FC05EB8000D0F8C8B584
:107CF00023F0DEFC05EB8000D0F8C86522F040FCE4
:107D000005EB80004246D0F8C83505998048CDE99A
:107D10000263CDE900AB4B46FCF7EAF97D4B1B68EB
:107D2000DA031CD57C4B93F80080B8F1000F16D015
:107D30007A48DFF84892DFF848A24146FCF7D8F9C4
:107D40000026B9F90220314650460136FCF7B6F953
:107D5000F3B2434509F11009F3D3FCF72DF90020E4
:107D6000FEF76CFE6E4B6F4A1E886F4B6F491B68A7
:107D70006F48DFF810A2DFF81092DFF81082DFF80A
:107D800010B2C3F500739B00FCF7B2F9694A6A4B65
:107D90006A48D31A6A4AB6B231461288FCF7A8F983
:107DA0006848FCF72FF904265AF8041B6648FCF7CC
:107DB00085F96648FCF7CEF819F8011B002940F058
:107DC000EB816348FCF7C6F86248FCF7C3F858F843
:107DD000041B002940F0E4815D48FCF713F9013EE3
:107DE000E2D1398C5C48FCF769F95C490A6F5AB1F9
:107DF00007EE902ADFED5A6AF8EEE77A86EEA77A68
:107E0000FDEEC77A17EE902AD1F800315BB107EE8C
:107E1000903ADFED536AF8EEE77A86EEA77AFDEE48
:107E2000C77A17EE903A896A59B107EE901ADFEDDA
:107E30004C6AF8EEE77A86EEA77AFDEEC77A17EE7F
:107E4000901A0091B4F80C114648474F474EDFF89E
:107E50004491FCF74DF94648FCF77CF83B684FF03D
:107E600001081E40002E40F09F81FCF7A5F83B68FA
:107E70005B0140F191800DA810F0B8F9002840F0A6
:107E80008B800D9B40F2912293429DBF39480C227A
:107E900002FB0300304616A910F04EF8364816A92A
:107EA000FCF733F978E000BF2A4A07089E2C070840
:107EB000A72C0708B02C0708202007083320070844
:107EC000852C07087D2C070858DD0020A09D06089A
:107ED000706E0120BC2C0708CE2C07081C2D00203A
:107EE000003107081A3107082B310708000100206C
:107EF0005031070840420F00603107086831070819
:107F00007D3107088F310708A1310708B331070811
:107F1000C5310708686E0120646E01201832070819
:107F2000482E0020000002206C34002000180000C1
:107F30004C3207080080000800400008843207081F
:107F40009A3E0020BE320708D1320708D93207080E
:107F5000772D0708EF320708F9320708C808002014
:107F60000024744909330708C06D0120C0FFFD7F5C
:107F700046330708C47E06085D330708C43D002069
:107F80003D32070878A306085DDE0020E860002087
:107F9000E83207087D2D07083E68370509D500201F
:107FA0003CF084FA042840F012819F499F48FCF776
:107FB0009FF89F48FBF7CEFFD4F81011002900F07E
:107FC00019810B7B4A7B9B488968FCF777F8FBF7A4
:107FD000F3FF9948FBF7BEFFD4F81401FBF75DFFF0
:107FE000002800F00B810DA9D4F81401FBF796FFCF
:107FF0009DF848109DF85430149A9048FCF75EF8AC
:10800000119911B18E48FCF759F80F9911B18D48AB
:10801000FCF754F8FBF7D0FF8B4B1B68180640F1B8
:10802000AC802BF053FA002800F0A7808748FBF7BC
:1080300091FF8748D0F8143DB3F5487F00F0EC80FD
:1080400000F2E080B3F5167F00F0E880B3F52F7FF3
:1080500000F0E6807F49804AB3F5FA7F08BF1146F9
:1080600090F8182D90F8193D90F81B0D072896BF31
:1080700005EB80000020D0F84C0600907748FCF714
:108080001DF800210F202BF02DFA10B17448FCF7D9
:1080900015F8744E9FED748AFBF78EFFF1797348E3
:1080A000FCF726F8738C07EE903AF8EEE77AC7EE05
:1080B000887A17EE900A47F0E7FC02460B466C48B8
:1080C000FCF716F8F38B07EE903AF8EEE77AC7EE76
:1080D000887A17EE900A47F0D7FC02460B466548AF
:1080E000FCF706F8338C07EE903AF8EEE77AC7EE25
:1080F000887A17EE900A47F0C7FC0B4602465E48A6
:10810000FBF7F6FF5D48FBF7F3FF5D48FBF77AFFEF
:108110005C48FBF777FF94F8183119070AD594F8F3
:10812000202194F821115848C2F3C002C1F3C001C4
:10813000FBF7DEFF94F818315A070AD594F820218E
:1081400094F821115148C2F38002C1F38001FBF77A
:10815000CFFF94F818319B070AD594F8202194F8A2
:1081600021114B48C2F34002C1F34001FBF7C0FFAD
:1081700094F81C114748FBF7BBFF474B1B7833B102
:1081800005EB83054548D5F86C16FBF7B1FF23B026
:10819000BDEC028BBDE8F08F5846FBF78FFF13E66E
:1081A0005846FBF7A5FF1AE696FAA6F3B3FA83F34F
:1081B00008FA03F2052B26EA02067FF753AE05EB19
:1081C00083034846D3F8D015FBF778FF4AE6012829
:1081D00001D13349EAE6022807D1760303D53148B5
:1081E000FBF786FFE5E63049E0E603287FF4E1AEE1
:1081F0002E48F5E72E48FBF7ADFEE8E62D48FBF7E5
:10820000A9FE07E7B3F5617F0CD012492A4AB3F5FE
:108210007A7F08BF114623E7284921E728491FE74D
:1082200028491DE728491BE7713307087C2D0708FB
:10823000E6330708EC330708053407080B34070852
:1082400029340708323407089C3E00204E340708C2
:1082500060CC00209B2F0708D5300708543407084E
:108260007B3407082C7100200000C8429B340708AB
:10827000A6340708B1340708BE340708CB34070812
:10828000E0340708013507080D3507081F350708D2
:108290003035070842350708868000205935070821
:1082A0008D330708A1330708BA330708D33307080B
:1082B000F933070841340708F8300708EA3007089F
:1082C000DC300708E3300708F13007082DE9F341F7
:1082D0001A481B4C1B4E1C4FDFF87080FBF708FF41
:1082E0000025E2792168A37994F808C006EB8202A0
:1082F00001F13F41D2F88406A28806EB830301F521
:108300007E01890AB2FA82F2D3F8E0314131C2F13A
:108310001F02BCF1000F0CD0CDE900C04046FBF7B6
:10832000E7FE0135312D04F10C04DAD102B0BDE8CD
:10833000F08100903846FBF7DBFEF2E77335070863
:108340001C750020A09D06089F3507088F3507087B
:1083500010B5F3F7CDFC124CD0B11248FBF772FE0A
:108360001148FBF7F7FD2068F7F766FA4FF47A70CB
:10837000FBF7D0F80D4B18681EF0D6FE0C4B1878A2
:10838000F8F79CFD02210120F2F706FEF9F70CF93F
:108390000848FBF7DFFD2068BDE81040F7F74CBA4E
:1083A00020820020AD350708922D07082C8200207E
:1083B000646E0120CD3507082DE9F0410446254EB5
:1083C000254DDFF8B0800020FDF7E6FD2348FBF7E0
:1083D00039FEB17822480131FBF78AFE2146202080
:1083E000FBF72EFF1F48FBF72DFEB3781E4A4FF414
:1083F000D67707FB0353D3ED057AF5EE407AF1EE1D
:1084000010FA0CBF012100212046FBF727FEB178AE
:108410007943143108EB010220462944FCF752FD50
:108420001248FBF70FFEB378114A07FB03532046AF
:10843000B3F9D610B1FA81F14909FBF70FFEB17813
:108440007943D43108EB010220462944BDE8F041CC
:10845000FDF740BD5885002080910020FC350708BD
:108460000A3607081D360708303607083F36070862
:1084700052360708AC830020A0F2DC50164BB0F552
:10848000FA7FA8BF4FF4FA70984210B5B8BF1846EB
:108490000C46114642F0FCF900B207EE900A9FED3F
:1084A0000F7AF8EEE77AE4B287EE870AFBEE096A04
:1084B000E0EE006A07EE904A9FED097AF8EE677ADF
:1084C000A7EEA67AF3EE097A20EE070A80EE270AD5
:1084D00048F068FE00B210BD0CFEFFFF0000C8426D
:1084E00000401C452DE9F041DFF8EC81744DD8F8CF
:1084F00000309F6A734B1B6813F0100F86B040F07A
:10850000A88095F82430002B00F0A3806E4CD4F89E
:108510002C3104F592709847002800F09A8094F866
:108520008331002B43D1022385F84430B4F98431E0
:1085300007EE903AB4F98631F8EEE77AC4ED537A53
:1085400007EE903AB4F98831F8EEE77AC4ED547A40
:1085500007EE903AF8EEE77AC4ED557A5B4903AA44
:10856000A1F10C0042F0B0FE03A994F8682108467E
:1085700021F016FF03A821F0D5FE94ED4F0A5449CF
:10858000534C03A842F0ADFE04F178080026B4EC89
:10859000010AD5F8243584ED020A40469847013691
:1085A000032E04ED010A08F5C078F0D151E095F8EA
:1085B0004430012BD2D1D4F840310393D4F8443164
:1085C000049303A9D4F84831059305F14400F5F765
:1085D00067F895F84430012B4FF0000669D0022B64
:1085E0005FD0039604960596DDED037A9DED047A3F
:1085F000DDED056AC4ED537A84ED547AC4ED556A15
:10860000FDEEE77ABDEEC77AFDEEE66A17EE903A28
:1086100017EE102A16EE901A1BB212B209B2A4F885
:108620008431A4F88621A4F888110120CDE9002125
:108630000421284AF5F7CAF9D8F8003000200021B3
:10864000C3E90C01C3E91001C3E90E01EE622E6318
:108650006E63EB695B0621D51B4C94F8D831EBB106
:10866000FE173146384647F077FED5ED0B6A94ED9C
:108670007B7A07EE900AA7EEA67AD4E97E32D5ED92
:108680000C6A84ED7B7A94ED7C7ADB19A7EEA67AEE
:1086900046EB0206C4E97E3684ED7C7A06B0BDE87E
:1086A000F081EB6D03936B6F0493D5F88C300593D9
:1086B0009AE7C4F84C61C4F85061C4F85461C5E746
:1086C000706E0120C06D012058DD0020A4DE002066
:1086D0009C6E01205F360708606E0120034B01226B
:1086E00083F80822022283F80922704758DD00200F
:1086F00070B50D4E35782D1A18BF01250328044694
:1087000034BF044600242046F6F7BEF8074A34700A
:1087100002F50473C4EB041403EB4403C2F80C32F7
:108720001AF048FC284670BD5885002058DD00200E
:10873000022810B50C4618D8FFF7DAFF0B48FBF7F4
:1087400081FC0B4B0B4819780131FBF7D1FC21461A
:108750000820FBF775FD21461020FBF771FD21462F
:108760002820BDE81040FBF76BBD10BD863607081A
:10877000588500209636070838B5154C154DAC4283
:1087800013D30020F6F780F8134820F017FF134AA0
:10879000136843F48003136000BF114B1878FFF790
:1087A000A7FFBDE838402CF0D9B9B4F90230002B4E
:1087B0004FF00001204607DAF6F756F8012120466F
:1087C000F6F752F802212046F6F74EF81434D6E7B1
:1087D0002082070870870708AB3607089C3E0020F8
:1087E0005885002010B504460A48FBF7B3FBFFF795
:1087F000C3FF20F0C7FEF5F705FF20F0CDFE064BC6
:108800000649002220461A70FDF7A4FC08B9FEF7BD
:1088100083FD10BDB4360708258200207A3707088B
:1088200010B5064B5C78241A18BF0124032828BF12
:108830000020587021F05EFB204610BD58850020B6
:10884000022810B50C4610D8FFF7EAFF0748FBF7DF
:10885000F9FB074B074859780131FBF749FC2146E2
:108860001820BDE81040FBF7EBBC10BDCA36070866
:1088700058850020DA3607082DE9F04F0D468DB0F7
:10888000B6490746FDF766FC0646002840F0B7806B
:10889000B3493846FDF75EFC0646002840F0B1803B
:1088A000B0493846FDF756FC0646002840F0AB803C
:1088B000AD493846FDF74EFC0646002840F0A5803D
:1088C000AA493846FDF746FC002806460ABF01249F
:1088D00010243E466D4205F020052C43A44DA54FC3
:1088E00095F800A095F8029095F80180DFF8F8B2AD
:1088F0005F45C0F08C80FFF73FFF5046FFF7F8FE62
:108900004846FDF749FB4046FFF78AFF9A49304643
:10891000FDF720FC08B144F0400414F0110301936A
:1089200000F05C829548FBF78DFB0020FEF772FAA1
:108930009348FBF787FB9348FBF764FB04F0300395
:10894000302B02D19048FBF77DFB9048904FFBF70E
:1089500079FB9048FBF776FB4FF0FF338E4A8F4947
:108960002046FDF763FD8E48FBF76CFB8D4A8E4970
:108970002046FDF7F5F98D48FBF764FB8C4A8D49DD
:108980002046FCF7E5FE8C48FBF75CFB8B4A8C49E4
:108990002046FCF7D5FD8B48FBF754FB8A4B1E683D
:1089A0008A4BD3F800908A4B00939B4669EA0603F2
:1089B0004FF0000A02935BF8043B002B34D01A7886
:1089C000D2B1029A03934FF0010808FA0AF812EAAA
:1089D000080F14BF012100213A462046FBF758FB3F
:1089E00066EA090212EA080F039B3A4614BF012106
:1089F00000212046FBF732FB0AF1010ADBE70124E4
:108A000068E7022466E7082464E7042462E77B88B9
:108A1000C3F30B021B04D7E9011048BF02EB42026B
:108A20004CF03EFB143763E71F46DFF8C0A169EA4C
:108A300006030293009B53F804BB0093BBF1000FA5
:108A400025D09BF8002002B34FF0010808FA07F880
:108A500019EA080F0BD066EA090212EA080F5B4612
:108A6000524614BF012100212046FBF711FB16EAF4
:108A7000080F0AD0029B13EA080F52465B4614BF48
:108A8000012100212046FBF7E9FA0137D2E75148DE
:108A9000DFF85CA1FBF7D6FA4F4AD2F800804F4AC4
:108AA000126888EA02025E46D343DFF848B10093B9
:108AB000009B0127B7403B4214BF4FF001094FF024
:108AC000000918EA07070CBF52465A46304603927F
:108AD0001AF030FE039A0290034649462046FBF7FF
:108AE000D7FA0136002F0CBF5A465246029B494620
:108AF0002046FBF7B3FA182EDAD13948DFF8F8A090
:108B0000DFF8F880DFF8F890FBF79CFA354BD3F8E4
:108B100074720026F3B20AEB8302D2F854B3BBF1AD
:108B2000000F6FD00121994039405B460CD04A4676
:108B300000212046FBF792FA5B464A460021204678
:108B4000FBF7A6FA0136E5E7424620460091FBF71F
:108B500085FA00995B464246F1E700BF04370708F3
:108B600086360708FC350708CA3607080B3707089A
:108B700058850020208207080F3707081C37070890
:108B8000243707083C3707084837070883370708A2
:108B9000D33707088D37070878800020A894002075
:108BA0009D370708EE8A00207E8B0020AD3707082E
:108BB000A0870020FC8E0020B63707089086002092
:108BC0005C8F0020CA370708A03E00209C3E002092
:108BD00070A00608EA3707089C940020B0800020A7
:108BE000F137070858DD002070870708DF370708CE
:108BF000F9360708EF360708A09D0608063807086B
:108C0000FA3707089848FBF71DFADFF82CC3974896
:108C1000974ACDF820B0CDF810B0042601271CF8F3
:108C2000013F10F801EB03F13001694401F820EC39
:108C300012F8011F01F13008E84408F810EC002F89
:108C400000F0EF80A3EB010EDEF1000141EB0E011D
:108C5000013E0F46E3D1874A8DF8146008AB2046E9
:108C6000FBF716FA04AB3946824A2046FBF7F6F9C1
:108C70008148FBF7E7F9814A81492046FBF714FF59
:108C80008048FBF7DFF9804A80492046FCF70CFE5C
:108C90007F48FBF7D7F97F4A7F492046FCF728FF3A
:108CA0007E48FBF7CFF9784A78492046FCF7B8FFB1
:108CB0007B48FBF7C7F97B4A7B492046FBF728FE38
:108CC0007A48FBF7BFF97A4A7A492046FCF70EF852
:108CD0007948FBF7B7F9794A79492046FCF718FA41
:108CE0007848FBF7AFF9784A78492046FCF7B0FAA4
:108CF0007748FBF7A7F97749204641F0CBFC764847
:108D0000FBF7A0F94FF0FF331A467449204641F0B3
:108D10004DFD7348FBF796F94FF0FF33714A7249E6
:108D20002046FDF733FA7148FBF78CF9704A714918
:108D30002046FDF7B3FA7048FBF784F96F4A704993
:108D40002046FDF7EBFA6F48FBF77CF96E4A6F4956
:108D50002046FDF725FD6E48FBF774F921463046A5
:108D6000FBF76EFAE7065ED52146304695F800908F
:108D700095F802806F78FFF7DBFC21460120FFF7B2
:108D8000D7FC21460220FFF7D3FC2046FFF714FB57
:108D900021463046FFF754FD21460120FFF750FDE4
:108DA00021460220FFF74CFD4846FFF7A1FC404654
:108DB000FDF7F2F83846FFF733FD5648FBF742F966
:108DC000554809F10101FBF793F9544808F10101F5
:108DD000FBF78EF95248791CFBF78AF90026A007A9
:108DE00003D528782146FFF7A3FC210704D5AB78EB
:108DF00013B92046FFF7E0FA620703D568782146E9
:108E0000FFF71EFD019B13B14648FBF71BF92EB17E
:108E10004548FBF717F94548FBF7F4F8444C454D36
:108E20001CE0394614E728782146FFF781FCAB782F
:108E300013B92046FFF7C0FA68782146FFF700FD16
:108E40000126CCE76388C3F30B021B04D4E90101BC
:108E500048BF02EB42024CF023F91434AC42F1D388
:108E60000DB0BDE8F08F00BF1338070868A20608F0
:108E700000D900202938070830380708048300206B
:108E8000CC93002036380708008800200E8C002084
:108E90003B380708808A00208E8E0020453807085E
:108EA0005438070831820020FC93002060380708FE
:108EB00034830020549300207738070880850020F1
:108EC000709100208838070890850020709000205D
:108ED00094380708F8DF0020B338070858E9002065
:108EE000C4380708B4CC0020A0EE0020D73807080B
:108EF000B4D10020A0F30020F538070814D20020D8
:108F000000F400201239070884D2002070F40020F9
:108F100004370708273907084A3907085D39070861
:108F20006E390708813907089A390708B0390708E8
:108F30002082070870870708D4DF002000219BE407
:108F4000012199E42DE9F04FCB4CDFF868A385B0FF
:108F5000CA4B9C42C0F07E81C94CCA4E2078FFF7B4
:108F6000C7FB6078FFF75CFCA078C74CFDF714F8EE
:108F7000B6F89421B6F87031C44804329A42A4BFBE
:108F80005A1FA6F89421B6F89621043A9342A8BF36
:108F9000053394F83127A8BFA6F8963194F83037F6
:108FA0009A4224BF002384F83037F5F71FFCB84BF2
:108FB0001A68B84B934312D100212520F0F726FF01
:108FC000054660B100212720F0F720FF38B1026884
:108FD0002B689A4203D14FF48030F5F707FC002745
:108FE000DFF8B4823D464FF0FF0948F2B83A58F82E
:108FF00027004308810801F0333103F077330B4435
:10900000C10801F01131C31A5B1A03EB131310F0FE
:10901000010203F00F33B3FBF9F1C1EB012118BFDB
:109020000135A3EB010318BFEDB2012B40F28A8199
:10903000022B00F07E8198480D2144F0B1F9B4F87C
:109040006037B4F85E27643B9342A8BF1346A4F888
:109050005E3700BF94F8D63713B9082384F8D637A3
:1090600000200FF0C3F8DFF850B2DBF80030002822
:1090700000F0718123F08063CBF80030D6F80C3219
:10908000029315F0F7FD074615F0DEFDBBB2019324
:10909000029B1978C21B4A43642192FBF1F212FA37
:1090A00087F2A4F8EC277D4A00261D78A6EB050878
:1090B0000FFA88F8B8F1000FA94640F34F81C5F1C7
:1090C0006405EDB293F801A00392029315F0BCFD84
:1090D00008FB08FC0AFB0CFCCAF1640A15FB05F549
:1090E00009EB89099CFBF5F555440A2108FB05F5B8
:1090F00095FBF1F505EB49090FFA89F9C01B4FF40F
:109100007A7300FB09F90E4499FBF3F9019B039A6A
:10911000B6B299446E2E22F8029B029BC5D120F074
:1091200003FF18F025FE302200215D484DF0DAF8EB
:109130000EF030FE94F8243853BB5A49C4F8303846
:1091400091F83E00C4F834386422C82512FB005060
:10915000C4F8280891F83F00C4F8383812FB0052D0
:10916000C4F82C28C4F83C3891F84120C4F84038A1
:10917000C4F8443884F8513884F8523884F82538D3
:10918000C4F854384FF07A7384F85028C4F858382B
:10919000DBF8003044499B060A6800F1E280B4F82D
:1091A0002607B4F824370343B4F8280703431BB257
:1091B000002B40F0D680B4F92A37B3F5805F40F039
:1091C000D080B4F92C37B3F5805F40F0CA80B4F991
:1091D0002E37B3F5805F40F0C48022F400720A603D
:1091E00020F0BAFDB4F85C18DFED307A304A07EEB3
:1091F000101AB8EEC77AB4F85E18C7EE276A02F5FF
:10920000A86307EE101AB8EEC77AC3ED006AC7EE7E
:10921000276AB4F8601807EE101AB8EEC77AC3EDE3
:10922000016AC7EE276AB4F8621807EE101AB8EEA2
:10923000C77AC3ED026AC7EE276AC3ED036A94F8E2
:10924000643882F8503517F095FA05B0BDE8F04F54
:109250003BF0D6B9B4F90230DFF86080002BA7BF2D
:10926000002637460326012700257919C9B28E4208
:1092700026D214346CE600BF2082070870870708E6
:109280005885002058DD002050EE00202063140691
:109290009C3E0020400001000483002098730120C0
:1092A00040F6002060CC0020686E012000401C4683
:1092B000706E012001400008C06D01200080000890
:1092C000534603F1060BC3454ED21A88002A4BD0F1
:1092D00003EB020CC44547D2052A45D92088B3F8D0
:1092E00002E0C0F30B00864521D1587900F003005D
:1092F00088421CD12946204693F804900192F5F744
:10930000B3FA2188019AB9EB113F0ED161886068E8
:10931000C1F30B03063A9A42A8BF1A46090448BF94
:1093200003FB050059464BF0BBFE01359DE7634644
:10933000C7E712B110EA0A0F04D142F0EDFC002891
:109340003FF479AE03370C2F7FF451AE013D022D6F
:109350007FF675AE6FE643F080638DE608BF0125AA
:10936000B0E642F400723AE729462046F5F77CFA67
:10937000DBE710B5144C94F80932022B18D120F019
:1093800001F9F5F73FF9FFF7DDFD20F005F90120C0
:109390001AF0B4F90D4B0E491B6803F59C530022DB
:1093A000083384F80822C1F86C3884F8092210BD0B
:1093B000012BFCD120F0E6F8F5F724F920F0ECF8C9
:1093C000002384F80932F2E758DD00201C2D00202C
:1093D00050EE002010B50446FFF78AF938B120F0AE
:1093E000D1F8F5F70FF9FFF7ADFD20F0D5F8601CC7
:1093F000C0B2BDE810401AF081B938B50C4D044632
:109400002046FBF731F838B10A4B0B481978BDE814
:1094100038400131FAF76CBE2046F5F791F8013873
:10942000022804D8C0B2FFF7D5FF2C46E8E738BDC4
:109430002A4A0708588500204A39070810B504460B
:10944000FFF7EEF938B120F09DF8F5F7DBF8FFF7FC
:1094500079FD20F0A1F8601CC0B2BDE810401AF000
:109460004DB938B50C4D04462046FAF7FDFF38B12A
:109470000A4B0B485978BDE838400131FAF738BE3D
:109480002046F5F75DF80138022804D8C0B2FFF78E
:10949000D5FF2C46E8E738BD2A4A07085885002042
:1094A0006E39070810B50446FCF776FD38B120F098
:1094B00069F8F5F7A7F8FFF745FD20F06DF8601C97
:1094C000C0B2BDE810401AF019B970B50C4E044690
:1094D0002046FAF7C9FF054638B10A4B0A48997881
:1094E000BDE870400131FAF703BE2046F5F728F8D1
:1094F000012804D12846FFF7D5FF3446E8E770BDC0
:109500002A4A0708588500205D39070838B5144DE8
:10951000EC69630702D53DF02FFFF8B1200703D5B2
:10952000104B1B68D90519D5A20602D53DF0D4FF12
:10953000A0B13DF0B5F910B9FCF75EFD68B995F83A
:109540005435012B04D1A30702D5FCF755FD20B9F2
:1095500022F02CF980F00100C0B238BD0120FCE7F8
:10956000706E0120686E01202DE9F0418B4D2C6852
:1095700014F0040705D0BDE8F04101210020F7F701
:10958000C7B8FFF7C3FF864E002800F0A28044F45E
:1095900000742C6086F8707896F852382C68012B8D
:1095A00096F8723814BF44F4802424F480242C608C
:1095B0003BB90EF097F9002800F0998024F40024BC
:1095C0002C603BF059FA48B10A202C680EF072F971
:1095D000002800F08F8044F400042C60714BDFF809
:1095E000E8811F682C68B8F82030390754BF44F46C
:1095F000807424F48074632B8CBF44F4806424F45E
:10960000806400202C603AF051FF002875D044F4AB
:109610000064D8F81C301A0772D5F80570D444F4E9
:10962000805499072C606ED5BA056CD4FCF7E4FC25
:10963000002868D044F400542C6022F051F800282F
:1096400064D144F4004412202C600EF0F1F900289B
:109650005FD044F480341B202C600EF0E9F9002820
:109660005AD044F080742C60F9F762FE4E4A52E9F9
:109670000232C01A4D4B61EB02015A7A022A4ED8CF
:109680004B4B4C4C002A18BF234698424A4B2C683F
:1096900093F82A3071F1000134BF44F0005424F0F3
:1096A00000542C6093B12A200EF0C2F900283DD05E
:1096B00096F88038002B40D0B6F8762832B13F4B70
:1096C000D6F884181B685B1A934236D224F0805473
:1096D00035E096F8703824F400742C60002B7FF489
:1096E0005BAF012086F8700819F0D6FE54E744F409
:1096F000002465E724F400046FE724F4006488E79D
:1097000024F480548DE724F4005495E724F40044B5
:1097100099E724F480349EE724F08074A3E7284B73
:10972000234C033A012A88BF2346AEE7012386F87B
:109730008038224B1B68C6F8843844F0805463009C
:109740002C6006D500200EF073F910B924F0804487
:109750002C6000200EF06CF92C681A4B1C4216D0BD
:10976000B8B144F480442C602A681A4214BF012323
:1097700000235B0086F88838F9F7DAFDD6F88C38D4
:10978000C01A002808DBBDE8F0411EF070BA0028BE
:10979000EAD124F48044E6E7BDE8F081C06D012001
:1097A00050EE0020686E0120D0F60020B08000202E
:1097B00000171100407E050060CC00201C2D002009
:1097C00060CC0500C0FFFD7F706E01202DE9F84FD1
:1097D0008E4D95F825082DED028BB0EE408A80B3B2
:1097E0008B4E8C4F00244FF0060805F5026995F862
:1097F000503808FB0373234493F8023753B1012B0D
:109800000DD00134042C06F10206F0D1BDEC028B20
:10981000BDE8F88F09EB44039B8E3380F1E7032CFE
:1098200001D00023F9E77C4B1B68DB0406D415F05C
:1098300021FA00B2794BA3F8BA05E2E740F2DC5016
:10984000F8E7764C1FF0DAFE754BD4F8BCA5D3F8D8
:109850000C7295F890881AF4807B14BF7E7C3E7B56
:1098600042463146FEF708FEA4F8B40581460120C1
:109870001FF0C4FE42463146FEF7FEFD8046A4F8C6
:10988000B60502201FF0BAFEBBF1000F7FD0B97CF5
:1098900095F89128FEF7F0FD464236B2A4F8B86577
